:0A0000000C94A2000C9400000C9474
:10000A0000000C9400000C9400000C9400000C9466
:10001A0000000C9400000C9400000C9400000C9456
:10002A0000000C9400000C9400000C9400000C9446
:10003A0000000C9400000C9400000C9400000C9436
:10004A0004010C9400000C94D1000C9400000C9450
:10005A0000000C9400000C9400000C9400000C9416
:10006A0043460C9400000C9400000C9400000C947D
:10007A0000001027E80364000A00010000100001D4
:10008A0010000100000000000A000400FBFFFBFF53
:10009A00FBFFFBFFE8030000000000000000000077
:1000AA000000000000000000000000000000000046
:1000BA000000000000000000000000000000000036
:1000CA000000000000000000000000000000000026
:1000DA000000000000000000000000000000000016
:1000EA000000000000000000000000000000000006
:1000FA0000000000000000000000000A0A0A0A0AC4
:10010A000A0A0A0A0A0A0A0A0A0A0A00070002006E
:10011A0002008E000200040090000100090592000E
:10012A0001004D07940008007C07960002000C08A5
:10013A009E000100340816010000F894EE27EFBB78
:10014A00F1E0F5BFE5BF8DE0A2E0BB27ED938A950C
:10015A00E9F780E090E1A0E0B1E0ED930197E9F7DB
:10016A00E8E1F1E085919591009761F0A591B5914B
:10017A0005901590BF01F00105900D920197E1F7E6
:10018A00FB01F0CFE4E0EEBBEFEFEDBFE0E1EEBF45
:10019A00C0E0D5E00C945001AA93EA93FA93EFB722
:1001AA00EA931A930A931091C0000091C600E12FB6
:1001BA00EC71E9F4E0912F08EF5FE0932F08E1502A
:1001CA00F0E0E25EF74F0083A0912F08A13119F405
:1001DA00E0E0E0932F08A0913108AF5FA0933108C7
:1001EA00A13129F4E0E0E0933108689432F80991EA
:1001FA001991E991EFBFF991E991A9911895AA93FB
:10020A00BA93EA93FA93EFB7EA93E0910507F0916C
:10021A0006073196E0930507F0930607A0910507B4
:10022A00B0910607A83BE0E0BE0719F4E1E0E093CD
:10023A004505A0910507B0910607A037E1E0BE0782
:10024A0041F4E2E0E0934505E0E0E0930507E0933E
:10025A000607E991EFBFF991E991B991A99118952A
:10026A00AA93E881E0937C0088E28A95F1F7E0910D
:10027A007A00E064E0937A00E0917A00E071E1F3B9
:10028A00E0917A00E061E0937A00E0917800F091E1
:10029A00790021960895EF97EE9785E7A8E0B0E0F8
:1002AA00E0EAF0E00E94465CFF2411E001E0E0E8A9
:1002BA00E0936100E0E0E0936100E1B9E2B9EAEDC0
:1002CA00E4B9E5E2E5B9ECE3E7B9E3ECE8B9E0EF74
:1002DA00EAB9EFE0EBB9E1EAE4BDE3E0E5BDE0E06D
:1002EA00E6BD0E94C647E1EAE0938000E3E0E093BE
:1002FA008100E0E0E0938500E0938400E0938700CA
:10030A00E0938600E0938900E0938800E0938B00F5
:10031A00E0938A00E093B600E1EAE093B000E4E0FB
:10032A00E093B100E0E0E093B200E093B300E09321
:10033A00B400E1E0E0936E00E0E0E0936F00E09348
:10034A007000E0936900EDBBE0936800E093C000A1
:10035A00E8E9E093C100E6E0E093C200E0E0E09360
:10036A00C500EDE4E093C400E0E0E093C900E0E8F2
:10037A00E0BFE0E0E0937F00E0937E00E0937C0042
:10038A00E6EAE0937A00E0E0E0937B00ECBDA4E6C5
:10039A00B0E00E94A7457894299AA4EFB1E00E94A0
:1003AA0075580E94CA47A1E00E94D645A0916405EB
:1003BA00A03849F40E94DA47E0E4E09367050E9416
:1003CA00E2470E94E9470E94F247A0E00E94D64510
:1003DA00A0E03799A1E00E940448A0916405EFEFDC
:1003EA000E94A65AE02909F4D7C00E94DA47E2E33C
:1003FA00E0936705E0E5E0936805EEE1E0936905BF
:10040A00E3E2E0936A05E2E3E0936B05E4E6E09356
:10041A006C05E0E0E0936D05E2E3E0936E05EAE047
:10042A000E940948E3E0E0937105E8EEE093720563
:10043A00E4E6E0937305E09374050E940F48E1E057
:10044A00E0937905E2E2E0937A05E1E0E0937B0547
:10045A00EAE0E0937C05E1E0E0937D05E0E0E093EB
:10046A007E05E6E9E0937F05E9E0E0938005E4ECA8
:10047A00E0938105E3E0E0938205E4E80E941948ED
:10048A00E2E0E0938605EEE7E0938705E0E0E0939B
:10049A008805E2E40E942148E4EBE0938C05EAE057
:1004AA00E0938D05E1E0E0938E05E2E00E942948A1
:1004BA00E1E0E0939805E0E0E0939905E1E0E0935C
:1004CA009A05E0E00E943D48E4E2E093A005E0E0FE
:1004DA00E093A105E093A205E093A305E1E00E9461
:1004EA004948E4EA0E946548E2E3E0936A05E0E0ED
:1004FA00E0936B05EFEFE0936C05E0936D05EEE199
:10050A00E0936E05E0E00E9409480E946F48E0E52A
:10051A00E0937305E7E4E0937405E0E50E940F4871
:10052A000E947548E0E0E0937C05E0937D05E09346
:10053A007E05E0937F05E3E0E0938005E8EEE09333
:10054A008105E0E0E09382050E941948E0E0E0932B
:10055A008605E0938705E09388050E942148E0E03C
:10056A00E0938C05E0938D05E0938E050E9429485F
:10057A00E0E0E0939805E6E9E0939905E0E0E0938E
:10058A009A05E6E90E943D48E0E0E093A0050E9452
:10059A007D48EDE30E948448369924C00E94904821
:1005AA00E0E00E946548E0E0E0936A05E0936B05AD
:1005BA00E0936C05E0936D05E3E0E0936E05E8EEE9
:1005CA000E9409480E946F48E0E0E0937305E093B7
:1005DA0074050E940F480E9475480E947D48E8E110
:1005EA000E9484484A9912C00E949748E0E0E0932A
:1005FA006605E09367050E949E480E94E947AAE0C3
:10060A00B0E00E947558E1E0E0935F05189905C0D3
:10061A00689424F8E1E0E0936005689426F8E0E243
:10062A00E09317050E94A548E8ECF0E00E94AC4868
:10063A00E0EDF7E00E94B148E8ECF0E0E0934E0705
:10064A00F0934F070E94F247A1E40E94D645E09139
:10065A006405E0931805E0916505EBABE09166054A
:10066A00E0931905E0916705E0931B050E94B648DF
:10067A00A0916805A0830E94BB48A0916905A08348
:10068A000E94C048A0916A05A083E0916B05E0939F
:10069A001C05E0916C05E0931D05E0916D05E09362
:1006AA002105E0916E05E0932605E0916F05F0E0E3
:1006BA000E94C548F0910907E0E00E94C548E09110
:1006CA007005F0E00E94CA48EA0FFB1F0E94C54865
:1006DA000E94CF48A0917105A0830E94D448A0919E
:1006EA007205A0830E94D948A0917305A083E09166
:1006FA007405EEAFE0917505EFAFFE01FD963396F6
:10070A00A0917605A083E0917705F0E0E9A7FAA722
:10071A00F9A5E0E0E9A7FAA7E0917805F0E0A9A534
:10072A00BAA5EA0FFB1FE9A7FAA7E0917905E093BA
:10073A003405E0917A05E0933605E0917B05E09374
:10074A003505E0917C05F0E0EB8FFC8FFB8DE0E056
:10075A00EB8FFC8FE0917D05F0E00E94DE48EB8F85
:10076A00FC8FE0917E05F0E0EDA7FEA7FDA5E0E095
:10077A00EDA7FEA7E0917F05F0E0ADA5BEA5EA0FC3
:10078A00FB1FEDA7FEA7E0918005F0E0EBA3FCA319
:10079A00FBA1E0E0EBA3FCA3E0918105F0E0ABA1B3
:1007AA00BCA1EA0FFB1FEBA3FCA3E0918205AEED0F
:1007BA00B7E00E94E3480E94EB480E94F4480E9476
:1007CA00FB48E0918305F0E00E94EB480E9404494F
:1007DA000E94FB48E0918405F0E00E940B49F091E9
:1007EA000F07E0E00E940B49E0918505F0E00E94C6
:1007FA001049EA0FFB1F0E940B49E0918605FF276B
:10080A00662777270E9415490E941E49E8E00E9440
:10081A006A5A0E941549E0918705F0E00E941E4934
:10082A000E9427490E941549E0918805E0935E05D8
:10083A00E0918905F0E00E942C49F0911907E0E067
:10084A000E942C49E0918A05F0E00E943149EA0FA2
:10085A00FB1F0E942C49E0918B05E0930805E0916B
:10086A008C05E0930A05E0918D05E0930B05E09174
:10087A008E05E0930C05E0918F05E0930D05E0915C
:10088A009005E0930E05E0919105AAEFB7E00E946A
:10089A00E3480E9436490E94F4480E943F49E09189
:1008AA009205F0E00E9436490E9404490E943F499D
:1008BA00E0919305E0932A05E0919405E0932B05D6
:1008CA00E0919505E0932C05E0919605E0932D05BE
:1008DA00E0919705E0932E05E0919805E0932F05A6
:1008EA00E0919905E0933005E0919A05E09331058E
:1008FA00E0919B05F0E00E944849F0912107E0E071
:10090A000E944849E0919C05F0E00E944D49EA0F97
:10091A00FB1F0E944849E0919D05F0E00E94524960
:10092A00F0912D07E0E00E945249E0919E05F0E027
:10093A000E945749EA0FFB1F0E945249E0919F0506
:10094A000E94335C31F8E091A005E0931105E09133
:10095A00A105E8AFE091A205F0E0EDA3FEA3FDA199
:10096A00E0E0EDA3FEA3E0936205E6E4E09363050D
:10097A000E949E48E2E0EA93E4E6F5E0FA93EA93FD
:10098A00A6E30E94D645E0916405F0E0ADA1BEA1C0
:10099A00EA0FFB1FEDA3FEA3E0916505E0934C056A
:1009AA00E0916605E0934D05E0916705E0934E05F9
:1009BA00E0916805E0931E05E0916905E093200542
:1009CA00E0916A05E0932205E0916B05E093230527
:1009DA00E0916C05E0931605E0916D05FF27662707
:1009EA0077270E945C490E9465490E946E49E091FE
:1009FA006E050E9472490E947549E0916F050E9436
:100A0A0072490E947549E09170050E9472490E94DC
:100A1A005C49E0917105E0935905E0917205E09314
:100A2A005A05E0917305E0935B05E0917405E09344
:100A3A005D05E0917505E0934605E0917605E09342
:100A4A004705E0917705E0934805E0917805F0E0E5
:100A5A000E947849F0912307E0E0E0932307F0939E
:100A6A002407E0917905F0E0A0911608B0911708E3
:100A7A00EA0FFB1F0E947849E0911608F0911708C7
:100A8A000E947D490E9486490E947D49E0917A052B
:100A9A00AAECB7E00E94E3480E948B490E94F448FE
:100AAA000E949449E0917B05F0E00E948B490E94E4
:100ABA0004490E9494490E949D490E94A6490E94A5
:100ACA00AD490E94C3590E9494490E94B3490E94A9
:100ADA00C3590E943F49F698F19831FE06C0C0906A
:100AEA007C05E0917D05E0930005E0917E05E093A9
:100AFA000A08E0917F05E0930B08E0918005F0E099
:100B0A000E94B949F0910C08E0E00E94B949E091CD
:100B1A008105F0E00E94BE49EA0FFB1F0E94B94915
:100B2A00E0918205F0E00E94C349F0910E08E0E0EE
:100B3A000E94C349E0918305F0E00E94C849EA0F88
:100B4A00FB1F0E94C349E0918405F0E00E94CD4951
:100B5A00F091A807E0E00E94CD49E0918505F0E018
:100B6A000E94D249EA0FFB1F0E94CD49E0918605F7
:100B7A00F0E00E94D749F0911008E0E00E94D749BE
:100B8A00E0918705F0E00E94DC49EA0FFB1F0E9412
:100B9A00D749E0918805F0E00E94E149F0911208F6
:100BAA00E0E00E94E149E0918905F0E00E94E6490F
:100BBA00EA0FFB1F0E94E149E0918A05F0E00E94DA
:100BCA00EB49F0911408E0E00E94EB49E0918B05B3
:100BDA00F0E00E94F049EA0FFB1F0E94EB49E09106
:100BEA008C05F0E00E94F549F0911808E0E00E94B7
:100BFA00F549E0918D05F0E00E94FA49EA0FFB1FE2
:100C0A000E94F549E0918E05E093EE05E0918F058B
:100C1A00E093C805E0919005E093EF05E091910516
:100C2A00E093F005E0919205E093F105E0919305D8
:100C3A00E093F406E0919405E093F506E0919505BA
:100C4A00E093F906E0919605F0E0ED8FFE8FFD8DB9
:100C5A00E0E0ED8FFE8FE0919705F0E0AD8DBE8D5F
:100C6A00EA0FFB1FED8FFE8FE0919805F0E0EF8F02
:100C7A00F8A3FF8DE0E0EF8FF8A3E0919905F0E08B
:100C8A000E94FF490E94044AA091F406A43618F073
:100C9A00E0E0E093F406A091F506A43618F0E0E04F
:100CAA00E093F506A8ADA43019F00E94094A02C0E3
:100CBA000E94174AE0933A050E94254AE1E0E09330
:100CCA004305E093F8066E2E0E94294AA091450535
:100CDA000E942F4AA0914505E2E00E94A65AE02907
:100CEA0009F405C3A13019F4E0E0E0934505A091A9
:100CFA000307B0910407E5E0F0E00E94ED5A0E2EDA
:100D0A00A0912905EEE00E94BF5AE02121F0E0916E
:100D1A002905EF5F03C023FC03C0E0E0E093290547
:100D2A00A0912905AE3011F4689423F8A0913305F7
:100D3A00A13029F4F69B02C0F69801C0F69AF79BF7
:100D4A0002C0F79801C0F79A0E94344A0E943D4AAD
:100D5A00E093EA07F093EB076093EC077093ED07D3
:100D6A000E94444AAEECB7E00E94494A0E94504AA7
:100D7A00A6EFB7E00E94494A0E94554A0E945E4A7D
:100D8A00E093CE07F093CF076093D0077093D10713
:100D9A00A091F607B091F7078091F8079091F907AB
:100DAA00E0E0F0E060E772E40E94C359E093F607DE
:100DBA00F093F7076093F8077093F9070E94654A62
:100DCA000E946A4A0E2E0E946F4A0E946A4AE021D5
:100DDA0061F1E091F607F091F7076091F8077091D9
:100DEA00F9070E94554A0E94C359E093F207F0930B
:100DFA00F3076093F4077093F5070E94744AA7E11A
:100E0A00B7E00E947D4AA091F207B091F307809162
:100E1A00F4079091F5070E943D4AE093D607F093B4
:100E2A00D7076093D8077093D9070E94824A0E9415
:100E3A008B4A0E94EB480E9425590E94FB480E9457
:100E4A00824A0E94944A0E942E5A0E2E0E94994A61
:100E5A00E8EEFDEF0E94E75AE021D1F00E94824AB3
:100E6A000E948B4AA091FE07B091FF07809100086B
:100E7A00909101080E949E4AE093FE07F093FF07B3
:100E8A006093000870930108A3E2B7E00E947D4ACC
:100E9A000E94824A0E948B4A0E94A34A0E942559B4
:100EAA00E0930208F093030860930408709305081E
:100EBA000E94AC4A0E94B54A0E949E4AA6EBB7E03D
:100ECA000E94B4580E94F15B0E94AC4AAAE0B0E0CA
:100EDA0080E090E00E942B5B0E94A34A0E94E9589E
:100EEA000E94085A70F0E0E0E0930208E0930308D9
:100EFA00E0930408E09305080E94C84A31960E94CC
:100F0A004849E091BE07F091BF076091C007709110
:100F1A00C1070E94824A0E94CD4AE0E0F0EA6CE8EA
:100F2A0077E40E94C359E093EE07F093EF076093CA
:100F3A00F0077093F1070E9436490E9425590E94D2
:100F4A003F490E94D24A0E941E49662777270E947B
:100F5A002B5BDF01CB01E091FA07F091FB0760916F
:100F6A00FC077091FD070E94055C0E949E4AA8E555
:100F7A00B7E00E94D74A0E94344A0E94235C3CF59B
:100F8A00A091EE07B091EF078091F0079091F107D9
:100F9A000E94DC4A7F936F93FF93EF93A091EA0735
:100FAA00B091EB078091EC079091ED070E94DC4A23
:100FBA00AF91BF918F919F910E94C359E093E60729
:100FCA00F093E7076093E8077093E90709C0E0E048
:100FDA00E093E607E093E707E093E807E093E90781
:100FEA00A091E907AA23AAF40E94E34AE0E0F0EC00
:100FFA0069E774EC0E94085A18F40E94EC4A08C087
:10100A000E94F34A0E947F58A0E6B7E00E94D74A9E
:10101A0014C00E94E34AE0E0F0EC69E774E40E943D
:10102A00085A09F008F403C00E94EC4A06C00E945C
:10103A00F34AA0E6B7E00E94D74A0E94FC4A0E94FF
:10104A008B490E9425590E949449E091CE07F0915C
:10105A00CF076091D0077091D1070E94054B0E947B
:10106A00085A68F5E091D607F091D7076091D8073A
:10107A007091D9070E94054B0E942559E093D20727
:10108A00F093D3076093D4077093D5070E94054B5A
:10109A000E949D490E941E59DF01CB010E94744A99
:1010AA000E94C359A0E0B0E081E695E40E94755918
:1010BA00A4E5B7E00E94D74A689422F802C0E4E0A7
:1010CA002E260E94FC4A0E940E4B0E942559E0934C
:1010DA00DA07F093DB076093DC077093DD070E9461
:1010EA000E4B0E94174B0E94085A09F008F41FC0C1
:1010FA00E0E0E093DA07E093DB07E093DC07E093B4
:10110A00DD070E941C4BEF5FFF4F6F4F7F4F0E941E
:10111A005C490E941C4BE0931A08F0931B086093E9
:10112A001C0870931D080E94254B0E944E4B0E947A
:10113A006549A034E2E4BE07EFE08E07E0E09E07CF
:10114A00A8F0E0E0E0933507E0933607E09337072D
:10115A00E0933807E0931A08E0931B08E0931C0811
:10116A00E0931D080E94254B0E944E4B0E94AD49F8
:10117A000E9475590E94A6490E94574B0E2EE09173
:10118A00F606A091F4060E94A65A0E22A091F50630
:10119A00E091F7060E94A65AE02119F0E0E0E093F8
:1011AA00F806A0912705AC3319F4E2E0E093F806BB
:1011BA00A0914505A23009F09AC0E0E0E093450508
:1011CA00A09126050E945D4B0E94624B0E94944AA0
:1011DA000E94F35A0E220E94574B0E946B4B0E94A8
:1011EA00714BE02191F0E0912705EF5FE09327052D
:1011FA00E0912605F0E03296A0912705B0E0EA17C3
:10120A00FB0719F4ECE3E0932705033631F4E1E038
:10121A00E0932705E0E0E093F806D394A091100547
:10122A00A13028F4E0911005EF5FE09310050E94C9
:10123A00784BE8E5F2E00E94E75A0E2E0E94314907
:10124A000E946A4AE02199F0E0911B07F0911C077D
:10125A003196E0931B07F0931C070E94784B0E947B
:10126A007D4BEA1BFB0BE0931F07F0932007ECE38F
:10127A00ED1589F4DD24C394EC1569F4CC24E091CE
:10128A000005EF5FE0930005A0910005A43119F471
:10129A00E0E0E0930005A0912E05A130D0F0E091A6
:1012AA001305EF5FE0931305A0911305A23088F0B0
:1012BA00E0911205EF5FE0931205E0E0E093130579
:1012CA00E0912E05A0911205EA1718F4E0E0E093E8
:1012DA001205E0912E05E03019F4E0E0E0931205E2
:1012EA00A0912E05A23019F4E1E0E0931205E8EC92
:1012FA005E1648F45394EEE1E51529F4E1E04E2E2A
:10130A00E0E0E0934A050E94824BA4E00E94350186
:10131A00E98FFA8FE7E2E0937A000E94824BA7E016
:10132A000E943501EF8BF88FE7E2E0937A000E9482
:10133A00824BA3E00E948A4B3B9748F1A3E00E94AC
:10134A003501662777270E948F4BA8EEB3E080E02D
:10135A0090E00E942B5BDF01CB010E94924B662733
:10136A0077270E94735B0E948F4BAEEBB7E00E9417
:10137A00E9580E94F15BE0910905EF5FE0930905E6
:10138A000E94974B20F0E881F981ED87FE87E7E21A
:10139A00E0937A00E0E03699E1E06E2EE091F806FB
:1013AA00E03059F4E0E04A99E1E09E2E0E949D4B1C
:1013BA00BE2EE0E03799E1E0AE2EA091F806A1300A
:1013CA0099F4E0E03699E1E0E093C905E0E04A9952
:1013DA00E1E0E093CA050E949D4BE093CB05E0E073
:1013EA003799E1E0E093CC05A091F806A23039F4F0
:1013FA000E94294AE0E0E093F606E093F706A091FE
:10140A00C9050E940448A091CD050E94A54BA09150
:10141A0024050E94AA4B89F0E1E0E093CD05E09112
:10142A00F606E65FE093F606A091F606A43628F0E3
:10143A00E091F606E456E093F606A091CA050E94EA
:10144A000448A091CE050E94AA4B79F0E1E0E0930E
:10145A00CE05E091F606EF5FE093F606A091F60658
:10146A00A43618F0E0E0E093F606A091CB050E94BE
:10147A000448A091CF050E94AA4B89F0E1E0E093CD
:10148A00CF05E091F706E65FE093F706A091F7062D
:10149A00A43628F0E091F706E456E093F706A09107
:1014AA00CC050E940448A091D0050E94AA4B79F06D
:1014BA00E1E0E093D005E091F706EF5FE093F706ED
:1014CA00A091F706A43618F0E0E0E093F706A091A1
:1014DA00C905A13019F4E0E0E093CD05A091CA0551
:1014EA00A13019F4E0E0E093CE05A091CB05A1303C
:1014FA0019F4E0E0E093CF05A091CC05A13019F4EE
:10150A00E0E0E093D0050E94254AE7EAE0937A00FA
:10151A00A0E00E948A4BEFA7F8ABE7E2E0937A00DB
:10152A000E94254A0E94AF4B0E94B44BE7E2E09327
:10153A007A00E0911105E03009F09CC0E1E0E51580
:10154A0091F50E94B94B5E9710F4E1E0ECAF0E946E
:10155A00BE4B0E94B94BEAEFF0E00E94E75AE02145
:10156A0011F0E2E0ECAF0E94B94BAB3FE0E0BE07FE
:10157A0010F0E3E0ECAFAFA5B8A95E9710F4E1E094
:10158A00EBAF0E94C54BEAEFF0E00E94E75AE02178
:10159A0011F0E2E0EBAFAFA5B8A9AB3FE0E0BE07C0
:1015AA0010F0E3E0EBAF0E94B94B0E94CD4BACAD1B
:1015BA000E94AA4B11F0E4E009C00E94B94B0E94B4
:1015CA00D84BACAD0E94AA4B11F0E5E0ECAFAFA549
:1015DA00B8A90E94CD4BABAD0E94AA4B11F0E4E032
:1015EA0009C0AFA5B8A90E94D84BABAD0E94AA4BBF
:1015FA0011F0E5E0EBAFACAD0E945D4BACAD0E94E3
:10160A00E34B69F0EFA5F8A90E94B44BE8E2F0E0D9
:10161A00EFA7F8ABAC85AC3511F40E94E84BACAD42
:10162A000E94EE4BACADE5E00E94A65AE02911F00B
:10163A000E94E84BABAD0E945D4BABAD0E94E34B01
:10164A0069F0E8E2F0E0EFA7F8ABACAD0E945D4BC1
:10165A00ACAD0E94E34B11F00E94E84BABAD0E9487
:10166A00EE4B0E94F34BE02921F0ECE3F0E0EFA708
:10167A00F8AB03C0E0E0ECAFEBAFA0915D05A130A1
:10168A0041F4EFA5F8A9AFA5B8A90E94F84BEFA7B6
:10169A00F8ABA0914605A13041F40E94004C0E948B
:1016AA00B94B0E94F84B0E94B44BAFA5B8A9A73D0D
:1016BA00E0E0BE0720F0E6EDF0E0EFA7F8ABE0913E
:1016CA005E05E03039F5A8ADA330F0F4A885B985F8
:1016DA000E941F5C34F4E885F98535960E94054C12
:1016EA0012C0A985AA2332F4E885F98535970E94A4
:1016FA00054C09C0E0E0E093E207E093E307E093DA
:10170A00E407E093E50704C0E885F9850E94054CE3
:10171A000E940E4CA0915E05A130E1F5E98DFA8D8B
:10172A000E94154CEC83FD836E837F83AC81BD815F
:10173A008E819F81E0E0F0E060E874E40E94C35982
:10174A00A0E0B0E48CE995E40E947559DF01CB0171
:10175A00EDA5FEA50E941A4C0E949E4ADF01CB010C
:10176A00E8EBFEE165ED70E40E94C359DE011896CC
:10177A000E94D74AA0911005A13018F4E0E0E8874A
:10178A00E987E885F9850E94054C0E94974B10F07D
:10179A000E940E4C0E94974B08F481C1E0912D05DE
:1017AA00E03009F06CC0A98DBA8D0E941F4CA2E6E8
:1017BA00B7E00E94D74A0E94334CB1F4A091860741
:1017CA00B09187070E941F4CA4E6B7E00E94D74A4F
:1017DA00A0918E07B0918F070E941F4CA6E6B7E032
:1017EA000E94D74A0E94444CA9A9A130B1F4E091C1
:1017FA008807F09189070E94524CAAE6B7E00E9436
:10180A00D74AE0919007F09191070E94524CACE6BA
:10181A00B7E00E94D74A0E94684CA9A9A230B1F445
:10182A00E0918A07F0918B070E94524CA0E7B7E03B
:10183A000E94D74AE0919207F09193070E94524C76
:10184A00A2E7B7E00E94D74A0E94764CA9A9A33022
:10185A00B1F4E0918C07F0918D070E94524CA6E7F3
:10186A00B7E00E94D74AE0919407F09195070E9449
:10187A00524CA8E7B7E00E94D74A0E94844CA09134
:10188A002D05A13009F06CC0A98DBA8D0E94924C29
:10189A00E0937C07F0937D070E94334CB1F4A0914A
:1018AA008607B09187070E94924CE0936407F093F1
:1018BA006507A0918E07B0918F070E94924CE09322
:1018CA006607F09367070E94444CA9A9A130B1F4B6
:1018DA00A0918807B09189070E94924CE0936A0709
:1018EA00F0936B07A0919007B09191070E94924CD8
:1018FA00E0936C07F0936D070E94684CA9A9A23087
:10190A00B1F4A0918A07B0918B070E94924CE093A0
:10191A007007F0937107A0919207B09193070E9404
:10192A00924CE0937207F09373070E94764CA9A930
:10193A00A330B1F4A0918C07B0918D070E94924C0C
:10194A00E0937607F0937707A0919407B0919507F3
:10195A000E94924CE0937807F09379070E94844C96
:10196A00A0916407B09165070E94984C34F4E09105
:10197A006407F09165070E949F4CA0916A07B09195
:10198A006B070E94984C34F4E0916A07F0916B0758
:10199A000E949F4CA0917007B09171070E94984CC9
:1019AA0034F4E0917007F09171070E949F4CA09166
:1019BA007607B09177070E94984C34F4E091760745
:1019CA00F09177070E949F4CA0916607B091670734
:1019DA000E94A44C34F4E0916607F09167070E94D4
:1019EA00AB4CA0916C07B0916D070E94A44C34F4E3
:1019FA00E0916C07F0916D070E94AB4CA0917207C1
:101A0A00B09173070E94A44C34F4E0917207F091EC
:101A1A0073070E94AB4CA0917807B09179070E9496
:101A2A00A44C34F4E0917807F09179070E94AB4C0A
:101A3A00A0916807B09169070E94B04C34F4E09114
:101A4A006807F09169070E94B74CA0916E07B091A0
:101A5A006F070E94B04C34F4E0916E07F0916F0763
:101A6A000E94B74CA0917407B09175070E94B04CC0
:101A7A0034F4E0917407F09175070E94B74CA09175
:101A8A007A07B0917B070E94B04C34F4E0917A0750
:101A9A00F0917B070E94B74CE0E0E0930905E091E2
:101AAA00EE050E94BC4C0E94EB5BA0E0B1E080E036
:101ABA0090E00E942B5BDF01CB01E091EE05F0E0A4
:101ACA00E65CFA4FE081F0E00E942749AAEBB7E012
:101ADA000E94E9580E94F15B0E94C44CE0E0F0E6E3
:101AEA006AEE76E40E94085A09F008F40AC00E94D5
:101AFA00CD4CA0E0B0E080E897E40E941E590E9415
:101B0A00D64CA8ADA43051F40E94C44CEEEFF4EDCB
:101B1A0068EC7FE30E94C3590E94D64C0E94CD4CC8
:101B2A00A0E0B0E080E192E40E94C359DF01CB015A
:101B3A000E94DF4C0E941A4C0E9475590E94D64C92
:101B4A000E94CD4CABE0B7E00E947D4AA091BD0750
:101B5A00AA2342F40E94CD4C0E947F58ABE0B7E022
:101B6A000E947D4A0E94C44CE0E0F0E060E070E42C
:101B7A000E942E5A0E2E0E94C44CE0E0F0E060E073
:101B8A0070EC0E94345AE021B1F0E0E0E093B20731
:101B9A00E093B307E093B407E093B507E093C60771
:101BAA00E093C707E093C807E093C907E0930B07E0
:101BBA00E0930C071BC00E94C44C0E945E4AA2EB31
:101BCA00B7E00E94B4580E94F15BA091B507AA231E
:101BDA001AF00E94E44C04C00E94E44C0E94485A45
:101BEA00A6ECB7E00E94EB580E94F15B0E94E34A20
:101BFA000E94ED4CEF930E94AC4A0E94B54A0E94A3
:101C0A00345AAF91EA23C1F10E94EB48E0E0F0E0D8
:101C1A0068EC72E40E94C3590E941E490E94055C46
:101C2A000E949E4A0E94F14CA091C207B091C3073C
:101C3A008091C4079091C507E0E0F0E064E172E4A6
:101C4A000E947559DF01CB010E94F34A0E94C359D1
:101C5A00A0E0B0E080E291E40E9475590E94F14C44
:101C6A00E091C207F091C3076091C4077091C5075C
:101C7A00DE011A960E94D74AAA2D0E940448A0E0C3
:101C8A00F3FCA1E00E94FA4CE02109F449C0E4E126
:101C9A00EEAB6894F3F8A62D0E9404480E94624BAA
:101CAA00E2E0F0E060E070E00E94FB5AE02119F007
:101CBA00E1E0E0931505A12F0E942F4A0E94FE4CF5
:101CCA0021F0F298F39A12E01BC0A12F0E94014D55
:101CDA000E94FE4C61F0F398F49A0E94064DA130DE
:101CEA0010F013E003C0F498F29A11E009C0A12F92
:101CFA000E940B4D0E94FE4C19F0F498F29A11E0E2
:101D0A00A62D0E942F4A0E94624BEEEFFFEF6FEF63
:101D1A007FEF0E94035BE02119F0E0E0E0931505F4
:101D2A00E091FD06E09344050E94BE4BA091F8069F
:101D3A000E94AA4B09F464C00E94004C0E94104DF4
:101D4A00E12F0E94174D0E94B44B0E94B94BA93C47
:101D5A00E0E0BE0720F0E8ECF0E00E94B44BE12F8F
:101D6A000E94234D0E942C4D0E94314D0E94B44B7B
:101D7A000E94364DAC91A13008F441C00E943D4DFD
:101D8A000E94464D0E942E5C4CF40E94364D0E94E1
:101D9A00524D0E943A5A0E945C4D23C00E94654DE2
:101DAA000E94674DEF930E94654D0E94704DAF915E
:101DBA00EA2379F00E94364D0E94524D0E943F5A02
:101DCA00A093AA07B093AB078093AC079093AD0793
:101DDA0008C00E94654D0E94794D1CF00E94834DF7
:101DEA000EC0A091AA07B091AB078091AC07909161
:101DFA00AD070E948B4D0E94985B0E94B44B04C0B1
:101E0A000E94E84B0E94834DA62D0E9404480E941E
:101E1A00904D0E220E94954D81F16894F0F80E942F
:101E2A00994D0E941B5C49F5E091B207F091B30706
:101E3A00E0933307F09334070E94B94B0E941F5C6A
:101E4A0010F4E4E1ECAB0E94A24D0E94ED4C0E2E80
:101E5A000E94AB4DE02139F0E3E0E09337050E94A0
:101E6A00B14D0E94BB4D0E94004CA6E0B8E00E9412
:101E7A00494A689420F8E894F4F8A0913005A13012
:101E8A0081F50E94C14D0E2EA0914405E0E50E9405
:101E9A00BF5A0E94C34D0E94CC4D0E22A0E0F4FC12
:101EAA00A1E00E94D44D21F00E94D94D0E94DF4D3D
:101EBA000E94C54BE0E5F0E00E94E75A0E220E941C
:101ECA00EA4D0E94CC4DE02161F00E94D94D0E945A
:101EDA00EC4D0E94F74D0E94FB4D19F0E3E00E9481
:101EEA00014EA0913005A23091F50E94044E0E9445
:101EFA00FB5A0E2E0E94EA4D0E94C34DE02121F0AA
:101F0A000E94D94D0E94DF4D0E94044E0E94035B3D
:101F1A000E940C4EE021EF930E94994D0E94B94B0A
:101F2A00882799270E94075C0E94285AAF91EA23C2
:101F3A000E940C4E0E22A885B985E5E0F0E00E94C9
:101F4A00DB5AE02121F00E94D94D0E94EC4D0E94FB
:101F5A00AB4D0E94124E0E94A24D0E94944A0E94CA
:101F6A00F35AE02121F0E0E0E093290506C0A091B0
:101F7A002905A23010F4E89423F80E941B4E3CF481
:101F8A000E94994DA3E0B7E00E947D4A06C00E94D4
:101F9A00004CE0930307F09304070E94004C30972B
:101FAA0029F4E89420F86894F4F82BC0A0E020FC07
:101FBA00A1E00E9404480E94C14D0E22A091300562
:101FCA000E94AA4B1E2E0E94EA4D0E941F4EA0910B
:101FDA004405EFE40E94C45A0E22A09130050E94E3
:101FEA00D44D1E2A0E94EA4D0E941F4E0E94244E82
:101FFA0041F00E94B14D0E94E84BE89421F86894A0
:10200A0020F84B990DC0E0E0E0933307E0933407E2
:10201A000E94B14DE89421F8689420F8E1E001C0EB
:10202A00E0E0E093FA06E09106050E94B94BF0E081
:10203A00EA17FB0720F4E091FD06E09306050E94EB
:10204A002C4E0E94035B0E22A09134050E94AA4BDB
:10205A001E2E0E942C4E0E94FB5A0E22A09135057C
:10206A000E94AA4BE12961F0E091FD06E093060582
:10207A000E94F74D0E943B4E19F0E2E00E94014E89
:10208A000E941B4E94F4689421F80E94004C0E940E
:10209A00A24D0E941A4C0E94085A30F00E94994D93
:1020AA00ADEFB6E00E947D4A02C0E89421F80E9492
:1020BA003F4EA0E025FCA1E00E94A54BA8AD0E94DE
:1020CA00E34B31F0689425F80E94004C0E94AC481A
:1020DA000E943F4EA8AD0E94E34B51F10E94504E20
:1020EA000E94594E90F0A881B981E9A5FAA5EA1B88
:1020FA00FB0BA3E0B0E00E94235B0E94614EAE1B83
:10210A00BF0BA0935007B09351070E94504E0E94F4
:10211A00235C28F40E94664E32970E94AC48A09134
:10212A005107AA232AF4E0E0E0935007E09351070D
:10213A000E946B4E0E941B5B0E94724E71F10E94BC
:10214A006B4E0E943F5A0E94594E60F0A9A5BAA54B
:10215A00E881F981EA1BFB0B0E94614EEA0FFB1F23
:10216A000E94AC480E946B4E0E943F5AA230E0E0A7
:10217A00BE07E0E08E07E0E09E0728F00E94664E68
:10218A0031960E94AC480E94614EAB3FE0E0BE0728
:10219A0024F0EAEFF0E00E94AC480E94664E0E94EA
:1021AA00B94B0E94E75A0E94724E11F0E89425F842
:1021BA000E94664E0E94B94B0E94ED5A0E94724ECE
:1021CA0021F00E94664E0E94B44B0E94754EA09167
:1021DA0061050E94A54B0E94FB4D39F0E1E0E093B6
:1021EA0061050E947D4E0E94B1480E94754E0E9470
:1021FA00FB4D19F10E94824E339760F00E94824E85
:10220A000E94825A0E94894EAE1BBF0BA0935207AE
:10221A00B09353070E94824E0E94175C28F40E94D2
:10222A008E4E35970E94B148A0915307AA232AF4EB
:10223A00E0E0E0935207E0935307EB8DFC8DA8850D
:10224A00B9850E94E75A0E2E0E94FB4D21F10E9489
:10225A00934E349760F00E94934EA5E0B0E00E943E
:10226A00235B0E94894EEA0FFB1F0E94B1480E941D
:10227A00934E0E94175C28F40E948E4E35960E9457
:10228A00B1480E94894EA53CE9E0BE0724F0E4EC7F
:10229A00F9E00E94B1480E947D4EDF010E948E4EF5
:1022AA000E94E75A0E2E0E94FB4D19F0E0E0E093DF
:1022BA0061050E947D4EDF010E948E4E0E94ED5AFA
:1022CA000E2E0E94FB4D21F00E94894E0E949A4ECA
:1022DA000E949F4E0E94035B0E2EA0E027FCA1E005
:1022EA000E94AA4B31F0689427F80E947D4E0E9402
:1022FA00A54E0E949F4E0E94295C54F50E94AA4E48
:10230A000E94594E94F0EBA9F0E0A091B207B09167
:10231A00B307AE1BBF0BE3E0F0E00E94B24EAE1B68
:10232A00BF0BA0935A07B0935B070E94AA4E0E9464
:10233A00235C2CF40E94B94E32970E94A54EA091BC
:10234A005B07AA232AF4E0E0E0935A07E0935B07CD
:10235A000E949F4E0E942E5C84F50E94BE4EA430BD
:10236A00E0E0BE07E0E08E07E0E09E0784F0ABA95C
:10237A00BB27E091B207F091B307AE1BBF0BE2E0B7
:10238A00F0E00E94B24EEA0FFB1F0E94A54E0E9487
:10239A00BE4E0E94235C2CF40E94B94E32960E94D3
:1023AA00A54EA0915A07B0915B07A53CE9E0BE078C
:1023BA0024F0E4ECF9E00E94A54E0E947D4EDF0174
:1023CA000E94B94EAE17BF0710F4E89427F80E948E
:1023DA007D4EDF010E94B94EEA17FB0730F4A09147
:1023EA005A07B0915B070E949A4EE2EAF7E00E9410
:1023FA00C64EE4EAF7E00E94C64EE6EAF7E00E941B
:10240A00C64E0E94CB4E0E94D54E0E94DB4E91F0E2
:10241A000E94CB4E0E94E24EE093A207F093A307DC
:10242A00A091A207B091A307549724F4E2EAF7E037
:10243A000E94E74E0E94EC4E0E94D54E0E94F64E34
:10244A0091F00E94EC4E0E94E24EE093A407F093B2
:10245A00A507A091A407B091A507549724F4E4EA2C
:10246A00F7E00E94E74E0E94FD4E0E94D54E0E9460
:10247A00074F91F00E94FD4E0E94E24EE093A6079C
:10248A00F093A707A091A607B091A707549724F441
:10249A00E6EAF7E00E94E74EE091A207F091A3076F
:1024AA000E940E4F30F4E091A207F091A3070E9418
:1024BA00B44BE091A407F091A5070E940E4F30F4A7
:1024CA00E091A407F091A5070E94B44BE091A607FA
:1024DA00F091A7070E940E4F30F4E091A607F09101
:1024EA00A7070E94B44BE09114050E94B94BF0E093
:1024FA00EA17FB0720F4E091FD06E0931405E0914A
:10250A001405F0E035970E94B94B0E94E75A6E2FE6
:10251A000E2EA0E025FCA1E00E94D44D1E2E062E10
:10252A00A09161050E94D44D1E2A062EA0E027FC28
:10253A00A1E00E94D44DE12979F0E091FD06E093F3
:10254A0014050E94F74DA8ADE3E00E94AB5AE021C2
:10255A0019F0E2E00E94014EA0913705A13078F00F
:10256A000E94E84BA0913705A13021F4EAE0F0E09F
:10257A000E94B44BE0913705E150E09337050E9481
:10258A00124F0E94AA4B1E2EAFA5B8A9E0E5F0E0B3
:10259A000E94ED5A0E2EA0913005E1E00E94A65A43
:1025AA000E94CC4DE0211E2A0E94124F0E941C4F0D
:1025BA000E943B4E1E2AAFA5B8A9E2E3F0E00E94B2
:1025CA00ED5A0E2E0E94244ED9F0E0E0E093070562
:1025DA000E941B4E1CF4E2E0E09337050E94B14DC5
:1025EA00EFA5F8A9F2970E941A4CA6EFB8E28CE977
:1025FA009FE30E947559DE019F960E947D4A03C09F
:10260A00E0E0EFA7E8ABA0914D05A130E9F5E09134
:10261A004705E03031F4AB8DBC8D0E94214F0E94FA
:10262A00264FA0914705A13031F4AD8DBE8D0E9491
:10263A00214F0E94264FA0914705A23031F40E94F3
:10264A002D4F0E94214F0E94264FA0914705A3308B
:10265A0041F4AF8DB8A10E94214F0E94344FEFA3DD
:10266A00F8A7A0914705A43071F4ED8DFE8D0E9464
:10267A00DE480E94FF49A9A1BAA1AE0FBF1F0E945E
:10268A00214F0E94264F04C00E94004CEFA3F8A7D6
:10269A000E94394F0E2EA0912B050E94D44D11F0A5
:1026AA002C9A01C02C980E94394F0E2EA091FA063E
:1026BA00E1E00E94A65AE02911F0E3E001C0E0E05F
:1026CA00E0934F05A62D0E9404480E94904DE021F8
:1026DA0019F0EFA5E0935C05A0915C05A130A8F084
:1026EA00E0915C05AFA5B8A9F0E0EA17FB0728F06E
:1026FA00E0915C05F0E0EFA7F8AB0E94B94B0E94AD
:10270A001F5C18F4E0E0E0935C05A62D0E940448E3
:10271A00A0912805EEEF0E94BF5A0E22A02FE3E6F1
:10272A000E94AB5A0E220E94AB4D0E22AFA5B8A949
:10273A00E0E0F0E00E94C95A0E220E94624BE1E0FA
:10274A00F0E060E070E00E94FB5A0E220E94624BA9
:10275A00EFEFFFEF6FEF7FEF0E94035B0E94714B79
:10276A000E22A091F406BB27E091F506F0E00E9444
:10277A003C4F0E94DB5AE02169F0E0912805EF5FA7
:10278A00E0932805A0912805A43119F4E2E0E0932A
:10279A00F80603C0E0E0E0932805A82DE0E00E94D7
:1027AA00A65A6E2F0E2EA0E0F099A1E00E941C4FAF
:1027BA000E94574B0E22AC85EDE50E94AB5A0E944F
:1027CA00414F1E2E062EA0E0F099A1E00E941C4F58
:1027DA000E94574B0E946B4BE0211E2A0E947D4BA0
:1027EA000E94784B0E94C95A0E2E0E94574B0E2205
:1027FA000E9431490E946A4AE021E12909F47EC017
:10280A00F09B7CC0F098E0E0E0936405ECE5E0938F
:10281A006505E0910807E0936605E09107070E94C5
:10282A00484F0E94E9470E944B4FE0E0E09364055D
:10283A00EEE1E09365050E944F4FA6E6B5E00E94DF
:10284A00B258EC93A7E6B5E00E94574F0E947D4824
:10285A000E94E9470E944B4F0E9497480E94B34941
:10286A000E94CD4A0E94634FA6E6B5E00E94B25884
:10287A00EC930E94B3490E947559A7E6B5E00E94FD
:10288A00B258EC930E947D480E94E9470E944B4F40
:10289A00E0E0E0936405E7E3E0936505E091220751
:1028AA00E0936605E09121070E94484F0E94E9479C
:1028BA000E944B4FE0E0E0936405EEE5E093650586
:1028CA00C0926605E09100050E94484F0E94E947C0
:1028DA000E944B4F0E946A4FE0912407E0936605DD
:1028EA00E09123070E94484F0E94E947A4E6B0E01E
:1028FA000E9475582998E2E3E0934B05AB2D0E949C
:10290A002F4A0E94904DE02139F0E894F2F8E0E075
:10291A00E0936005E0934105AB2D0E940448A09125
:10292A0060050E94FA4CE02171F0E0914105EF5FE9
:10293A00E0934105A0914105AA3029F4E0E0E09333
:10294A004105E0933305AB2D0E940448A091600530
:10295A000E94A54BA0E0F2FCA1E00E94FA4CE02103
:10296A00D9F1E4E1EDAB6894F2F8E0913305EF5F59
:10297A00E0933305A09133050E940B4D0E94954DBB
:10298A0019F0E1E0E0933305A09133050E94EE4B84
:10299A000E94954D19F0E2E0E0933305A0913305CA
:1029AA000E940B4DA0912B050E94A54BA8ADE3E018
:1029BA000E94AB5AE02119F0E1E0E0933305A091BF
:1029CA0033050E94EE4BA0E0F0FCA1E00E94D44D3A
:1029DA0019F0E3E0E0933305E091F806E03009F0FE
:1029EA003BC1E0E0E0935005E0935105E093FB061C
:1029FA00E093FC06E0913305E030A1F4F698A0914B
:102A0A002B05A23011F40E94C647A0914C050E94E2
:102A1A005D4B0E946D4F11F00E94744FE0E0E0930D
:102A2A00320549C0A0913305A130A1F4A0914C050B
:102A3A00A33010F40E94744FA0914C05A33021F4E6
:102A4A00E0912105E09350050E94794F11F40E940C
:102A5A00804F31C0A0913305A230A9F4F69AA09113
:102A6A004C05A33010F40E94744FA0914C05A3307A
:102A7A0021F4E0912205E09350050E94794F11F468
:102A8A000E94804F18C0A0913305A330A1F4F69A92
:102A9A00A0914C05A33018F4E091EF0501C0EFEFC7
:102AAA00E0935005EFEFE09351050E94794F19F436
:102ABA00EFEFE7BDE8BDA0914F050E940B4DA09135
:102ACA004C05E1E00E94C45A0E220E946D4F19F093
:102ADA00EFEFE0935005A0914F050E9404480E9431
:102AEA008A4F29F00E94744FE1E0E093FB06A0911F
:102AFA004F050E945D4B0E948A4F31F0EFEFE09341
:102B0A005005E0E0E093FB06A0914F050E940448BF
:102B1A000E94914F29F00E94744FE0E0E093FB0677
:102B2A00A0914F050E945D4B0E94914F31F0EFEF4B
:102B3A00E0935005E2E0E093FB060E94984FE081A3
:102B4A00E0938A000E94C14D0E2E0E94394F0E2238
:102B5A000E943B4E1E2E0E94AB4D0E94124EA62D85
:102B6A000E94A54BA02FE3E60E94AB5A0E220E94B8
:102B7A009E4F0E22A0912B050E94AA4B1E2AA091BD
:102B8A00FA060E942F4A0E94C14DE021E12909F468
:102B9A003BC0A091FA06A13011F40E94E84BA09123
:102BAA002A05A13019F4EFEFE0938800E0910505BA
:102BBA00EF5FE0930505A0912A05A33031F4E27096
:102BCA00AFEFEA02F001E0938800A0910505E5E085
:102BDA000E94C45A0E2EE4E10E94BF5AE02161F01D
:102BEA000E94A34FE0938A00A0912A05A23021F403
:102BFA000E94A34FE0938800A0910505A03118F028
:102C0A00E0E0E093050527C0E0E0E0938800A0E05B
:102C1A0024FCA1E00E942F4AA09133050E94AA4BEE
:102C2A00D1F0E0914005EF5FE0934005A0914005A7
:102C3A00A13019F4EFEFE0938A00A0914005A33088
:102C4A0019F4E0E0E0938A00A0914005A43019F459
:102C5A00E0E0E093400507C00E94C647E0E0E09349
:102C6A008800E0938A000E94AA4FF0F0E0911D05C7
:102C7A00A0911F05AE1728F4E0911F05EC5FE093C1
:102C8A001F05E0911D05A0911F05EA1728F4E091A0
:102C9A001F05E250E0931F05033621F4E0911D055C
:102CAA00E0931F056894F6F80E94AA4FF0F4E091A9
:102CBA001E05A0911F05AE1728F4E0911F05EC5FD1
:102CCA00E0931F05E0911E05A0911F05EA1728F45D
:102CDA00E0911F05E250E0931F05033621F4E091CD
:102CEA001E05E0931F05E894F6F8A091F806A230B5
:102CFA0018F4E0911F0501C0E0E0E093B300E1E0C1
:102D0A00E91529F4E894F1F8E0E0E0935F05A92DCC
:102D1A000E940448A0915F050E94A54BA0E0F1FC27
:102D2A00A1E00E94FA4CE02139F16894F1F8E091AF
:102D3A000F05EF5FE0930F05E0E0EAAFAAADA5301B
:102D4A0088F40E94B14FA081A13018F0E5E0EAAF03
:102D5A0005C0E0910F05EF5FE0930F05EAADEF5F65
:102D6A00EAAFECCFA0910F05A53018F0E0E0E093B0
:102D7A000F050E94B14F0081A92D0E940448A0911D
:102D8A002505EFEF0E94BF5AE02121F0E0912505C9
:102D9A00EF5F03C0E894F1F8E0E0E0932505A09125
:102DAA002505A43109F0BAC1AC85E0E00E94BA5AFF
:102DBA000E2E0E94904DE02119F0EC85E150EC872F
:102DCA00033610F403E6AAC101E0E0E0E0930F0540
:102DDA000E94B74FE0911805E0936605EBA9E093CE
:102DEA006705E0911905E0936805E0911B05E093FA
:102DFA0069050E94BD4FE0936A050E94C24FE093A5
:102E0A006B050E94C74FE0936C05E0911C05E093A7
:102E1A006D05E0911D05E0936E05E0912105E093B3
:102E2A006F05E0912605E0937005E0910A07E093AB
:102E3A007105E0910907E0937205FE01EE5BFF4F11
:102E4A00E081E0937305FE01ED5BFF4FE081E093C3
:102E5A007405FE01EC5BFF4FE081E0937505EEAD72
:102E6A00E0937605EFADE0937705FE01E05CFF4F56
:102E7A00E081E0937805EAA5E0937905E9A5E09376
:102E8A007A05E0913405E0937B05E0913605E093FD
:102E9A007C05E0913505E0937D05EC8DE0937E0598
:102EAA00EB8DE0937F05EEA5E0938005EDA5E09319
:102EBA008105ECA1E0938205EBA1E09383050E94D2
:102ECA004F4FA4E8B5E00E94B258EC93A5E8B5E0EC
:102EDA000E94574FE0911007E0938605E0910F0793
:102EEA00E09387050E941E49E8E00E94765AE09323
:102EFA008805E0913907E0938905E0915E05E09342
:102F0A008A05E0911A07E0938B05E0911907E0938F
:102F1A008C05E0910805E0938D05E0910A05E093A0
:102F2A008E05E0910B05E0938F05E0910C05E09387
:102F3A009005E0910D05E0939105E0910E05E0936F
:102F4A0092050E94B3490E94CD4A0E94634FA3E9A9
:102F5A00B5E00E94B258EC930E94B3490E94755999
:102F6A00A4E9B5E00E94B258EC93E0912A05E093F7
:102F7A009505E0912B05E0939605E0912C05E093E9
:102F8A009705E0912D05E0939805E0912E05E093D1
:102F9A009905E0912F05E0939A05E0913005E093B9
:102FAA009B05E0913105E0939C05E0912207E093AF
:102FBA009D05E0912107E0939E05E0912E07E0939D
:102FCA009F05E0912D07E093A005E0E031FCE1E0E8
:102FDA00E093A105E0911105E093A205E8ADE09325
:102FEA00A305EEA10E944948EDA1E0936605E09190
:102FFA004C05E0936705E0914D05E0936805E09183
:10300A004E05E0936905E0911E05E0936A05E0919B
:10301A002005E0936B05E0912205E0936C05E091B1
:10302A002305E0936D05E0911605E0936E050E9475
:10303A006549E8E10E94765AE0936F050E941C4BAD
:10304A000E94915AE09370050E946549E8E00E9447
:10305A00765AE0937105E0913507E0937205E091A5
:10306A005905E0937305E0915A05E0937405E091E0
:10307A005B05E0937505E0915D05E0937605E091C7
:10308A004605E0937705E0914705E0937805E091DE
:10309A004805E09379050E947D48E7E10E9484484B
:1030AA00E0E0E0936405E0E7E0936505E091EE0572
:1030BA00E0936605E091C805E0936705E091EF05A6
:1030CA00E0936805E091F005E0936905E091F10568
:1030DA00E0936A05E091F406E0936B05E091F5064A
:1030EA00E0936C05E091F906E0936D05EE8DE093AF
:1030FA006E05ED8DE0936F05E8A1E0937005EF8D05
:10310A00E09371050E947D48EEE00E948448E1E068
:10311A004E2EE0E0E0934A050E94CC4FA92D0E9472
:10312A000448A0E0F1FCA1E00E94A54BAC85E4E6CE
:10313A000E94B55A0E94414F51F06894F1F8EC850B
:10314A00EF5FEC87AC85A43611F4E0E0EC87E1E0B0
:10315A00E61511F4E894F0F8A62D0E940448A0E0C0
:10316A00F0FCA1E00E94A54BAC85E0E00E94B05AB9
:10317A000E94414F51F06894F0F8EC85E150EC87D9
:10318A00AC85AF3F11F4E3E6EC87AA2D0E94044810
:10319A000E94D64FC1F00E94DC4FA9F4A0913E05CF
:1031AA00A43119F4E7E0E0933E05E0E0E0933F053F
:1031BA00E894F3F8A0913E05A33028F0E0913E058B
:1031CA00E150E0933E05AB2D0E9404480E94D64F81
:1031DA00C1F00E94DC4FA9F4A0913E05A43119F474
:1031EA00E7E0E0933E05E0E0E0933F05E894F2F87B
:1031FA00A0913E05A33028F0E0913E05E150E0930E
:10320A003E05AB2D0E942F4AAA2D0E94D44D31F0C3
:10321A00E0E0E0933F05E4E1E0933E05E1E0EA15F2
:10322A0011F4E894F3F8AA2D0E940448A0E0F3FCF4
:10323A00A1E00E94A54B0E94D64F09F434C46894B9
:10324A00F3F8AC85A13049F4A0911805A13028F40F
:10325A00E0911805EF5FE0931805AC85A23031F4D0
:10326A00ABA9AF3518F4EBA9EF5FEBABAC85A33094
:10327A0049F4A0911905A63928F4E0911905EF5FE0
:10328A000E94E74FAC85A43049F4A0911B05A832EF
:10329A0028F4E0911B05EF5FE0931B05AC85A53090
:1032AA0041F40E94FA4FA43620F40E94B6480E94C4
:1032BA00FF4FAC85A63041F40E940450A43620F496
:1032CA000E94BB480E94FF4FAC85A73041F40E9480
:1032DA00064DA43620F40E94C0480E94FF4FAC85D8
:1032EA00A83049F4A0911C05A13028F4E0911C05EE
:1032FA00EF5FE0931C05AC85A93049F4A0914C0519
:10330A00A53028F4E0914C05EF5FE0934C05AC85BD
:10331A00AA3049F4A0914D05A13028F4E0914D0559
:10332A00EF5FE0934D05AC85AB3049F4A0914E05B3
:10333A00A13028F4E0914E05EF5FE0934E05AC858D
:10334A00AC3059F40E945749A436E0E0BE0728F48D
:10335A000E94D24A31960E945249AC85AD3059F446
:10336A000E94CA48A43CE9E0BE0728F40E94924B96
:10337A0031960E94C548AC85AE3051F4DE01AE5B91
:10338A00BF4FAC91AD3720F40E94CF480E9409503C
:10339A00AC85AF3051F4DE01AD5BBF4FAC91AD37B8
:1033AA0020F40E94D4480E940950AC85A03151F4FF
:1033BA00DE01AC5BBF4FAC91AD3720F40E94D94817
:1033CA000E940950AC85A13131F4AEADA83C18F485
:1033DA00EEADEB5FEEAFAC85A23131F4AFADA83CF8
:1033EA0018F4EFADEB5FEFAFAC85A33159F4DE0112
:1033FA00A05CBF4FAC91A83C28F4FE01FD96339621
:10340A000E940950AC85A43159F40E943149A8356B
:10341A00E2E0BE0728F40E947D4B7E960E942C496A
:10342A00AC85A531D1F40E940E50E0EFF0E00E9485
:10343A00E75A0E941750E8E6F1E00E94E75A0E9414
:10344A002250E0EEF1E00E94E75AE021E12929F05A
:10345A00E9A5FAA53196E9A7FAA7AC85A63149F4F8
:10346A00A0913405A13028F4E0913405EF5FE09390
:10347A003405AC85A73149F4A0913605A23328F466
:10348A00E0913605EF5FE0933605AC85A83149F443
:10349A00A0913505A13028F4E0913505EF5FE0935E
:1034AA0035050E942D500E94AA4B29F00E943550E2
:1034BA0010F40E943B500E942D500E94D44D59F0A6
:1034CA00AD8DBE8DA43FE1E0BE0728F4ED8DFE8DE3
:1034DA003A96ED8FFE8F0E942D500E94415039F08E
:1034EA000E94355020F40E943B500E9446500E9490
:1034FA002D500E944B5059F0AF8DB8A1A43FE1E086
:10350A00BE0728F4EF8DF8A13A960E94044A0E9459
:10351A002D500E94505059F00E94355040F40E949C
:10352A003B500E944650EF8FF8A3E9A3FAA3AC855B
:10353A00AA3159F40E941049A03BE4E0BE0728F4DE
:10354A000E94DF4C31960E945550AC85AB3191F404
:10355A000E941E49A73EE3E0BE07E0E08E07E0E0D6
:10356A009E0740F40E94AC4AEF5FFF4F6F4F7F4FB8
:10357A000E941549AC85AC3149F4A0915E05A13091
:10358A0028F4E0915E05EF5FE0935E05AC85AD310E
:10359A0069F40E94654AAE3DE3E0BE0738F40E9432
:1035AA00444A3A96E0931107F0931207AC85AE317C
:1035BA0069F40E946F4AA835E2E0BE0738F40E9417
:1035CA00504A3A96E0931D07F0931E07AC85AF3137
:1035DA0049F4A0910805AA3028F4E0910805EF5FA4
:1035EA00E0930805AC85A03249F4A0910A05A03100
:1035FA0028F4E0910A05EF5FE0930A05AC85A13251
:10360A0049F4A0910B05A03128F4E0910B05EF5F76
:10361A00E0930B05AC85A23249F4A0910C05A031C8
:10362A0028F4E0910C05EF5FE0930C05AC85A3321A
:10363A0049F4A0910D05A03128F4E0910D05EF5F42
:10364A00E0930D05AC85A43249F4A0910E05A03192
:10365A0028F4E0910E05EF5FE0930E05AC85A532E4
:10366A0049F4A0912A05A33028F4E0912A05EF5FD6
:10367A00E0932A05AC85A63249F4A0912B05A23025
:10368A0028F4E0912B05EF5FE0932B05AC85A73278
:10369A0049F4A0912C05A33028F4E0912C05EF5FA2
:1036AA00E0932C05AC85A83249F4A0912D05A130F0
:1036BA0028F4E0912D05EF5FE0932D05AC85A93242
:1036CA0049F4A0912E05A23028F4E0912E05EF5F6F
:1036DA00E0932E05AC85AA3249F4A0912F05A330B8
:1036EA0028F4E0912F05EF5FE0932F05AC85AB320C
:1036FA0049F4A0913005A23028F4E0913005EF5F3B
:10370A00E0933005AC85AC3249F4A0913105A13083
:10371A0028F4E0913105EF5FE0933105AC85AD32D5
:10372A0091F40E946549AF39E6E8BE07E1E08E07E9
:10373A00E0E09E0740F40E941C4BE65FFF4F6F4F8C
:10374A007F4F0E945C49AC85AE3259F40E944D49C4
:10375A00A031E7E2BE0728F40E94C84A3A960E94BE
:10376A004849AC85AF3261F4A0E031FCA1E0A13058
:10377A0038F4E0E031FCE1E0EF5F0E94335C31F8BD
:10378A00AC85A03349F4A0911105A13028F4E09149
:10379A001105EF5FE0931105AC85A13331F4A8ADB3
:1037AA00A43018F4E8ADEF5FE8AFAC85A23359F462
:1037BA00ADA1BEA1A435E2E0BE0728F4EDA1FEA1A9
:1037CA003196EDA3FEA3AC85A33349F4A091160567
:1037DA00A43628F4E0911605EF5FE0931605AC8550
:1037EA00A43349F4A0915905A33828F4E091590566
:1037FA00EF5FE0935905AC85A53349F4A0915A05CA
:10380A00A73428F4E0915A05EF5FE0935A05AC8596
:10381A00A63349F4A0915B05A53628F4E0915B052F
:10382A00EF5FE0935B05AC85A73349F4A0915D0592
:10383A00A13028F4E0915D05EF5FE0935D05AC856A
:10384A00A83349F4A0914605A13028F4E091460531
:10385A00EF5FE0934605AC85A93349F4A09147058B
:10386A00A43028F4E0914705EF5FE0934705AC8563
:10387A00AA3349F4A0914805A43028F4E0914805F8
:10388A00EF5FE0934805AC85AB3349F4A091EE05B0
:10389A00A33028F4E091EE05EF5FE093EE05AC85E6
:1038AA00AC3349F4A091C805A13028F4E091C805C9
:1038BA00EF5FE093C805AC85AD33E1F4E091010513
:1038CA00EF5FE0930105A0910105AC3318F0E0E049
:1038DA00E09301050E94B74F0E946E50E295E07F87
:1038EA006E2F0E947650E60FE09366050E94E2472B
:1038FA000E947E50AC85AE3381F4A091EF05AA3FB9
:10390A0028F4E091EF05E65FE093EF05A091EF055B
:10391A00AB3F18F0EAEFE093EF050E9487500E9450
:10392A00E15AE02149F0A091F005AF3F28F4E09177
:10393A00F005EF5FE093F0050E9487500E94ED5A70
:10394A00E02149F0A091F105AF3F28F4E091F1059B
:10395A00EF5FE093F105AC85A03461F4E091F506E0
:10396A00EF5FE093F506A091F506A43618F0E0E0C3
:10397A00E093F506AC85A13449F4A091F906A1308B
:10398A0028F4E091F906EF5FE093F906AC85AB35D0
:10399A0049F4A0914D07AF372CF4E0914D07EF5F42
:1039AA00E0934D07AC85AC3549F4A0910705AA3FD1
:1039BA0028F4E0910705EB5FE0930705AC85AD3588
:1039CA0059F40E949150A73138F40E949650EF5F43
:1039DA00DE01A75BBF4FEC93AC85AE3549F4A091ED
:1039EA005705A93028F4E0915705EF5FE093570592
:1039FA00AC85AF3559F4ADA5BEA5A83BEBE0BE0733
:103A0A0028F4EDA5FEA53196EDA7FEA7AC85A03654
:103A1A0059F4ABA1BCA1A83EE3E0BE0728F4EBA190
:103A2A00FCA13A96EBA3FCA3AC85A13649F4A0917C
:103A3A002605AC3328F4E0912605EF5FE0932605CE
:103A4A00AC85A23691F40E94984FA081AA3F21F436
:103A5A000E949B50EB5FEC930E94984FA081AA3F73
:103A6A0020F40E949B50E65FEC930E94A2500E94B1
:103A7A00E15AE02149F0A0911D05AA3F28F4E091FE
:103A8A001D05E65FE0931D050E94A2500E94ED5AB3
:103A9A00E02149F0A0911E05AA3F28F4E0911E05F5
:103AAA00E65FE0931E05E1E0EB1511F4E894F2F805
:103ABA00AB2D0E940448A0E0F2FCA1E00E94A54BB5
:103ACA000E94D64F09F443C46894F2F8AC85A13039
:103ADA0049F4A0911805A13028F0E0911805E150A9
:103AEA00E0931805AC85A23031F4ABA9A63018F0E2
:103AFA00EBA9E150EBABAC85A33049F4A0911905D1
:103B0A00AD3328F0E0911905E1500E94E74FAC85EA
:103B1A00A43049F4A0911B05A53128F0E0911B05BA
:103B2A00E150E0931B05AC85A53041F40E94FA4FA1
:103B3A00A13020F00E94B6480E94AC50AC85A63055
:103B4A0041F40E940450A13020F00E94BB480E9418
:103B5A00AC50AC85A73041F40E94064DA13020F04C
:103B6A000E94C0480E94AC50AC85A83049F4A0918C
:103B7A001C05A13028F0E0911C05E150E0931C05DA
:103B8A00AC85A93049F4A0914C05A13028F0E09108
:103B9A004C05E150E0934C05AC85AA3049F4A0915C
:103BAA004D05A13028F0E0914D05E150E0934D0517
:103BBA00AC85AB3049F4A0914E05A13028F0E091D4
:103BCA004E05E150E0934E05AC85AC3049F40E94B5
:103BDA005749559728F00E94D24A31970E94524974
:103BEA00AC85AD3059F40E94CA48A538E3E0BE0757
:103BFA0028F00E94924B31970E94C548AC85AE309E
:103C0A0051F4DE01AE5BBF4FAC91A63020F00E94AA
:103C1A00CF480E94B150AC85AF3051F4DE01AD5BA4
:103C2A00BF4FAC91A63020F00E94D4480E94B150F8
:103C3A00AC85A03151F4DE01AC5BBF4FAC91A6302C
:103C4A0020F00E94D9480E94B150AC85A13131F4CC
:103C5A00AEADA13018F0EEADE550EEAFAC85A231B5
:103C6A0031F4AFADA13018F0EFADE550EFAFAC8550
:103C7A00A33159F4DE01A05CBF4FAC91A13028F00A
:103C8A00FE01FD9633960E94B150AC85A43151F4E1
:103C9A000E9431490E941F5C28F40E947D4B7E9746
:103CAA000E942C49AC85A531D1F40E940E50EBEC50
:103CBA00F0E00E94ED5A0E941750E2E2F1E00E9401
:103CCA00ED5A0E942250E9E7F1E00E94ED5AE02104
:103CDA00E12929F0E9A5FAA53197E9A7FAA7AC8560
:103CEA00A63149F4A0913405A13028F0E0913405B9
:103CFA00E150E0933405AC85A73149F4A09136052B
:103D0A00A23028F0E0913605E150E0933605AC8503
:103D1A00A83149F4A0913505A13028F0E091350584
:103D2A00E150E09335050E942D500E94AA4B31F0D4
:103D3A00AB8DBC8D1B9710F00E94B6500E942D507F
:103D4A000E94D44D49F0AD8DBE8D1B9728F0ED8DA4
:103D5A00FE8D3A97ED8FFE8F0E942D500E944150A2
:103D6A0041F0AB8DBC8D1B9720F00E94B6500E948B
:103D7A0046500E942D500E944B5049F0AF8DB8A179
:103D8A001B9728F0EF8DF8A13A970E94044A0E94E7
:103D9A002D500E94505061F0AB8DBC8D1B9740F0A6
:103DAA000E94B6500E944650EF8FF8A3E9A3FAA3E7
:103DBA00AC85AA3159F40E941049A73DE1E0BE073B
:103DCA0028F00E94DF4C31970E945550AC85AB31E8
:103DDA0091F40E941E49AB30E0E0BE07E0E08E0796
:103DEA00E0E09E0740F00E94AC4AE150F04060409B
:103DFA0070400E941549AC85AC3149F4A0915E052A
:103E0A00A13028F0E0915E05E150E0935E05AC85B3
:103E1A00AD3161F40E94654A0E941F5C38F40E9429
:103E2A00444A3197E0931107F0931207AC85AE31FB
:103E3A0061F40E946F4A0E941F5C38F40E94504A43
:103E4A003197E0931D07F0931E07AC85AF3149F413
:103E5A00A0910805A23028F0E0910805E150E0930E
:103E6A000805AC85A03249F4A0910A05A23028F0D1
:103E7A00E0910A05E150E0930A05AC85A13249F4C4
:103E8A00A0910B05A13028F0E0910B05E150E093D9
:103E9A000B05AC85A23249F4A0910C05A13028F09B
:103EAA00E0910C05E150E0930C05AC85A33249F48E
:103EBA00A0910D05A13028F0E0910D05E150E093A5
:103ECA000D05AC85A43249F4A0910E05A13028F065
:103EDA00E0910E05E150E0930E05AC85A53249F458
:103EEA00A0912A05A13028F0E0912A05E150E0933B
:103EFA002A05AC85A63249F4A0912B05A13028F0F9
:103F0A00E0912B05E150E0932B05AC85A73249F4EB
:103F1A00A0912C05A13028F0E0912C05E150E09306
:103F2A002C05AC85A83249F4A0912D05A13028F0C2
:103F3A00E0912D05E150E0932D05AC85A93249F4B5
:103F4A00A0912E05A13028F0E0912E05E150E093D2
:103F5A002E05AC85AA3249F4A0912F05A13028F08C
:103F6A00E0912F05E150E0932F05AC85AB3249F47F
:103F7A00A0913005A13028F0E0913005E150E0939E
:103F8A003005AC85AC3249F4A0913105A13028F056
:103F9A00E0913105E150E0933105AC85AD3269F429
:103FAA000E9465490E94235C40F40E941C4BE15028
:103FBA00F040604070400E945C49AC85AE3251F4DA
:103FCA000E944D490E941F5C28F40E94C84A3197FA
:103FDA000E944849AC85AF3279F4A0E031FCA1E0F7
:103FEA00A13050F0A0E031FCA1E0E1E00E94135CB6
:103FFA00EA1B0E94335C31F8AC85A03349F4A091E6
:10400A001105A13028F0E0911105E150E093110566
:10401A00AC85A13331F4A8ADA13018F0E8ADE15078
:10402A00E8AFAC85A23359F4ADA1BEA1A53FE0E04B
:10403A00BE0728F0EDA1FEA13197EDA3FEA3AC8542
:10404A00A33349F4A0911605A23028F0E091160591
:10405A00E150E0931605AC85A43349F4A0915905C3
:10406A00A53128F0E0915905E150E0935905AC8556
:10407A00A53349F4A0915A05A53128F0E0915A05D3
:10408A00E150E0935A05AC85A63349F4A0915B054B
:10409A00A53128F0E0915B05E150E0935B05AC8522
:1040AA00A73349F4A0915D05A13028F0E0915D05A0
:1040BA00E150E0935D05AC85A83349F4A09146052B
:1040CA00A13028F0E0914605E150E0934605AC8521
:1040DA00A93349F4A0914705A13028F0E09147059A
:1040EA00E150E0934705AC85AA3349F4A09148050D
:1040FA00A13028F0E0914805E150E0934805AC85ED
:10410A00AB3349F4A091EE05A13028F0E091EE0519
:10411A00E150E093EE05AC85AC3349F4A091C805B3
:10412A00A13028F0E091C805E150E093C805AC85BC
:10413A00AD3359F5E0910205EF5FE0930205A091D6
:10414A000205AD3018F0E1E0E0930205E2E0E09309
:10415A006405A09102050E94BC50E295E07F6E2F93
:10416A000E94C250E60FE0936505E0916505E05CA8
:10417A00E09365050E94E247E2E0EA93E0E0F0E0BE
:10418A00FA93EA93A0E00E94D645AC85AE3381F457
:10419A00A091EF05A13028F0E091EF05EA50E093F5
:1041AA00EF05A091EF05AA3018F4E0E0E093EF05DF
:1041BA000E9487500E94E15AE02149F0A091F0053F
:1041CA00A13028F0E091F005E150E093F0050E945B
:1041DA0087500E94ED5AE02149F0A091F105A130E3
:1041EA0028F0E091F105E150E093F105AC85A034A7
:1041FA0061F4E091F406EF5FE093F406A091F4060F
:10420A00A43618F0E0E0E093F406AC85A13449F452
:10421A00A091F906A13028F0E091F906E150E09367
:10422A00F906AC85AB3551F4A0914D07E1E8EA17E0
:10423A002CF4E0914D07E150E0934D07AC85AC3585
:10424A0049F4A0910705A13028F0E0910705E5504F
:10425A00E0930705AC85AD3559F40E949150A13021
:10426A0038F00E949650E150DE01A75BBF4FEC93F5
:10427A00AC85AE3549F4A0915705A13028F0E091FC
:10428A005705E150E0935705AC85AF3559F4ADA514
:10429A00BEA5A13DE7E0BE0728F0EDA5FEA5319732
:1042AA00EDA7FEA7AC85A03659F4ABA1BCA1A536F3
:1042BA00E0E0BE0728F0EBA1FCA13A97EBA3FCA330
:1042CA00AC85A13649F4A0912605A13028F0E091E9
:1042DA002605E150E0932605AC85A236D1F40E946A
:1042EA00984FBF01A0810E945D4BFB01A081EFEFB7
:1042FA000E94BF5AE02121F00E949B50EA50EC93A1
:10430A000E94984FA081AF3F21F40E949B50E55034
:10431A00EC930E94A2500E94E15AE02149F0A09138
:10432A001D05A13028F0E0911D05EA50E0931D0516
:10433A000E94A2500E94ED5AE02149F0A0911E0568
:10434A00A13028F0E0911E05EA50E0931E05A62D43
:10435A000E940448A0912405EDEF0E94BF5A0E94D2
:10436A006B4B0E22A09128050E94AA4B29F0E091DE
:10437A002405EF5FE0932405A62D0E942F4AA09101
:10438A002405EFEF0E94BF5A0E946B4B0E22A091A8
:10439A0028050E94AA4B29F0E894F0F8E0E0E0939F
:1043AA002405A0912405EEE10E94A65A0E2E0E9431
:1043BA00904D0E22A091F8060E94415029F0E1E0AA
:1043CA00E093F806E0932705E0912605E03019F41A
:1043DA00E0E0E09327050E949E4F0E2E0E94574B65
:1043EA000E22A0912705E0E00E94C45AE02119F0AC
:1043FA00E1E0E0932705A0912705AC3311F40E9470
:10440A00CA50A0910705A13028F0E0910705F0E015
:10441A000E94B44BA09131050E942F4A0E94394F45
:10442A00E02159F1EFA9EF5FEFABF0E03196BF0160
:10443A00AFA5B8A90E94344FE617F70790F40E9477
:10444A00CF500E940B5B0E2E0E94D650E4EAF1E098
:10445A0060E070E00E94F35AE02919F0E0E0EFA76B
:10446A00E8ABAFA5B8A90E94344FAFA9B0E0EA17EC
:10447A00FB0710F4E0E0EFAB02C0E0E0EFAB0E9414
:10448A00394F0E2E0E94CF500E941B5B0E22ADA107
:10449A00BEA1E4EAF1E00E94CF5A0E22A8AD0E9422
:1044AA00E34B51F0AFA5B8A9A639E0E0BE0720F466
:1044BA00E6E9F0E0EFA7F8ABE8ECE51509F0F8C09B
:1044CA00E0910A080E94624BFF27662777270E941D
:1044DA00295C94F4E091B207E0930A08E0E0E093E3
:1044EA006405E0E6E0936505E0910A08E093660555
:1044FA000E947D480E947E500E94FA49EAE00E948A
:10450A004B5BA885B985EA17FB07A0F40E94D9502E
:10451A000E94F549E0E0E0936405EEE6E093650564
:10452A00E0911908E0936605E09118080E94484F47
:10453A000E94E947E0910C08F0910D08AD85BE850F
:10454A000E94E75A0E2EE8ECF0E00E94DB5AE021C6
:10455A00A1F0ED85FE850E94B949E0E0E09364058B
:10456A00E2E6E0936505E0910D08E0936605E091C7
:10457A000C080E94484F0E94E947E0910E08F0910A
:10458A000F08AD85BE85EA17FB07A0F4ED85FE8509
:10459A000E94C349E0E0E0936405E4E6E093650520
:1045AA00E0910F08E0936605E0910E080E94484FDB
:1045BA000E94E9470E94E050E0911008F09111082A
:1045CA000E94E5500E94AB4DE021B1F0E0917E07D8
:1045DA00F0917F070E94D749E0E0E0936405E8E69E
:1045EA00E0936505E0911108E0936605E0911008F3
:1045FA000E94484F0E94E9470E94E850E091120841
:10460A00F09113080E94E5500E94AB4DE021B1F0F1
:10461A00E0918007F09181070E94E149E0E0E09390
:10462A006405EAE6E0936505E0911308E093660500
:10463A00E09112080E94484F0E94E9470E94ED50FB
:10464A00E0911408F09115080E94E5500E94AB4DC4
:10465A00E021B1F0E0918207F09183070E94EB49D3
:10466A00E0E0E0936405ECE6E0936505E091150867
:10467A00E0936605E09114080E94484F0E94E947BA
:10468A00A0911608B09117080E948649EA1BFB0BF5
:10469A00E436A0E0FA0760F00E946A4FE09117083A
:1046AA00E0936605E09116080E94484F0E94E94788
:1046BA00ED85FE85A885B9850E94515B0E94F2505E
:1046CA00E0939E07F0939F07E091A807F091A9074E
:1046DA000E94F850EA17FB07D4F4E0919E07F09184
:1046EA009F070E94CD49E0E0E0936405E6E6E09387
:1046FA006505E091A807F091A9070E948C5AE093FA
:10470A006605E091A8070E94484F0E94E9470336D0
:10471A0010F00C94622C0E94B14F0081A0913805D0
:10472A000E945D4BA8AD0E94FD5049F4F79907C05D
:10473A00A0E0F699A1E0EA2FE295E07F19C0A0E097
:10474A00F699A1E0EA2FE295E07F0E2EA0E0F29919
:10475A00A1E0EA2FEE0FEE0F0E0EA0E0F399A1E012
:10476A00EA2FEE0FA02DAE0FE0E0F499E1E0EA0F98
:10477A00DE01A65BBF4FEC93A985AA232AF40E9407
:10478A000251E05A0E940751EAE00E940C51EAE005
:10479A000E9411510E9416510E941C51EAE00E9487
:1047AA002151EAE00E9426510E942B510E94315168
:1047BA00E89430F8A0E025FCA1E00E942F4AA091DD
:1047CA006105E1E00E94A65A0E2AA0E027FCA1E0BA
:1047DA00E1E00E94A65AE02921F0E894F79968944A
:1047EA0001C0E894F5F8A091FA06A13011F4689492
:1047FA00F5F8E0912F05E03021F40E9453510E9410
:10480A006351A0912F05A13081F4A0E021FCA1E021
:10481A00EA2FEE0FE75F0E2EA0E021FCA1E0EA2FBF
:10482A00EE0FEE0FE00D0E947251A0912F05A230FB
:10483A0099F40E945351A0E021FCA1E0EA2F0E94C2
:10484A0082510E0EA0E021FCA1E0EA2FE295E07F62
:10485A00EE0F0E0E0E946351A0912F05A33031F482
:10486A00E0E021FCE1E0E85F0E9472510E945749B2
:10487A00589769F50E948751A23DE0E0BE071CF0F7
:10488A00E1E0E0930305AD85BE85A83FE0E0BE0701
:10489A001CF0E3E0E0930305AD85BE85AF3FE0E0A1
:1048AA00BE071CF0E7E0E0930305AD85BE85A430A2
:1048BA00E1E0BE071CF0EFE0E0930305AD85BE859D
:1048CA00AE30E1E0BE071CF0EFE1E09303050E9481
:1048DA005749949769F50E948751A633E1E0BE07CC
:1048EA001CF0E1E0E0930305AD85BE85AA34E1E062
:1048FA00BE071CF0E3E0E0930305AD85BE85AE3547
:10490A00E1E0BE071CF0E7E0E0930305AD85BE8554
:10491A00A836E1E0BE071CF0EFE0E0930305AD85A1
:10492A00BE85AC37E1E0BE071CF0EFE1E09303057A
:10493A000E945749D09769F50E948751A638E1E04D
:10494A00BE071CF0E1E0E0930305AD85BE85AC3CF3
:10495A00E1E0BE071CF0E3E0E0930305AD85BE8508
:10496A00A63DE1E0BE071CF0E7E0E0930305AD8554
:10497A00BE85A03EE1E0BE071CF0EFE0E093030530
:10498A00AD85BE85AF3EE1E0BE071CF0EFE1E093E6
:10499A000305A0911505A13081F4A0E0F799A1E0E3
:1049AA00EA2F0E9482510E2EA0E0F799A1E0EA2F89
:1049BA00E295E07FEE0FE00D4E0FA0910405A431C1
:1049CA0008F04AC00E94624B0E948F5134F0E3E61D
:1049DA00F0E060E070E00E9497510E94624B0E94F2
:1049EA00A05134F4E7EFFFEF6FEF7FEF0E9497518A
:1049FA00A091B507AA23EAF00E94624B0E94A8512F
:104A0A006CF0FE01E359FF4F3396FF93EF930E9438
:104A1A00B0510E94B651AF91BF91EC930E94C1511F
:104A2A00FF93EF930E94B0510E94B25BAF91BF9186
:104A3A00EC93A091B507AA2372F4EDE00E94C65147
:104A4A000E94C151FF93EF930E94E44C0E94CB5104
:104A5A00AF91BF91EC930DC0F79B05C0E0E40E94B3
:104A6A00C651E0E402C00E941651DE01AF58BF4FA2
:104A7A00EC93AEA9A130A8F0EEA9E150EEABEEE5B9
:104A8A000E94C651E0911505E03029F4FE01E35970
:104A9A00FF4F148306C0E0E50E94C651EAE00E9477
:104AAA001C51ADA9A13058F0EDA9E150EDABE8E3F6
:104ABA000E94C6510E94C151A0913305A083ACA99E
:104ACA00A13048F0ECA9E150ECABE9E30E94C651F1
:104ADA00E0E50E941C51E0911205E03009F042C065
:104AEA004058EAE00E940C51E0E00E941151A09166
:104AFA005C07B0915D070E941F5C84F40E94D65146
:104B0A000E94DB510E94E0511A9724F00E94E5515D
:104B1A000E94EC510E94F4510E94F951A0915D0744
:104B2A00AA2302F5E0915C07F0915D070E94025208
:104B3A000E94DB51E0E40E940C510E94F451A091C2
:104B4A005E07A0830E94E0511A9754F00E94E55133
:104B5A000E94EC510E94F4510E94F951689401C0DC
:104B6A00E89430F8A0911205A13009F047C00E94DC
:104B7A000251E85F0E9407510E940652FF2392F4F5
:104B8A00E0E40E940C510E940652E73FAFEFFA0799
:104B9A0014F4689401C0E89430F80E9406520E9406
:104BAA00445A04C0E89430F80E940652E0935E0723
:104BBA00F0935F070E94E0511A9724F00E94E55192
:104BCA000E94EC510E94F4510E94F9510E9406522F
:104BDA00BF01DF01E3E6F0E00E94DB5A0E2EDB01A3
:104BEA00EDE9FFEF0E94D55AE02941F0E89430F848
:104BFA00E0E40E940C51E0E40E9411510E9412521A
:104C0A00BF01AD85BE850E9417520E941C52BF018A
:104C1A00AD85BE850E94D6510E94EC510E94215258
:104C2A00BF01AD85BE850E942652AD85BE85A639D7
:104C3A00E0E0BE0764F4E0E40E942151E0E40E944F
:104C4A002651E0E40E942D52E0E0E0930305013092
:104C5A0009F053C00E9432520E943A52A83EE3E041
:104C6A00BE0798F0505E0E943F520E9445523E96FF
:104C7A00BF010E943A520E94314D0E9454520E9432
:104C8A005C520E94344FDF0118C050560E943A52BB
:104C9A00A436E0E0BE0730F00E943F520E94314D38
:104CAA000E9454520E946252BF010E943A520E94CC
:104CBA00344F0E9454520E945C52EAE0F0E00E9493
:104CCA006752A0910005AA3010F00E946C520E940F
:104CDA007252A0910005BB270E9426520E94785268
:104CEA00BF01AC2D0E94BC500E94EC510E947D5223
:104CFA00BF01AC2DBB270E942652023009F06DC0BD
:104D0A00505C0E946549A03AE6E8BE07E1E08E07DA
:104D1A00E0E09E0778F00E947852FF93EF930E949A
:104D2A006549E0EAF6E861E070E00E948252AF91DC
:104D3A00BF91EC930E9465490E948D5278F00E94BF
:104D4A007D52FF93EF930E946549E0E1F7E260E04C
:104D5A0070E00E948252AF91BF91EC930E94654924
:104D6A000E94955268F00E949D52FF93EF930E9411
:104D7A0065490E948B4D0E948252AF91BF91EC937C
:104D8A000E9465490E948F5168F00E94A252FF93C7
:104D9A00EF930E9465490E94A7520E948252AF91E6
:104DAA00BF91EC930E9465490E94A85158F00E9455
:104DBA006252FF93EF930E94AC520E948252AF91CB
:104DCA00BF91EC930E94B352FF93EF930E94AC52AF
:104DDA000E94AE5BAF91BF91EC93033009F0BDC066
:104DEA00E7E70E94B8520E94C2520E948D527CF09C
:104DFA000E947D52FF93EF930E94C252E0E1F7E2D4
:104E0A0060E070E00E94B651AF91BF91EC930E94AE
:104E1A00C2520E9495526CF00E949D52FF93EF93EA
:104E2A000E94C2520E948B4D0E94B651AF91BF910F
:104E3A00EC930E94C2520E948F516CF00E94A252BF
:104E4A00FF93EF930E94C2520E94A7520E94B6514A
:104E5A00AF91BF91EC930E94C2520E94A8515CF09C
:104E6A000E946252FF93EF930E94CB520E94B65166
:104E7A00AF91BF91EC93A091B907AA235AF00E946F
:104E8A00B352FF93EF930E94CB520E94B25BAF9151
:104E9A00BF91EC93A091B907AA236AF40E94B35276
:104EAA00FF93EF930E94D1520E94CB51AF91BF91D1
:104EBA00EC930E94DA520E94C2520E94A0517CF4E2
:104ECA000E946252FF93EF930E94E0520E94E652C0
:104EDA000E94B651AF91BF91EC930E94EB520E948F
:104EEA00C252AD39EFEFBE07EFEF8E07EFEF9E0725
:104EFA007CF40E94A252FF93EF930E94E0520E9418
:104F0A00A7520E94B651AF91BF91EC930E94F15201
:104F1A000E94C252A931ECEFBE07EFEF8E07EFEF06
:104F2A009E077CF40E949D52FF93EF930E94E052E9
:104F3A000E948B4D0E94B651AF91BF91EC930E9493
:104F4A00F7520E94C252A13FE8EDBE07EFEF8E076B
:104F5A00EFEF9E0714F40E94FD52A02F0E94EE4B21
:104F6A00A02FE9E00E94A65AE02909F484C050580B
:104F7A00093011F40E946C52EEE30E94B8520E946A
:104F8A000853A031E7E2BE074CF00E947D52BF01F0
:104F9A000E940853E0E1F7E20E940D530E94085371
:104FAA00A83EE3E0BE073CF00E949D52BF010E946A
:104FBA0008530E9410530E940853A436E0E0BE072B
:104FCA003CF00E94A252BF010E9408530E9417524D
:104FDA00A0915907AA2382F00E946252BF010E943F
:104FEA0008530E94D6510E94EC510E94B352BF014D
:104FFA000E9408530E942652A0915907AA2392F4AC
:10500A000E9462520E9413530E9402520E94EC5163
:10501A000E94B3520E9413530E94445A0E94EC51B8
:10502A000E94EB520E940853AD39EFEFBE0754F4C9
:10503A000E94A2520E9413530E9419530E94EC51DB
:10504A000E94F1520E940853A931ECEFBE075CF4AA
:10505A000E949D520E9413530E94445ADF010E94EB
:10506A0010530E94F7520E940853A13FE8EDBE0771
:10507A0014F40E94FD52A02F0E941C53A02FEAE0B4
:10508A000E94A65AE029C1F150580A3011F40E9430
:10509A006C52EEE30E94B8520E942153A091E90794
:1050AA00AA2312F40E94EB520E94E34AE0E0F0E0E5
:1050BA0066EC72EC0E94085A10F40E94F1520E94A7
:1050CA002753A436E0E0BE073CF00E94A252BF017B
:1050DA000E9427530E9417520E946252BF010E94E7
:1050EA0027530E94D6510E94EC510E94B352BF012D
:1050FA000E9427530E942652063099F55058E0E044
:10510A000E942C53E5E00E9431530E943653AA852F
:10511A00BB85A83EE3E0BE073CF00E949D52BF015A
:10512A00AA85BB850E941053AA85BB85A436E0E0F8
:10513A00BE073CF00E94A252BF01AA85BB850E940D
:10514A0017520E946252BF01AA85BB850E94D6519E
:10515A000E94EC510E94B352BF01AA85BB850E94EE
:10516A002652073009F0A1C0AFA5B8A90E941F5C5A
:10517A0018F5ECE00E942C530E943C53E436A0E060
:10518A00FA0738F00E947852BF01AFA5B8A90E9469
:10519A0041530E943C533A9738F00E947D52BF0116
:1051AA00AFA5B8A90E9446530E949D52BF010E9412
:1051BA003C530E94545279C0A0914D050E94044864
:1051CA00A0914D05E2E00E94A65AE02911F1EBE018
:1051DA000E942C530E944B53E436A0E0FA0738F0A1
:1051EA000E947852BF01AFA1B8A50E9441530E9404
:1051FA004B533A9738F00E947D52BF01AFA1B8A530
:10520A000E9446530E949D52BF010E944B530E9426
:10521A005452A0914D050E942F4AA0914D05E3E0FA
:10522A000E94A65AE02909F440C0EBE00E942C53E0
:10523A00AFA1B8A5A436E0E0BE0748F00E947852B4
:10524A00BF01AFA1B8A50E94314D0E9454520E94DD
:10525A007D52BF01AFA1B8A50E94344F0E9454529B
:10526A00E7E70E9450530E945553AFA1B8A5A83E44
:10527A00E3E0BE07D0F00E947852BF01AFA1B8A503
:10528A000E9445523B96BF01AFA1B8A50E94314D7D
:10529A000E9454520E949D52BF01AFA1B8A50E941C
:1052AA00344F0E9454520E945B53083009F078C070
:1052BA000E943252A0915407B0915507A135EBEFE5
:1052CA00BE0734F4E1E5FBEFE0935407F09355078A
:1052DA00A0915407B0915507A03BE4E0BE0734F013
:1052EA00EFEAF4E0E0935407F0935507A0915507CD
:1052FA00AA234AF40E94F152E0915407F09155070B
:10530A000E94445A04C0E0915407F0915507E09373
:10531A005607F0935707A0915607B0915707ECE349
:10532A00F0E00E946E5BE0931307F09314070E946B
:10533A006153ECE30E944B5BA0915607B09157076B
:10534A00AE1BBF0BA0931507B093160722FE20C011
:10535A000E9461531A9710F00E946C520E94725276
:10536A000E9461530E9466530E947852BF01A09125
:10537A001507B09116070E94344F0E9454520E949A
:10538A007D52BF01A0911507B09116070E9466537E
:10539A00E3E70E946953E8E30E946E530E94735345
:1053AA000B3081F55054E9E30E9479530E944D492C
:1053BA00A83EE3E0BE0738F00E949D52BF010E945A
:1053CA004D490E9480530E944D49A436E0E0BE0731
:1053DA0048F00E94A252BF010E944D490E94314DDD
:1053EA000E9454520E946252BF010E944D490E947B
:1053FA00344F0E9454520E94B352BF010E944D4939
:10540A000E9466530C3009F073C00E946C52EEE39E
:10541A000E942C530E94F850E0E0F0E00E9485536D
:10542A00E6EFFFEF0E94DB5AE02111F00E94DA5208
:10543A000E94F850E7EFFFEF0E948553ECE9FFEF77
:10544A000E94DB5AE02111F00E94EB520E94F850B0
:10545A00EDE9FFEF0E948553E8E1FCEF0E94DB5A79
:10546A00E02111F00E94F1520E94F850A931ECEFAC
:10547A00BE0714F40E94F752A0919F07AA2352F480
:10548A00E0919E07F0919F070E94445AE0939E077D
:10549A00F0939F070E94F850A83EE3E0BE073CF055
:1054AA000E949D52BF010E94F8500E9410530E9410
:1054BA00F850A436E0E0BE073CF00E94A252BF01B9
:1054CA000E94F8500E9417520E94F8501A974CF006
:1054DA000E946252BF010E94F8500E94D6510E9457
:1054EA00EC510E94B352BF010E94F8500E9426520A
:1054FA000D3099F50E9489530E948E53A0917F071F
:10550A00AA234AF40E94EB520E946252DF01E09100
:10551A007E07E19507C00E946252BF010E94E050D7
:10552A000E949453EC930E94E050A436E0E0BE0738
:10553A003CF00E949D52BF010E94E0500E94175207
:10554A000E94E0501A974CF00E94A252BF010E949A
:10555A00E0500E94D6510E94EC510E3099F50E94FB
:10556A009A530E948E53A0918107AA234AF40E945B
:10557A00EB520E946252DF01E0918007E19507C079
:10558A000E946252BF010E94E8500E949453EC9319
:10559A000E94E850A436E0E0BE073CF00E949D520B
:1055AA00BF010E94E8500E9417520E94E8501A97C1
:1055BA004CF00E94A252BF010E94E8500E94D651AC
:1055CA000E94EC510F3099F50E949F530E948E530E
:1055DA00A0918307AA234AF40E94EB520E946252C6
:1055EA00DF01E0918207E19507C00E946252BF0184
:1055FA000E94ED500E949453EC930E94ED50A43601
:10560A00E0E0BE073CF00E949D52BF010E94ED50AF
:10561A000E9417520E94ED501A974CF00E94A25213
:10562A00BF010E94ED500E94D6510E94EC510031F8
:10563A0009F043C00E9432520E94CA47A3E00E9466
:10564A00D645E0916505E295EF70AAE0EA02F0011D
:10565A00E0930105E0916505EF70A0910105EA0F5D
:10566A00E0930105E0916605E295E170AAE0EA029D
:10567A00F001E0930205E0916605EF70A091020542
:10568A00EA0FE0930205A0910205AA3010F00E94E9
:10569A006C520E9472520E94C250DB01EC930E942B
:1056AA007852BF010E946E500E94EC510E947D52B6
:1056BA00BF010E947650DB01EC93ACAD0E945D4BBA
:1056CA00ABADE0E00E94C45AE02909F4B2C05F77AA
:1056DA00E0913905E170EE0F4E23E0913905E69528
:1056EA000E94A4530E2EE0913905E695E695E170E5
:1056FA00AE2FE0E0F5FCE1E0EA2BEE0FEE0FE00D55
:10570A004E0F0E943151ABAD0E945D4BACADE0E053
:10571A000E94C45AE02159F1ABADA13029F40E948C
:10572A00A953ECE00E945053ABADA23029F40E9479
:10573A00A953EDE00E945053ABADA33029F40E9467
:10574A00A953EBE00E9450530E94AC5329F00E94E7
:10575A00A953ECE00E9450530E94F34B0E94B653A7
:10576A0029F00E94A953EBE00E94505328C0ABAD28
:10577A00A13021F40E94BC530E94C053ABADA230A9
:10578A0029F40E94BC53EDE00E94C653ABADA3308E
:10579A0029F40E94BC53EBE00E94C6530E94AC530A
:1057AA0021F00E94BC530E94C0530E94F34B0E94F6
:1057BA00B65329F00E94BC53EBE00E94C653ACAD2D
:1057CA00A13039F40E945B53E9E30E946E530E94B0
:1057DA00C053ACADA23041F40E945B53E9E30E948E
:1057EA006E53EDE00E94C653ACADA33021F40E9483
:1057FA005B530E94CB53ACADE4E00E94A65A0E94D0
:10580A00B65339F00E945B53E9E30E946E530E943B
:10581A00C053ACADE5E00E94A65A0E94B65321F0EF
:10582A000E945B530E94CB53E0911205E03009F4C9
:10583A0040580E94CB4E0E94D54E0E94CF530E94E0
:10584A00DB4E69F0E1E00E94D453E7E30E94315352
:10585A000E943653E0E50E94D9530E94DB530E940E
:10586A00EC4E0E94D54E0E94CF530E94F64E49F04C
:10587A00E2E00E94D4530E949A530E9455530E9418
:10588A00DB530E94FD4E0E94D54E0E94CF530E94C8
:10589A00074F69F0E3E00E94D453E9E30E943153D1
:1058AA000E943653E0E50E94D9530E94DB53A0912F
:1058BA00F806A13011F44B7F4F5F033611F00C94B8
:1058CA000E3A31E0303140F40E94E353EAE0EC93BF
:1058DA00E89430F83F5FF6CFAC85EAE50E94EB53D7
:1058EA00E9E50E94A65AE02911F0E1E4EC87AC85CB
:1058FA00A23411F4EBE5EC87EC85E03029F4E09171
:10590A001705F0E0EBA7FCA7AC85A13029F4E091DC
:10591A001805F0E0EBA7FCA7AC85A23021F4EBA9AF
:10592A00F0E0EBA7FCA7AC85A33029F4E0911905B8
:10593A00F0E0EBA7FCA7AC85A43029F4E0911B05A5
:10594A00F0E0EBA7FCA7AC85A53029F40E94BD4F77
:10595A00F0E0EBA7FCA7AC85A63029F40E94C24F61
:10596A00F0E0EBA7FCA7AC85A73029F40E94C74F4B
:10597A00F0E0EBA7FCA7AC85A83029F4E0911C0560
:10598A00F0E0EBA7FCA7AC85A93029F4E0914C051F
:10599A00F0E0EBA7FCA7AC85AA3029F4E0914D050D
:1059AA00F0E0EBA7FCA7AC85AB3029F4E0914E05FB
:1059BA00F0E0EBA7FCA7AC85AC3021F40E94D24AF8
:1059CA00EBA7FCA7AC85AD3021F40E94924BEBA764
:1059DA00FCA7AC85AE3039F4FE01EE5BFF4FE081E7
:1059EA00F0E0EBA7FCA7AC85AF3039F4FE01ED5B24
:1059FA00FF4FE081F0E0EBA7FCA7AC85A03139F4BA
:105A0A00FE01EC5BFF4FE081F0E0EBA7FCA7AC8561
:105A1A00A13121F4EEADF0E0EBA7FCA7AC85A231F1
:105A2A0021F4EFADF0E0EBA7FCA7AC85A33139F484
:105A3A00FE01E05CFF4FE081F0E0EBA7FCA7AC853C
:105A4A00A43121F40E947D4BEBA7FCA7AC85A531BC
:105A5A0021F4E9A5FAA5EBA7FCA7AC85A63129F4A0
:105A6A00E0913405F0E0EBA7FCA7AC85A73129F457
:105A7A00E0913605F0E0EBA7FCA7AC85A83129F444
:105A8A00E0913505F0E0EBA7FCA70E942D500E949B
:105A9A00AA4B11F00E94F0530E942D500E94D44D3F
:105AAA0021F0ED8DFE8D0E94FD530E942D500E9423
:105ABA00415011F00E94F0530E942D500E944B5009
:105ACA0021F0EF8DF8A10E94FD530E942D500E94F3
:105ADA00505011F00E94F053AC85AA3121F40E9473
:105AEA00DF4CEBA7FCA7AC85AB3131F4E091390769
:105AFA00F0913A07EBA7FCA7AC85AC3129F4E09109
:105B0A005E05F0E0EBA7FCA7AC85AD3121F40E945D
:105B1A00444AEBA7FCA7AC85AE3121F40E94504A57
:105B2A00EBA7FCA7AC85AF3129F4E0910805F0E0BA
:105B3A00EBA7FCA7AC85A03229F4E0910A05F0E0B6
:105B4A00EBA7FCA7AC85A13229F4E0910B05F0E0A4
:105B5A00EBA7FCA7AC85A23229F4E0910C05F0E092
:105B6A00EBA7FCA7AC85A33229F4E0910D05F0E080
:105B7A00EBA7FCA7AC85A43229F4E0910E05F0E06E
:105B8A00EBA7FCA7AC85A53229F4E0912A05F0E041
:105B9A00EBA7FCA7AC85A63229F4E0912B05F0E02F
:105BAA00EBA7FCA7AC85A83229F4E0912D05F0E01B
:105BBA00EBA7FCA7AC85A93229F4E0912E05F0E009
:105BCA00EBA7FCA7AC85AA3229F4E0912F05F0E0F7
:105BDA00EBA7FCA7AC85AB3229F4E0913005F0E0E5
:105BEA00EBA7FCA7AC85AC3229F4E0913105F0E0D3
:105BFA00EBA7FCA7AC85AD3231F4E0913507F09103
:105C0A003607EBA7FCA7AC85AE3221F40E94C84A3E
:105C1A00EBA7FCA7AC85AF3231F4E0E031FCE1E060
:105C2A00F0E0EBA7FCA7AC85A03329F4E0911105BD
:105C3A00F0E0EBA7FCA7AC85A13321F4E8ADF0E0D6
:105C4A00EBA7FCA7AC85A23321F4EDA1FEA1EBA73B
:105C5A00FCA7AC85A33329F4E0911605F0E0EBA785
:105C6A00FCA7AC85A43329F4E0915905F0E0EBA731
:105C7A00FCA7AC85A53329F4E0915A05F0E0EBA71F
:105C8A00FCA7AC85A63329F4E0915B05F0E0EBA70D
:105C9A00FCA7AC85A73329F4E0915D05F0E0EBA7FA
:105CAA00FCA7AC85A83329F4E0914605F0E0EBA700
:105CBA00FCA7AC85A93329F4E0914705F0E0EBA7EE
:105CCA00FCA7AC85AA3329F4E0914805F0E0EBA7DC
:105CDA00FCA7AC85AB3329F4E091EE05F0E0EBA725
:105CEA00FCA7AC85AC3329F4E091C805F0E0EBA73A
:105CFA00FCA7AC85AD3329F4E0910205F0E0EBA7EF
:105D0A00FCA7AC85AE3329F4E091EF05F0E0EBA7F0
:105D1A00FCA70E9487500E94E15AE02129F0E091F5
:105D2A00F005F0E0EBA7FCA70E9487500E94ED5A0D
:105D3A00E02129F0E091F105F0E0EBA7FCA7AC85A2
:105D4A00A13429F4E091F906F0E0EBA7FCA7AC85B1
:105D5A00AC3529F4E0910705F0E0EBA7FCA7AC8588
:105D6A00AD3529F40E949650F0E0EBA7FCA7AC856C
:105D7A00AE3529F4E0915705F0E0EBA7FCA7AC8516
:105D8A00AF3521F4EDA5FEA5EBA7FCA7AC85A0369F
:105D9A0021F4EBA1FCA1EBA7FCA7AC85A13629F461
:105DAA00E0912605F0E0EBA7FCA7AC85A23631F41A
:105DBA000E94984FE081F0E0EBA7FCA70E94A25056
:105DCA000E94E15AE02129F0E0911D05F0E0EBA7DD
:105DDA00FCA70E94A2500E94ED5AE02129F0E0910E
:105DEA001E05F0E0EBA7FCA7AC850E940448AC8531
:105DFA00E3E00E940954E1E10E940954E2E10E94B1
:105E0A000954E3E10E940954E5E10E940954EAE1D8
:105E1A000E940954EBE10E940954EDE10E940954E1
:105E2A00EEE20E94A65AE0291E2E0E940E540E94FB
:105E3A00CF5AE0211E2AAC85EEE50E94A65A0E2E04
:105E4A00A0915705E2E00E94C45A0E22E5E00E94A2
:105E5A00BF5AE021E12911F0F59A01C0F598A0E0B6
:105E6A00F599A1E0EA2FE795E0E0E7955E2F40E09B
:105E7A00E0E00E940751E0E0E0930305FE01E359E8
:105E8A00FF4F3396BF01AC85B0E0A7FDBFEF0E947C
:105E9A00D6510E94EC510E94C151BF01AC85B0E0BD
:105EAA00A7FDBFEF0E942652ABA5BCA5A031E7E231
:105EBA00BE0738F00E947D52BF01ABA5BCA50E9467
:105ECA001854ABA5BCA5A83EE3E0BE0738F00E9473
:105EDA009D52BF01ABA5BCA50E948053ABA5BCA532
:105EEA00A436E0E0BE0748F00E94A252BF01ABA56B
:105EFA00BCA50E94314D0E945452ABA5BCA51A976D
:105F0A0030F00E9462520E941D540E9454520E9414
:105F1A00B352BF01ABA5BCA50E946653EC85E03025
:105F2A0061F4ECE10E942154E0E50E942D52EDE675
:105F3A000E942454E0E50E945053AC85A13079F4C4
:105F4A00EBE50E942154EDE60E942B5411F40E94C5
:105F5A003054ABA5BCA5119711F40E943654AC85F8
:105F6A00A23031F4EDE60E942151E3E70E94395450
:105F7A00AC85A33031F4EEE50E943C54E7E70E9479
:105F8A002D52AC85A83069F40E943F540E942B54CC
:105F9A0011F40E943054ABA5BCA5119711F40E94CC
:105FAA003654AC85AA3049F50E944554E4E50E946E
:105FBA002B5471F4EEE30E942C53E0E00E947953D3
:105FCA00E8E70E9450530E945B53EDE30E94495454
:105FDA00ABA5BCA5119789F4E9E30E942C53EEE323
:105FEA000E9431530E942153E0E50E945053E9E791
:105FFA000E946953E4E50E944C54AC85AB3041F5EC
:10600A00EDE60E943C54EDE30E942B5471F4EDE658
:10601A000E943153E7E60E944F54EEE30E94505328
:10602A000E945B53E0E50E944954ABA5BCA51197B9
:10603A0079F4EDE60E944F54E0E30E945053E4E500
:10604A000E946953EEE30E946E53EDE60E94C65326
:10605A00AC85AC3031F4EEE30E945454ECE70E9474
:10606A002D52AC85E1E10E94EB53E2E10E94095412
:10607A00E3E10E940954E5E10E940954EDE10E941E
:10608A000954EEE20E94A65AE02931F00E946252B7
:10609A000E941D540E9454520E944B4F0E94AF4BC3
:1060AA00E093FF06F0930007E7E2E0937A00AC85FD
:1060BA000E941C53AC85EEE00E940954E1E10E9463
:1060CA00A65AE02911F0E1E07E2EAC85E6E00E94B6
:1060DA00EB53EFE00E940954E2E10E94A65AE0293C
:1060EA0011F0E2E07E2EAC85E7E00E94EB53E0E19E
:1060FA000E9409540E94575411F0E3E07E2EA091A9
:10610A00FF06B0910007D39708F468C00E945C5458
:10611A000E94104DE72D0E94174D0E946154A091D4
:10612A003107B0913207A93CE0E0BE0720F0E8EC65
:10613A00F0E00E946154E72D0E94234DA09131079F
:10614A00B09132070E9466540E9461540E946A54B8
:10615A00AC91A13008F441C00E9471540E947A5453
:10616A000E942E5C4CF40E946A540E9483540E943E
:10617A003A5A0E948D5423C00E9496540E94674D39
:10618A00EF930E9496540E94704DAF91EA2379F0E2
:10619A000E946A540E9483540E943F5AA093AE07F9
:1061AA00B093AF078093B0079093B10708C00E94DD
:1061BA0096540E94794D1CF00E9498540EC0A091EA
:1061CA00AE07B091AF078091B0079091B1070E94D6
:1061DA008B4D0E94985B0E94615407C0E0E0E093F7
:1061EA003107E09332070E949854AC85AD3051F5DF
:1061FA000E941252FF93EF930E94D6500E94A75218
:10620A000E948252AF91BF91EC930E941C52FF935D
:10621A00EF930E94D6500E94E6520E948252AF919A
:10622A00BF91EC930E942152FF93EF930E94D650A4
:10623A000E94E6520E94AE5BAF91BF91EC93E0E2FE
:10624A000E940751AC85A53149F4EEE30E94215121
:10625A00ECE00E942651E0E60E940751AC850E94BC
:10626A001C53AC85EEE00E940954E1E10E94A65A53
:10627A00E029F9F00E94A054E4E00E94AB5440F0F7
:10628A000E9412520E94B4540E94314D0E945452EC
:10629A000E94BA5440F00E941C520E94B4540E94B8
:1062AA00344F0E9454520E9421520E94B4540E94B8
:1062BA006653AC85E6E00E94EB53EFE00E94095476
:1062CA00E2E10E94A65AE029F9F00E94A054E2E015
:1062DA000E94AB5440F00E9412520E94B4540E9491
:1062EA00314D0E9454520E94BA5440F00E941C52EE
:1062FA000E94B4540E94344F0E9454520E94215268
:10630A000E94B4540E946653AC85E7E00E94EB53A6
:10631A00E0E10E9409540E945754F9F00E94A054E7
:10632A00E1E00E94AB5440F00E9412520E94B45421
:10633A000E94314D0E9454520E94BA5440F00E9469
:10634A001C520E94B4540E94344F0E9454520E941C
:10635A0021520E94B4540E946653AC850E941C5379
:10636A000E94C0541E2EAC85E6E00E94A65A0E2E4C
:10637A000E94C0541E2AAC85E7E00E94A65A0E2E3F
:10638A000E94C054E12909F46CC0E0914705E0304D
:10639A0061F4E72D0E94234DAB8DBC8D0E94C3543E
:1063AA00DF010E94314D0E94C754A0914705A130D8
:1063BA0061F4E72D0E94234DAD8DBE8D0E94C3541A
:1063CA00DF010E94314D0E94C754A0914705A230B7
:1063DA0059F40E94CC540E942D4F0E94344FDB0185
:1063EA000E9466540E94C754A0914705A33071F4D5
:1063FA00E72D0E94234DAF8DB8A10E94C354DF013F
:10640A00E2E3F0E00E945B5B0E94C754A09147055B
:10641A00A43099F40E94CC54ED8DFE8D0E94DE4882
:10642A000E94FF49A9A1BAA1AE0FBF1F0E94344F13
:10643A00DB010E9466540E94C7540E94BA5440F07D
:10644A000E9412520E94B4540E94344F0E94545225
:10645A000E941C520E94B4540E946653E7E70E94AD
:10646A002D52AC85A431E1F40E9412520E94D654F6
:10647A000E94314D0E9454520E941C520E94D654CE
:10648A000E94344F0E9454520E9421520E94D654B4
:10649A000E946653EBA5FCA5309711F40E94305474
:1064AA00AC85A63199F40E943F540E942D52EBE02C
:1064BA000E942C53EBA5FCA5309711F40E9430548E
:1064CA00ABA5BCA5119711F40E943654AC85A7312F
:1064DA0039F40E943F540E942D52E0E40E942C534A
:1064EA00AC85A83199F40E943F540E942D52ECE0E9
:1064FA000E942C53EBA5FCA5309711F40E9430544E
:10650A00ABA5BCA5119711F40E943654AC85A931EC
:10651A0031F50E941252BF01A885B9850E9417520F
:10652A000E941C52BF010E94D9500E94EC51A985B9
:10653A00AA2392F40E941252BF01E885F9850E94AB
:10654A0019530E94EC510E941C52BF01E885F9853B
:10655A000E9402520E94EC51E7E70E942D52AC853C
:10656A00AA31F9F40E94DC54A436E0E0BE0748F0F0
:10657A000E941252BF010E94DC540E94314D0E94B7
:10658A0054520E941C52BF010E94DC540E94344F94
:10659A000E9454520E942152BF010E94DC540E9460
:1065AA006653AC85AB3161F4ECE70E945454E8E7DA
:1065BA000E942D520E9462520E941D540E945452FF
:1065CA00AC85AC31C9F4E0E30E942151EDE60E94AA
:1065DA002651E4E50E942B5429F4E1E00E946E530F
:1065EA000E947353ABA5BCA5119731F4E0E00E9459
:1065FA006953EEE30E944C54AC85EDE10E94EB53E3
:10660A00EEE10E94A65AE02921F1E3E70E942C5309
:10661A00E8E30E943153AC85AD3111F4EEE501C0D7
:10662A00E8E7DE01A858BF4FEC930E94E1541A979D
:10663A0048F00E941C52BF010E94E1540E94344F4C
:10664A000E9454520E942152BF010E94E1540E94AA
:10665A006653AC85AF3149F4EEE30E942151EDE671
:10666A000E942651E3E70E942D52AC85EFE10E9479
:10667A00BA5A0E2EE5E20E94B55AE021D1F0EDE6B3
:10668A000E942151E8E50E94E654DF01EC85EF51B2
:10669A00EC93EBA5FCA5309761F4E1E00E9431533D
:1066AA00EDE30E944F54E4E50E94E854E0E50E94BD
:1066BA004954AC85A53241F40E94EB54E5E00E94AE
:1066CA002B5411F40E943054AC85A63241F40E9436
:1066DA00EB54E8E00E942B5411F40E943054AC852C
:1066EA00A73209F045C00E94EF54E3E60E942D52FA
:1066FA00E0912C05E03061F4EEE50E945053E0E3AE
:10670A000E946953EDE60E946E53E3E70E94C65366
:10671A00A0912C05A13079F4E7E30E944F54ECE5EF
:10672A000E945053E8E70E946953ECE50E946E53B9
:10673A00E0E50E94C653A0912C05A23031F4ECE7A3
:10674A000E946953E7E70E944C54A0912C05A3309C
:10675A0079F4E9E30E944F54ECE50E945053E4E5D2
:10676A000E946953E8E70E946E53E0E50E94C6530F
:10677A00AC85A832C1F40E94EF54E8E70E942D527A
:10678A00A0912D05A13079F4E8E30E944F54E7E384
:10679A000E945053E3E00E946953E5E00E946E5361
:1067AA00EEE50E94C653AC85A932F9F4E7E70E94E8
:1067BA002151E0E40E94F354E0912E05E03019F4EF
:1067CA00E7E70E94C653A0912E05A13039F40E9432
:1067DA005B530E94DA52E8E70E94C653A0912E0545
:1067EA00A23019F4E8E70E94C653AC85AA3259F4DC
:1067FA00E9E30E94F6540E942B51EBA5FCA53097C1
:10680A0011F40E943054AC85AB3249F4E9E30E949A
:10681A002151E0E50E942651EEE00E942D52AC85FE
:10682A00AC3259F5ECE70E942151E0E50E9426516D
:10683A00E0E50E942B5491F4E4E50E943153E0E034
:10684A000E944F54EAE00E945053E0E50E946953C7
:10685A00E9E70E946E53E5E00E94C653ABA5BCA5CA
:10686A00119759F40E942153E9E70E945053E5E039
:10687A000E946953E9E70E944C54AC85AD3231F469
:10688A00E0E00E94F654E0E00E942D52AC850E949E
:10689A001C53AC85E6E00E940954E7E00E94A65A20
:1068AA00E02919F0E3E70E942C53AC85EEE00E9440
:1068BA00EB53EFE00E940954E0E10E94A65AE02956
:1068CA0031F0EDE60E942C53E9E70E942454AC858E
:1068DA00E1E10E94EB53E2E10E9409540E945754FD
:1068EA0019F0E8E70E943153AC85AE3219F4E9E3B6
:1068FA000E94F954AC85AF3291F4E8E70E94215125
:10690A00E5E00E942651ECE10E942B5411F40E940A
:10691A003054ABA5BCA5119711F40E943654AC852E
:10692A00A03379F4E0E30E942154E0E50E942B545D
:10693A0011F40E943054ABA5BCA5119711F40E9422
:10694A003654AC85A133B1F4E3E70E942151E0E566
:10695A000E94F354A0910405A43160F0E4E50E947A
:10696A002C53EDE60E943153E0E30E944F54EDE3CD
:10697A000E945053AC85A23349F4EEE30E942151A0
:10698A00EBE00E942651E0E60E9407510E940E5455
:10699A000E94C95AE02111F00E943054AC85A333F9
:1069AA0031F4E3E70E942151E4E70E943954AC85AF
:1069BA00A43369F4E8E70E94F9540E948953ABA50D
:1069CA00BCA5A338E0E0BE0711F40E943054AC85A0
:1069DA00A53369F4E8E70E94F9540E949A53ABA5DB
:1069EA00BCA5A734E0E0BE0711F40E943054AC8580
:1069FA00A63369F4E8E70E94F9540E949F53ABA5B5
:106A0A00BCA5A536E0E0BE0711F40E943054AC855F
:106A1A00A73379F4E8E30E943C54ECE70E942B5434
:106A2A0011F40E943054ABA5BCA5119711F40E9431
:106A3A003654AC85A83379F4E8E30E943C54E7E77E
:106A4A000E942B5411F40E943054ABA5BCA5119797
:106A5A0011F40E943654AC85A93359F5E7E70E9430
:106A6A00FC54E0914705E03029F4E1E00E94E85443
:106A7A000E94FF54A0914705A13011F40E940355CA
:106A8A00A0914705A23021F40E9408550E94FF54A4
:106A9A00A0914705A33029F4E0E00E94E8540E943F
:106AAA000C55A0914705A43021F40E9408550E9474
:106ABA000C55AC85AA3359F5ECE70E94FC54E091D9
:106ACA004805E03029F4E1E00E94E8540E94FF54AE
:106ADA00A0914805A13011F40E940355A0914805E0
:106AEA00A23021F40E9408550E94FF54A091480543
:106AFA00A33029F4E0E00E94E8540E940C55A091CA
:106B0A004805A43021F40E9408550E940C55AC8512
:106B1A00AB3351F4E5E00E94FC540E94B352DF010A
:106B2A00E091EE05EF5FEC93AC85AC3311F5406173
:106B3A00E8E30E942151E9E30E942651EEE50E9412
:106B4A002D52E1E00E942C530E9478520F01A0912D
:106B5A00C805E3E0EA1BD001EC93ECE70E9450532E
:106B6A00E1E00E946953E7E70E946E53E5E00E9464
:106B7A00C653AC85AD3339F5E8E70E942151E1E00F
:106B8A000E942651E4E50E942D520E9410550E944F
:106B9A003252A0910205AA3010F00E946C520E9453
:106BAA0072520E94C250DB01EC930E947852BF01DC
:106BBA000E946E500E94EC510E947D52BF010E94B9
:106BCA007650DB01EC93AC85AE3371F4E3E70E94B7
:106BDA002151ECE70E9426510E942B51EBA5FCA5FE
:106BEA00309711F40E943054AC85AF33C1F4E8E316
:106BFA000E942151ECE70E9426510E94AA4F18F4E4
:106C0A00ECE00E942D520E94AA4F18F0EBE00E947D
:106C1A002D52EBA5FCA5309711F40E943054AC8597
:106C2A00A03459F5E9E30E942151E0E00E9426517F
:106C3A00EEE50E942D520E949D52BF01A091F406DA
:106C4A000E94BC500E94EC510E94A252BF01A09126
:106C5A00F406BB270E9426520E946252BF01A091ED
:106C6A00F5060E94BC500E94EC510E94B352BF012B
:106C7A00A091F506B0E00E942652AC85A13431F409
:106C8A00E4E70E945454E1E00E942D52AC85AB35F2
:106C9A0009F044C0E8E70E942151E5E00E94F3545C
:106CAA00A0914D07A03044F0E0914D07F0E0E7FDD8
:106CBA00FFEFEBA7FCA732C0E0914D07F0E0E7FD3C
:106CCA00FFEF0E94445AEBA7FCA7ABA5BCA50E9404
:106CDA006A4A0E2EABA5BCA5EAE0F0E00E94E75A8C
:106CEA00E02119F0EDE00E946E53ABA5BCA5E9E0E6
:106CFA00F0E00E94ED5A0E2EE4E6F0E00E94E75A18
:106D0A00E02119F0EDE00E946953ABA5BCA5A436B9
:106D1A00E0E0BE0718F0EDE00E945053AC85AC35B8
:106D2A0029F40E944554E9E30E942D52AC85AD3501
:106D3A0009F053C10E949150A83008F049C0E7E712
:106D4A000E942151EEE50E94E6540E949150A083D0
:106D5A000E94254AE7EAE0937A000E9491500E9435
:106D6A003501E0930107F0930207E7E2E0937A0026
:106D7A000E941455A83EE3E0BE0738F00E949D52D7
:106D8A00BF010E9414550E9480530E941455A436D4
:106D9A00E0E0BE0748F00E94A252BF010E941455CB
:106DAA000E94314D0E9454520E9414551A9748F07D
:106DBA000E946252BF010E9414550E94344F0E94E1
:106DCA0054520E94B352BF010E9414550E94665346
:106DDA000E949150E7E00E941955ECE00E94BF5AC8
:106DEA00E02121F1E6E70E942151E8E30E94E654FE
:106DFA00DF010E949650E750EC93E7E70E941D5589
:106E0A00E9E30E9420550E942255E170EC930E940A
:106E1A0062520E942255E695E170EC930E94B352A9
:106E2A000E942255E695E695E170EC930E949150F6
:106E3A00EBE00E941955E0E10E94BF5AE02171F18E
:106E4A00E1E00E942151E4E50E94E654DF010E943C
:106E5A009650EB50EC930E947D520E942A55E170A5
:106E6A00EC930E949D520E942A55E695E170EC939C
:106E7A000E94A2520E942A55E695E695E170EC938B
:106E8A000E9462520E942A550E943255EC930E9437
:106E9A00B3520E942A55E295E170EC930E949150F8
:106EAA00EFE00E941955E4E10E94BF5AE02161F126
:106EBA005068EEE30E943755DF010E949650EF506A
:106ECA00EC930E94A2520E9439550E94314D0E94B1
:106EDA005452FE01E658FF4FE081E03011F40E945F
:106EEA0055530E9462520E9439550E94344F0E94A3
:106EFA0054520E94B3520E9447557097A5E2B7E0D8
:106F0A000E944B550E9454520E949150E3E10E9404
:106F1A001955E8E10E94BF5AE02109F45EC05068A1
:106F2A00E7E70E943755DF010E949650E351EC9340
:106F3A000E945255FF231AF10E94A2520E944755FD
:106F4A000E9458550E94F2500E94EC510E945C55D2
:106F5A00E03011F40E9455530E9462520E94475534
:106F6A000E945855DF010E94D6510E94EC510E949E
:106F7A00B3520E9447550E9458550E94EC510E94F4
:106F8A005255FF2352F5EDE00E9469530E94525573
:106F9A00ED39AFEFFA076CF4EDE00E9450530E940E
:106FAA00A2520E9447550E9458550E9419530E94A6
:106FBA00EC510E9462520E9447550E9458550E9405
:106FCA0002520E94EC510E94B3520E9447550E94FD
:106FDA0058550E94445A0E94EC51AC85AE3509F0CE
:106FEA00BCC1EDE60E942151E8E70E942651E7E77D
:106FFA000E942D52E0915705E030C1F4EDE60E945F
:10700A006155A0910A08AA3048F00E946252BF0155
:10701A00A0910A080E94BC500E94EC510E94B352EF
:10702A00BF01A0910A08BB270E942652A0915705CA
:10703A00A130E9F4E0E30E941D55EBE00E944F54B1
:10704A000E94FA491A9748F00E94A252BF010E9470
:10705A00FA490E94344F0E9454520E946252BF0160
:10706A000E94FA490E946653E7E70E94C653A0911C
:10707A005705A230D9F4E0E30E946155A0910B08AC
:10708A00AA3048F00E94A252BF01A0910B080E94A8
:10709A00BC500E94EC510E946252BF01A0910B08A1
:1070AA00BB270E942652E7E70E94C653A0915705C4
:1070BA00A330E9F4EEE30E941D55ECE00E9420554E
:1070CA00BF010E94BE490E94314D0E9454520E9443
:1070DA006252BF010E94BE490E94344F0E9454521C
:1070EA000E94B352BF010E94BE490E946653A091FA
:1070FA005705A430E9F4EEE30E941D55EBE00E9427
:10710A002055BF010E94C8490E94314D0E94545225
:10711A000E946252BF010E94C8490E94344F0E94D5
:10712A0054520E94B352BF010E94C8490E9466533A
:10713A00A0915705A530B9F5E3E70E942C53EBE07F
:10714A000E9431530E94D249A83EE3E0BE073CF0B8
:10715A000E947D52BF010E94D2490E9410530E9490
:10716A00D249A436E0E0BE073CF00E949D52BF011E
:10717A000E94D2490E9417520E94D2491A974CF093
:10718A000E94A252BF010E94D2490E94D6510E9477
:10719A00EC510E946252BF010E94D2490E942652BB
:1071AA00EEE30E94C653A0915705A63059F5E8E7C9
:1071BA000E942C53E0E00E9466550E94DC49A436E6
:1071CA00E0E0BE0748F00E947D52BF010E94DC4900
:1071DA000E94314D0E9454520E94DC491A9748F08D
:1071EA000E949D52BF010E94DC490E94344F0E94B6
:1071FA0054520E94A252BF010E94DC490E94665367
:10720A000E946955A0915705A73059F5E8E70E94F1
:10721A002C53E1E00E9466550E94E649A436E0E05C
:10722A00BE0748F00E947D52BF010E94E6490E94B3
:10723A00314D0E9454520E94E6491A9748F00E9422
:10724A009D52BF010E94E6490E94344F0E94545247
:10725A000E94A252BF010E94E6490E9466530E9400
:10726A006955A0915705A83059F5E8E70E942C53B3
:10727A00E2E00E9466550E94F049A436E0E0BE07AB
:10728A0048F00E947D52BF010E94F0490E94314D90
:10729A000E9454520E94F0491A9748F00E949D5247
:1072AA00BF010E94F0490E94344F0E9454520E942A
:1072BA00A252BF010E94F0490E9466530E9469557A
:1072CA00A0915705A93009F048C0ECE70E942C5359
:1072DA00E0E50E9431530E94994AA031E7E2BE07D5
:1072EA0030F00E9472520E94994A0E9418540E94D9
:1072FA00994AA83EE3E0BE0738F00E947852BF01DF
:10730A000E94994A0E9480530E94994AA436E0E05A
:10731A00BE0748F00E947D52BF010E94994A0E940E
:10732A00314D0E9454520E94994A1A9748F00E947D
:10733A009D52BF010E94994A0E94344F0E945452A2
:10734A000E94A252BF010E94994A0E946653E4E534
:10735A000E946E53E7E70E94C653AC85AF3549F5E4
:10736A00E885F9850E94DB51A985AA2342F4E091B8
:10737A005E07F0915F070E94445A0E94DB510E9407
:10738A001252BF010E94E0510E9417520E941C52E1
:10739A00BF010E94E0510E94D6510E94EC510E9406
:1073AA0021520E94F951EEE50E942C53E1E00E941D
:1073BA003153AC85A03631F4E8E30E94F654EDE08F
:1073CA000E942D52AC85A13631F4E8E70E9454544C
:1073DA00EEE30E942D52AC85A23649F4E8E30E94FE
:1073EA003755A0913305A083E0E10E940751AC858F
:1073FA00A33679F4E8E30E94F6540E94AA4F18F4DF
:10740A00ECE00E942D520E94AA4F18F0EBE00E9475
:10741A002D52A0E0F099A1E00E940448A82D0E94F4
:10742A00AA4B61F15F774F7EEAE00E942C53E0E0BD
:10743A000E943153E1E70E944F54E1E70E94D95379
:10744A000E941055A0914B05A130C0F0A23319F447
:10745A00E1E0E0934305A0914B05A13319F4E0E084
:10746A00E0934305A0914B05AD3219F4E1E0E093B6
:10747A004305E0914B05E150E0934B05A091F806D6
:10748A00A13061F5EAE0DE01AB58BF4FEC93E3E7C8
:10749A000E942C530E947852BF01A091F6060E94C6
:1074AA00BC500E94EC510E947D52BF01A091F60689
:1074BA00B0E00E9426520E949D52BF01A091F70699
:1074CA000E94BC500E94EC510E94A252BF01A0919E
:1074DA00F706B0E00E9426520E94105531E0303182
:1074EA0008F089C00E94E353EC91E03021F40E9435
:1074FA00E353EFE3EC930E94E353AC91A63021F4FB
:10750A000E94E353EDE7EC930E94E353AC91A13060
:10751A0021F40E94E353E6E0EC930E94E353AC911A
:10752A00A23021F40E94E353EBE5EC930E94E3536B
:10753A00AC91A33021F40E94E353EFE4EC930E9450
:10754A00E353AC91A43021F40E94E353E6E6EC93B2
:10755A000E94E353AC91A53021F40E94E353EDE677
:10756A00EC930E94E353AC91A73021F40E94E353B9
:10757A00E7E0EC930E94E353AC91A83021F40E9417
:10758A00E353EFE7EC930E94E353AC91A93021F463
:10759A000E94E353EFE6EC930E94E353AC91AA30C6
:1075AA0021F40E94E353E0E0EC930E94E353AC9190
:1075BA00AB3021F40E94E353E1E0EC930E94E353E1
:1075CA00AC91AC3021F40E94E353E8E0EC930E94C2
:1075DA00E353AC91AD3021F40E94E353E0E4EC9321
:1075EA000E94E353AC91AE3021F40E94E353E9E0E8
:1075FA00EC933F5F74CFFE01E45AFF4F31960F01BF
:10760A00E0910305E695E6950E946D550E94725534
:10761A000E9477550E9472550E9481550E947255A8
:10762A000E948A550E947255E1700E949255E69511
:10763A00E170EE0F0E9492550E9495550E94925554
:10764A000E949B550E949F5532960F01E0910305B7
:10765A000E943255E295E07F0E94A6550E94775516
:10766A000E94AC550E9481550E94AC550E948A55D1
:10767A000E94B155E1700E94B655E695E170EE0F91
:10768A000E94B6550E9495550E94B6550E949B5578
:10769A000E949F5533960F01E0910305E6950E94DB
:1076AA006D550E94B1550E9477550E94B1550E94AE
:1076BA0081550E94B1550E948A550E94AC55E170CD
:1076CA00EA2B0E94A6550E94B9550E94A6550E940F
:1076DA009555EA2B0E94A6550E949B550E949F55DC
:1076EA0034960F01FE01EB58FF4FE0810E946D5561
:1076FA000E94BE550E9477550E94BE550E94815530
:10770A000E94BE550E948A55E52FE170EA2BAE2FE2
:10771A00E52F0E94B955AE2FE52F0E949555EA2B09
:10772A00AE2FE09103050E94A4530E949F553596FF
:10773A000F010E945C550E946D550E945C550E9483
:10774A00C3550E945C550E94CB550E945C550E940D
:10775A0032550E94D2550E9432550E94D9550E9434
:10776A00DC550E94D9550E94E2550E94D955E295EE
:10777A000E94A4530E949F5536960F010E94EA5513
:10778A000E946D550E94EA550E94C3550E94EA550F
:10779A000E94CB550E94EA550E9432550E94D2554A
:1077AA00E295E1700E94EF550E94DC550E94EF5568
:1077BA000E94E2550E94EF55E2950E94A4530E944E
:1077CA009F5537960F01E52F0E94F6550E94EA55FC
:1077DA000E9477550E94EA550E9481550E94EA55F7
:1077EA000E948A550E94FA55E1700E94FF550E9434
:1077FA00B955AE2F0E94FA550E9495550E94FF5521
:10780A000E949B550E949F5538960F010E9402566E
:10781A000E946D550E9402560E94C3550E9402564C
:10782A000E94CB550E9402560E9432550E94D255A0
:10783A000E940756E1700E94FF550E94DC550E9483
:10784A00FF550E94E2550E94FF55E2950E94A453FB
:10785A000E949F5539960F010E940C560E946D5541
:10786A000E940C560E94C3550E940C560E94CB558A
:10787A000E940C560E9432550E94D255EE1FE0E03B
:10788A00EE1FE1700E9411560E94DC550E941156AB
:10789A000E94E2550E941156E2950E94A4530E944A
:1078AA009F553A960F01E42FE2950E946D550E946A
:1078BA000C560E9477550E940C560E9481550E94D0
:1078CA000C560E948A550E94BE55E170EA2BAE2FD3
:1078DA000E94BE550E94B955AE2F0E94BE550E9405
:1078EA009555EA2BAE2F0E94BE550E949B550E94C9
:1078FA009F553B960F010E9418560E946D550E9493
:10790A0018560E94C3550E9418560E94CB550E94D1
:10791A0018560E9432550E941D56E0E030FCE1E004
:10792A000E942356E295E170EE0F0E9423560E94B0
:10793A00E2550E942356E295EF70E6950E94A45301
:10794A000E949F553C960F01FE01E259FF4FE081CC
:10795A000E943255E295E07FAE2FFE01E259FF4FB9
:10796A00E081E695E6950E942A560E942356E695FE
:10797A00E1700E9482510E942356E1700E941D56B6
:10798A00E42F0E943255EA2BAE2FE42F0E942F5685
:10799A00E42F0E943656E42FE6950E94A4530E94D3
:1079AA009F553D960F01E42F0E94F6550E943C56C2
:1079BA00E2950E942A56EA2BAE2F0E943C560E945C
:1079CA0081550E943C560E9441560E943C560E9494
:1079DA003255EA2BAE2F0E943C560E942F560E9427
:1079EA003C56E6950E9436560E943C560E94A45385
:1079FA000E949F553E960F01E42F0E9407560E944F
:107A0A006D550E9402510E942A560E944656E695DA
:107A1A00E1700E9482510E944656E695E695E17011
:107A2A000E941D56E0910305E295E170EA2BAE2F04
:107A3A00E42FEE1FE0E0EE1FE170EE0F0E944656C3
:107A4A000E943255EE0FEE0F0E944656E2950E94B2
:107A5A00A4530E949F553F960F010E9402510E9413
:107A6A00F6550E944956E2950E942A56EA2BAE2FF5
:107A7A000E9449560E9481550E9449560E944156C9
:107A8A000E944E560E943255EA2BAE2F0E944E5645
:107A9A000E942F560E944E56E6950E9436560E9424
:107AAA004E560E94A4530E949F5570960F010E9441
:107ABA0002510E9407560E946D550E944E56E29549
:107ACA000E942A56EA2BAE2F0E944E560E948155DA
:107ADA000E944E560E9441560E9449560E943255B3
:107AEA00EA2BAE2F0E9449560E942F560E944956F1
:107AFA00E6950E9436560E9449560E94A453EA2BE4
:107B0A00D001EC93A091F806A23071F431E0313142
:107B1A0030F40E945356E0E0EC933F5FF8CFE4E084
:107B2A00DE01A859BF4FEC9326FE09C031E031317E
:107B3A0030F40E945356EFEFEC933F5FF8CF0E9468
:107B4A005B563D3008F50E946156A091C805A130E8
:107B5A0061F4ECE0E31BA0E5B8E00E94615AE17031
:107B6A0011F4429801C0429A0BC0ECE0E31BA2E573
:107B7A00B8E00E94615AE17011F4429801C0429A39
:107B8A000E9466563F5FDDCF0E946E563D3088F4F4
:107B9A000E946156ECE0E31BA0E3B8E00E94615A40
:107BAA00E17011F4429801C0429A0E9466563F5F02
:107BBA00EDCF0E946E563D3088F40E946156ECE08B
:107BCA00E31BA2E0B8E00E94615AE17011F4429806
:107BDA0001C0429A0E9466563F5FEDCF0E946E56E0
:107BEA003D3088F40E946156ECE0E31BA6E0B8E061
:107BFA000E94615AE17011F4429801C0429A0E94AF
:107C0A0066563F5FEDCF0E946E563D30A8F50E9442
:107C1A0061560E9477560E947B56A0E0F099A1E037
:107C2A000E94D44D1E2E0E9477560E947B56A0E0D9
:107C3A00F099A1E00E94A54BA82D0E94AA4BE12928
:107C4A0061F0ECE0E31BA2E1B8E00E94615AE17046
:107C5A0011F4429801C0429A0BC0ECE0E31BA0E188
:107C6A00B8E00E94615AE17011F4429801C0429A48
:107C7A000E9466563F5FC9CF0E9477560E947B5684
:107C8A00A0E0F099A1E00E94D44D1E2E0E947756E2
:107C9A000E947B56A0E0F099A1E00E94A54BA82D76
:107CAA000E94AA4BE12919F0E1E0E0934205E09134
:107CBA004305E03019F4E0E0E0934205429A84E09B
:107CCA008A95F1F7449A84E08A95F1F7449884E01A
:107CDA008A95F1F731E03A3088F40E946156E9E07A
:107CEA00E31BA0E4B1E00E94615AE17011F44298EA
:107CFA0001C0429A0E9466563F5FEDCF21E02131D2
:107D0A00E0F431E03930B8F40E946156E22FF0E035
:107D1A00DE01A45ABF4FAE0FBF1FAC91E8E0E31BD0
:107D2A000E94505AE17011F4429801C0429A0E948E
:107D3A0066563F5FE7CF2F5FE2CF429A88E28A9585
:107D4A00F1F7449A8CE291E00197F1F7A62D0E948F
:107D5A000448A92D0E947F56AB2D0E947F56AA2D5A
:107D6A000E947F560E949E4F0E2AA885B985EBEF86
:107D7A00FFEF0E94D55A0E2A0E94394F0E2A0E94FE
:107D8A00C14DE02929F0E0E0E0931B07E0931C07CE
:107D9A00F09B03C0E0E0E0934305A82D0E942F4A20
:107DAA00A0E0F099A1E00E94AA4B29F00E94254A7E
:107DBA00F09AE89426F8A0910405AE3128F4E091EF
:107DCA000405EF5FE0930405A0910405AE31C9F400
:107DDA00E0E0E887E987E0933905E0938407E093D8
:107DEA008507A8ADA43019F00E94094A02C00E9472
:107DFA00174AE0933A05E0E0E0932F08E4E1E093C4
:107E0A000405E8ADE03031F50E948456ECE30E94A7
:107E1A008A56E7E00E949056EBE00E94A65AE021BB
:107E2A0089F0E0912008E0933805E0912108E09379
:107E3A003905A0912208EAE0EA9FF001E887F9876C
:107E4A000E949656A0912F08AC3020F00E94AD56A1
:107E5A000E94BA56A8ADA13009F50E948456E8E2FC
:107E6A000E94A65A0E2EA0912F08E8E00E94A65A58
:107E7A00E02161F0E1E0E0933805E0912208F0E0CA
:107E8A00E0938407F09385070E949656A0912F08E5
:107E9A00AC3020F00E94AD560E94BA56A8ADA3306D
:107EAA0009F057C00E948456ECE60E948A56EBE01D
:107EBA000E949056EFE00E94A65AE02109F443C0BE
:107ECA00E0912108E0933805E0912208E093390512
:107EDA00E0912308F0E0E887F987F885E0E0E88791
:107EEA00F987E0912408F0E0A885B985EA0FFB1F1D
:107EFA00E887F987E0912508E0935605E09128087C
:107F0A00E0935205E0912908FF2766277727E09337
:107F1A003D07F0933E0760933F0770934007E09157
:107F2A002A08E0933A05E0912608F0E0E0938607F4
:107F3A00F0938707E0912708F0E0E0938E07F0932B
:107F4A008F070E94C656A0912F08A03110F00E94F8
:107F5A00CC56A8ADA43009F01FC1A0911E08EBE6CB
:107F6A000E948A56EFE00E949056E0E10E94A65ACB
:107F7A00E02109F40BC1E0912108E370E093D505F3
:107F8A00A091D505B0E0AF52BA4FE09120080E9407
:107F9A00ED560E94F256AA52BA4F0E94F956E69539
:107FAA000E94FD56A652BA4F0E94F956E6950E94C3
:107FBA00FD56A252BA4F0E94F956E695EC93E0910B
:107FCA00D505F0E0E252FA4F7E2F8F2F6081E091C3
:107FDA002108E170AE2FE0E0F799E1E0EA02F00152
:107FEA00E62BA72FB82F0E94ED560E94F256AE51EB
:107FFA00BA4FE0912108E170EC930E940257AE0F4C
:10800A00BF1FF0912208E0E0ED93FC930E94025713
:10801A000E940A57E09123080E9412570E941B5798
:10802A00AE0FBF1FF0912408E0E00E9421570E9482
:10803A001B570E940A57E09125080E9412570E9476
:10804A00BC4CE0912608FF27662777270E94F15B40
:10805A00A091D505B0E0A65CBA4FE09127080E942E
:10806A00FD56AE5ABA4FE0912808E770EC93A8E2A1
:10807A00B8E0EC91E695E695E6950E94FD56AA5180
:10808A00BA4FE09128080E9426570E942F57A6E966
:10809A00B7E00E9437570E9426570E940A57E0917C
:1080AA002C080E9412570E9448570E942F57AEE888
:1080BA00B7E00E943757EC93E091D5050E944857E4
:1080CA000E940A57E0912B080E9412570E944E57AD
:1080DA000E942F570E944E57AE0FBF1FED91FD9180
:1080EA00FE2FE0E0FE93EE93E091D5050E944E57F5
:1080FA000E940A57E0912A08F0E0EA0FFB1FD0011C
:10810A00ED93FC930E94C656E989FA89AF85B8892E
:10811A00EA0FFB1FAB89BC89EA0FFB1FAD89BE8939
:10812A00EA0FFB1FE887F987E0E0E0933905E09161
:10813A00D605EE0FA091DA05AE0FE091DE050E949A
:10814A005457A091DB05E091D705EE0FAE0FE091F1
:10815A00DF050E945457A091DC05E091D805EE0F87
:10816A00AE0FE091E0050E945457A091DD05E09121
:10817A00D905EE0FAE0FE091E1050E945457E09148
:10818A00D505F0E0E651FA4FA0E0A083A0912F08B0
:10819A00A03110F00E94CC56E8ADE03009F0A1C041
:1081AA00E9ADE03019F0E0E00E945D570E946357A4
:1081BA004420B9F5E0911505E03041F4E12FF0E0F3
:1081CA0034960E94B94BEA0FFB1F03C00E94004C71
:1081DA003F96AFA5B8A9EA0FFB1FBF01A0913205D0
:1081EA00B0E0E7E00E94585AE60FF71F0E946A576C
:1081FA00AEE30E949D45A4E00E949D45E0911505CD
:10820A00E03011F4A12F01C0ABE00E949D45E0913E
:10821A003205E795E0E0E7950E946F57AFA50E9407
:10822A007657E1E0E41509F05CC04424A0911905F1
:10823A00B0E0E2E0F0E00E946E5BE0931A05F0E045
:10824A00BC96DF01E0911705F0E0AE0FBF1FE09189
:10825A001805F0E0AE0FBF1FEBA90E948157AE0FC1
:10826A00BF1F0E94BD4FF0E0AE0FBF1F0E94C24F5A
:10827A00F0E0AE0FBF1F0E94C74FF0E0AE0FBF1F66
:10828A00E0911C050E948857F0E0AE0FBF1FE091F5
:10829A004E05F0E00E949357AEE30E949D45ACE282
:1082AA000E949657ABA90E949D45A0911A050E946B
:1082BA00A0570E94FA4F0E949D450E9404500E94B6
:1082CA009D450E94064D0E94A657A0914C050E940A
:1082DA009D45A0914D050E949D45A0914E050E9485
:1082EA007657A8ADA13009F075C0A9ADA13019F033
:1082FA00E1E00E945D570E946357E0913205EE0F5C
:10830A00EE0FE0933205EF5FE0933205AFA5B8A90F
:10831A00A93CE0E0BE0710F00E94CA50AFA5B8A978
:10832A00E5E00E944B5BEFA7F8AB0E94B94BE5E092
:10833A000E944B5B0E94B44BE0913205AFE2EA2700
:10834A00A0911B05AE27E1E0AE27E6E3AE27E8A938
:10835A00F070EA27AFA5B8A9AE27BF27E091FE06BD
:10836A00F070EA27FB270E94B94BAE27BF27E1E04E
:10837A00F0E0AE27BF27E6E3F0E0AE27BF27EBA980
:10838A00F0E0AE27BF27E12FF0E0EA27FB270E94A3
:10839A006A57AFE20E949D45A09132050E949D4511
:1083AA00A0E00E94A0570E94AC57A8A90E949D4530
:1083BA00AFA50E949D45E091FE060E946F570E945C
:1083CA00AC57A0E00E949D45ABA90E949D45A12FF4
:1083DA000E94B257A8ADA33009F09AC0A9ADA33044
:1083EA0019F0E3E00E945D57E8E9E093C1004420F8
:1083FA0009F049C0E0911505E03051F4E12FF0E0B1
:10840A003596DF01E0914F05F0E0AE0FBF1F05C0C2
:10841A00E0914F05F0E07096DF01E0915005F0E041
:10842A00AE0FBF1FE0915105F0E0EA0FFB1F0E945B
:10843A00B94BEA0FFB1FAFA5B8A90E949357AEE646
:10844A000E949D45A5E00E949D45E0911505E030FA
:10845A0011F4A12F01C0ABE00E949D45A0914F05E8
:10846A000E949D45A09150050E949D45A0915105ED
:10847A000E949D45A091FD060E949D45AFA50E94C0
:10848A00B8570E94B257E1E0E41509F041C044240C
:10849A00E0911705F0E0BD96DF01E09118050E9412
:1084AA0088570E948157AE0FBF1FD296E0911C05D4
:1084BA00F0E0AE0FBF1FE0911605F0E0EA0FFB1FD8
:1084CA007E2F8F2FAB8DBC8DEAE00E944B5BE70FAE
:1084DA00F81F0E946A57AEE62BD3ADE20E94965768
:1084EA00A0914D0525D3A0914C050E94A057A2E367
:1084FA000E94B8570E94A657EB8DAAE0EA9FF001A6
:10850A00AE2F16D3A09116050E94B8570E94B257F3
:10851A00A8ADA43009F009C3A9ADA43039F0E4E04C
:10852A00E9AFECE0E093C4000E94254AEFE0EAAB31
:10853A00E9A9F0E0E651FA4FE081E03019F4E9A93F
:10854A00EF5FE9ABA9A9A43010F0E0E0E9ABA9A973
:10855A000E9404480E94BF5711F0E1E0E9ABA9A9C3
:10856A000E942F4A0E94C65711F0E2E0E9ABA9A97E
:10857A000E94014D0E94CD5711F0E3E0E9ABA9A991
:10858A000E940B4D0E94D45711F0E0E0E9ABA9A973
:10859A000E9404480E94BF5711F0E1E0E9ABA9A983
:1085AA000E942F4A0E94C65711F0E2E0E9ABA9A93E
:1085BA000E94014D0E94CD5711F0E3E0E9ABA9A951
:1085CA000E940B4D0E94D45711F0E0E0E9AB442021
:1085DA0009F0CDC1E091F305EF5FE093F305A091B7
:1085EA00F305A23018F0E0E0E093F305E091F0051E
:1085FA00E093F405E091F105E093F505EAE60E94BF
:10860A00DB57DF01E0E0F6FCE1E00E94E957DF0119
:10861A00EC91EE0F0E94E9570F01A081E0E021FCE6
:10862A00E1E0EA0FD0010E94E957DF01EC91E295FF
:10863A00E07F0E94E9570F01E081AAA9EA0FD00161
:10864A000E94E9570E94EF570E94E9570F01E08103
:10865A00A9A90E94F457A0914F050E94FC5733968E
:10866A000E94EF570E940158A091FB060E94F457FE
:10867A000E94EF570E940158A091FC060E94F457ED
:10868A000E94EF570E9409583396DF01EC91E10FDF
:10869A00EC93E091F806E03059F40E940E58A0914C
:1086AA0050050E94FC573596A0915105A0830BC036
:1086BA000E94CA50E0E0DE01A15BBF4FEC93DE01ED
:1086CA00A05BBF4FEC93AFA5B8A90E941F5C08F04E
:1086DA0042C0E0E0DE01AF5ABF4FEC93A0914805DB
:1086EA000E9404480E94135839F0FE01E55BFF4FCF
:1086FA003796AFA5A08305C0E0E0DE01AE5ABF4FB2
:10870A00EC93A09148050E942F4A0E94135839F011
:10871A00FE01E55BFF4F3896AFA5A08305C0E0E0F8
:10872A00DE01AD5ABF4FEC93A09148050E940B4D54
:10873A00A09148050E94FD5059F0FE01E55BFF4FEC
:10874A003996AFA50E94FC573A96AFA5A08302C0FE
:10875A000E941A5845C0E0EFDE01AF5ABF4FEC93B2
:10876A00A09147050E9404480E94245841F0FE0146
:10877A00E55BFF4F3796A091FD06A08305C0E0E0B8
:10878A00DE01AE5ABF4FEC93A09147050E942F4AD3
:10879A000E94245841F0FE01E55BFF4F3896A091F4
:1087AA00FD06A08305C0E0E0DE01AD5ABF4FEC93A1
:1087BA00A09147050E940B4DA09147050E94FD50CC
:1087CA0069F0FE01E55BFF4F3996A091FD060E9414
:1087DA00FC573A96A091FD06A08302C00E941A583F
:1087EA00FE01E55BFF4F36967E2F8F2F6081E09169
:1087FA001505AFE0EA02F001E60FA72FB82F0E9495
:10880A0009583B96A091F2050E94FC573B96DF015E
:10881A00EC91E295E07F0E9409583B960F01E081B6
:10882A00A091F3050E942B583C96DF01FE01EA5AFB
:10883A00FF4FE081F0E0EC50FA4FE081EC930E94A8
:10884A002E580E9438583F3030F40E943F580E94F8
:10885A0047583F5FF8CFE8E8E093C10030E03F3087
:10886A0030F40E943F58AC9163D13F5FF8CFA0919A
:10887A000D075ED18CED95E00197F1F7E0E9E09301
:10888A00C10030E0333008F04DC0E32FF0E0E6518C
:10889A00FA4FA081A43008F443C0E32FF0E0EA5273
:1088AA00FA4F0E944E58E652FA4F0E944E58E25230
:1088BA00FA4F0E944E58EE51FA4F0E944E58DE016E
:1088CA001F96EE0FFF1F0E943C4FED93FC93E32F80
:1088DA000E941B570E943C4FED93FC93E32FF0E05C
:1088EA00EE5AFA4F0E944E58EA51FA4FA0E0A0837E
:1088FA00E32FA6E9B7E0F0E0EE0FFF1F0E943C4F1E
:10890A00ED93FC93E32F0E9448570E943C4FED934E
:10891A00FC93E32F0E944E570E943C4FED93FC9329
:10892A003F5FB0CFE9A9F0E0E651FA4FA081A53048
:10893A0038F4A9A9B0E0A651BA4FEC91EF5FEC93D5
:10894A00A091EA05E3E00E94C45A0E2EA091EB051D
:10895A00E3E00E94C45A0E22A091EC05E3E00E94D3
:10896A00C45A0E220E94D45711F00E94CC4FE1E063
:10897A00E41509F0DAC0E8E8E093C100ECE60E94E9
:10898A00DB57A0911705A083E0E0DE01A25BBF4F91
:10899A00EC930E9453580E9409583396DF01EC91D8
:1089AA000E94095833960E94EF570E940158A091DD
:1089BA004D050E94F4570E94EF570E9409583396BA
:1089CA000E94FF4F0E9453580E940158A091F90635
:1089DA000E94F457DF01EC91EE0F0E940158A0911A
:1089EA004E05EA0FD001EC93E1E0DE01A15BBF4F37
:1089FA00EC930E940E580E945B5834960F01E08156
:108A0A00A09118050E942B5834960E945B58349600
:108A1A000E94FF4F0E940E580E945B5834960F0125
:108A2A00E081A0911C050E942B5834960E945B5845
:108A3A003496DF01EC910E94095834960E94EF5750
:108A4A000E94095834960F01E081A0914A050E94BC
:108A5A002B583596FF93EF930E945F580E946558F2
:108A6A00AF91BF910E94B2580E9409583696FF935F
:108A7A00EF930E945F580E946558AF91BF910E9480
:108A8A00B2580E9409583796A0912D070E94FC57A8
:108A9A0038960E946E58A9A5EA1BDB010E94095864
:108AAA0039960E946E58ADA10E94135CEA1BDB0145
:108ABA000E9409583A96A09116050E94FC573B96C7
:108ACA00A0914D070E94FC573C96A0914905A083AE
:108ADA000E942E58E0914A05EF5FE0934A05A09163
:108AEA004A05A43020F04424E0E0E0934A050E94BD
:108AFA0038583F3030F40E943F580E9447583F5F31
:108B0A00F8CFE8E8E093C10030E03F3030F40E944B
:108B1A003F58AC910DD03F5FF8CFA0910D0708D018
:108B2A000E944B4FE0E9E093C1000C946B06FFCF23
:108B3A00AA93E091C000E072E1F3E881E093C600F5
:108B4A0021960895BA93AA931A93689434F8E7E0A1
:108B5A00E0933408E0E0E0933D08E0933E08E093B8
:108B6A003F08E0934008419A409AE093BC00E091A4
:108B7A00B900EC7FE093B900E981FA81A0E7B7E197
:108B8A000E945B5B1E2F183008F018501093B80033
:108B9A00E091BC00E078E564E093BC00188123967C
:108BAA000895AA93249734FE66C0EA85EE0FE093EF
:108BBA003508E885F985E0933608F0933708E0E050
:108BCA00E0933208EF81E0933808ED81FE81E0936B
:108BDA003908F0933A08E0E0E0933308EC81E09337
:108BEA003B08E6E0E09334087894EF81E03081F0C6
:108BFA00E885F985309709F43EC0EC81E03021F030
:108C0A00AD81BE81109709F001C035C068940DC0CE
:108C1A00EC81E03051F1ED81FE81309761F1E09114
:108C2A003508E160E0933508E89433F8E89434F8BD
:108C3A00E091BC00EF70E06AE093BC00E0E2F1EA88
:108C4A0067E070E00E94005C34FC0FC00E94F65B93
:108C5A003197604070400E94005C31F4E5E0E09397
:108C6A003408689434F807C0EFCFA0913408E0E0E4
:108C7A000E94A65A01C0E0E02B9608950A921A9221
:108C8A00FA926A937A938A939A93AA93BA93EA93F3
:108C9A00FA93EFB7EA930E94385C10913308009177
:108CAA0032083091380820913408E12FA091390810
:108CBA00B0913A08F0E0EA0FFB1FAF01E091B9006A
:108CCA00E87FE83011F420E002C0E03119F4E091C5
:108CDA00350810C0E83111F0E83249F5031798F465
:108CEA00E02F0F5FA0913608B0913708F0E0AE0F81
:108CFA00BF1FEC91E093BB00E091BC00EF70E0680D
:108D0A00E093BC0013C0E0913B081E1770F4E09199
:108D1A003508E160E0933508E89433F8E091BC0047
:108D2A00EF70E06AE093BC0013C138C011C1E035AE
:108D3A0031F4E091BB00DA01EC931F5F02C0E0342A
:108D4A0089F4E0913B08E1501E1728F0E091BC003D
:108D5A00EF70E06804C0E091BC00EF70E06CE09353
:108D6A00BC00F6C0E83531F4E091BB00DA01EC93BF
:108D7A001F5F02C0E03209F402C0E03309F402C006
:108D8A00E83469F4203051F433FE03C0031728F0A5
:108D9A0005C0E0913B081E1708F424E0D1C0E8336F
:108DAA0031F422E0E091BC00EF70E068CDC0E83613
:108DBA0011F0E83711F422E005C0E03611F0E0378F
:108DCA00A9F420E010E0E89433F8E0913C08E030A0
:108DDA0031F421E0E091BC00EF70E06804C0E0915A
:108DEA00BC00EF70E06CE093BC00B2C0E03811F058
:108DFA00E03941F533FE02C021E0A2C0E091BB0098
:108E0A00DA01EC931F5FE0913C081E17C0F4E09171
:108E1A003D08F0913E08309711F426E091C0A0E099
:108E2A00E0913D08F0913E080995E03039F0E09173
:108E3A00BC00EF70E06CE093BC008AC002C068948A
:108E4A0033F802C0E83809F402C0E83939F4E0918D
:108E5A00BC00EF70E068E093BC007AC0E03AB9F475
:108E6A00E091BC00EF70E06CE093BC00689434F8C9
:108E7A00E0913D08F0913E08309739F0A1E0E09189
:108E8A003D08F0913E08099501C026E061C0E03B2B
:108E9A0011F422E002C0E83AB9F4E0913F08F091F7
:108EAA004008309759F0A0E0E0913F08F09140085F
:108EBA0009953E2FE03011F020E002C026E040C0C4
:108ECA0000E0E89433F802C0E83B01F533FE02C043
:108EDA0021E036C0E02F0F5FA0913608B091370825
:108EEA00F0E0AE0FBF1FEC91E093BB00031728F42C
:108EFA00E091BC00EF70E06C06C0689433F8E09132
:108F0A00BC00EF70E068E093BC0022C0E03C11F0C6
:108F1A00E83C99F4E091BC00EF70E06CE093BC008F
:108F2A00E0913F08F0914008309731F0A1E0E091DC
:108F3A003F08F0914008099509C0E03049F423E060
:108F4A00E091BC00EF70E06DE093BC00689434F8E7
:108F5A00109333080093320820933408309338086A
:108F6A000E943F5C2696E991EFBFF991E991B99188
:108F7A00A9919991899179916991F990199009909A
:108F8A001895E0E0E7BDE8BD0895E0E0E0936205EA
:108F9A00E8E6EA93E2E6F5E0FA93EA93E1E0EA9397
:108FAA00E4E6F5E0FA93EA930895E0E0E0936405D5
:108FBA00E0936505E09366050895E8E6EA93E4E63A
:108FCA00F5E0FA93EA930895E4E0EA93E0E0F0E04A
:108FDA00FA93EA93A0E00C94D645E0E0E0936205A8
:108FEA00E0936305E0E5EA93E2E6F5E0FA93EA93B3
:108FFA00E2E0EA93E4E6F5E0FA93EA930895E0E022
:10900A000E94A65A0E2E0895E0936F05E0E0E093C1
:10901A0070050895E0937505E0E0E0937605E09326
:10902A007705E09378050895E0938305E0E0E093FF
:10903A008405E09385050895E0938905E0E0E093CF
:10904A008A05E0938B050895E0938F05E0E0E093AD
:10905A009005E0939105E0939205E0939305E093E0
:10906A009405E0939505E0939605E0939705089596
:10907A00E0939B05E0E0E0939C05E0939D05E09377
:10908A009E05E0939F050895E093A405E0E5EA9321
:10909A00E4E6F5E0FA93EA93E1E4EA93E0E0F0E04B
:1090AA00FA93EA93A0E00E94D645AAE0B0E00E94B3
:1090BA007558E0E0E0936405E6E4E09365050895F9
:1090CA00E0936605E0E0E0936705E0936805E093C6
:1090DA0069050895E0E0E0937105E093720508954B
:1090EA00E0E0E0937905E0937A05E0937B05089543
:1090FA00E0E5EA93E4E6F5E0FA93EA930895EA9361
:10910A00E0E0F0E0FA93EA93A0E00E94D645AAE0F4
:10911A00B0E00C947558E0E0E0936405EAE5E0936A
:10912A0065050895E0E0E0936405EDE2E0936505E6
:10913A000895E0E5EA93E2E6F5E0FA93EA93089502
:10914A00EBE0E0932308E8EBE09324080895E0932A
:10915A005007F09351070895E0935207F09353078D
:10916A000895FE01EB5BFF4F31960895FE01EB5B1C
:10917A00FF4F32960895FE01EB5BFF4F3396089539
:10918A00E0930907F0930A070895A0910907B0919F
:10919A000A070895FE01EF5BFF4F31960895FE011D
:1091AA00EF5BFF4F32960895FE01EF5BFF4F339658
:1091BA000895AB8DBC8DEA0FFB1F0895FF27662724
:1091CA0077270E94EB580E94F15B0895A091DE0771
:1091DA00B091DF078091E0079091E1070895E0E000
:1091EA00F0E060E873E40E9475590895E093DE07A1
:1091FA00F093DF076093E0077093E10708950E94F8
:10920A009C5A0E94EB580E9425590895E0930F0733
:10921A00F09310070895A0910F07B09110070895D1
:10922A00E0933907F0933A0760933B0770933C0742
:10923A000895A0913907B0913A0780913B07909120
:10924A003C0708950E949C5A0E943A5A0895E09356
:10925A001907F0931A070895A0911907B0911A07F0
:10926A000895A091FA07B091FB078091FC079091AD
:10927A00FD070895E093FA07F093FB076093FC0754
:10928A007093FD070895E0932107F093220708954C
:10929A00A0912107B09122070895E0932D07F0933A
:1092AA002E070895A0912D07B0912E070895E093F7
:1092BA003507F09336076093370770933807089598
:1092CA00A0913507B09136078091370790913807FA
:1092DA000895E8E00E946A5AEACFF0E0F1DFB2CFDF
:1092EA00E6DFEEDFF6CFE0931608F093170808954D
:1092FA00AEEFB7E0662777270E94EB580E94F15B32
:10930A000895E0912307F09124070895A091CA07D0
:10931A00B091CB078091CC079091CD070895E09347
:10932A00CA07F093CB076093CC077093CD070895D3
:10933A00E091CA07F091CB076091CC077091CD07F5
:10934A000895A7E0B7E00E94B258ED93FC93089500
:10935A00DDDFE0E0F0E060E271E4089582DFE0E062
:10936A00F0E060E271E40895E0930C08F0930D08D0
:10937A000895A0910C08B0910D080895E0930E0885
:10938A00F0930F080895A0910E08B0910F08089560
:10939A00E093A807F093A9070895A091A807B091B0
:1093AA00A9070895E0931008F09311080895A09171
:1093BA001008B09111080895E0931208F093130869
:1093CA000895A0911208B09113080895E093140823
:1093DA00F09315080895A0911408B09115080895FE
:1093EA00E0931808F09319080895A0911808B0910D
:1093FA0019080895AF8DB8A1EA0FFB1F0895EF8FE2
:10940A00F8A3E9A3FAA30895EBE0F0E060E070E0C6
:10941A00E0933D07F0933E0760933F077093400740
:10942A00E8EB0895E5E7F0E060E070E0E0933D07DF
:10943A00F0933E0760933F0770934007E0E3089577
:10944A00AAE0B0E00C947558E1E09E2E8E2EBE2E56
:10945A00AE2E0895E1E00E94A65A0E2E0895A0911C
:10946A00C607B091C7078091C8079091C9070895A8
:10947A00E0E0F0E061EE75E40E94C3590895E091DE
:10948A001107F09112070895662777270E94EB5873
:10949A000E94F15B0895E0911D07F0911E0708955F
:1094AA00A091CE07B091CF078091D0079091D107B4
:1094BA000895E0E0F0E060E271E40E94C359089583
:1094CA00A0911107B09112070895E0E0F0E00E9420
:1094DA00ED5A0895A0911D07B0911E070895E091D5
:1094EA00F207F091F3076091F4077091F507089578
:1094FA000E94B258ED93FC930895A091E207B091AF
:10950A00E3078091E4079091E5070895E0E0F0E031
:10951A0068EC72E40E947559DF01CB01A9CFE0E043
:10952A00F0E060E070E00895A0912307B09124076D
:10953A0008950E940A5C0E941E590895A09102088B
:10954A00B091030880910408909105080895E0916C
:10955A003907F0913A0760913B0770913C070895EB
:10956A00A4E6B0E080E090E00E942B5BDF01CB0133
:10957A00E091DE07F091DF076091E0077091E10763
:10958A000E94055C0895E0912107F0912207089551
:10959A000E947559DF01CB010895E0912D07F091E2
:1095AA002E0708950E94B458ED93FC930895E0E0C5
:1095BA00F0E061EE75E40E9475590895A091E607FE
:1095CA00B091E7078091E8079091E9070895E7EEDF
:1095DA00F3E0E0936007F09361070895E091E607EE
:1095EA00F091E7076091E8077091E9070895E09123
:1095FA00EA07F091EB076091EC077091ED07089587
:10960A00A091D207B091D3078091D4079091D50742
:10961A000895A091DA07B091DB078091DC07909159
:10962A00DD070895E0E0F0E060E87FE30895E09167
:10963A003507F0913607609137077091380708951A
:10964A00E0E0E0936405EFE4E0936505A0911A0871
:10965A00B0911B0880911C0890911D08E8E10E94B6
:10966A00765AE0936605E0911A08F0911B0860911A
:10967A001C0870911D080E94915AE0936705E8E062
:10968A000E94765AE0936805E0911A08E09369050A
:10969A002FCDE6E0EA93E0E0F0E0FA93EA93A0E067
:1096AA000C94D645A0912705ECE30E94BF5A089571
:1096BA00E0E00E94C45A0E2E0895A091B207B0911C
:1096CA00B3078091B4079091B50708950E22A02F91
:1096DA00E3E60E94BF5A08950E22A091F806E0E040
:1096EA000E94A65A0895A0911B07B0911C070895DD
:1096FA00E0911907F0911A070895A3E0B0E00E94DB
:10970A007558E7EAE0937A0008950E9435010E94AD
:10971A00875A08950E94005C0895E0910907F09124
:10972A000A070895E0910805A0910905AE17089562
:10973A00E0E01A99E1E08E2EE0E01899E1E0089560
:10974A00E0E00E94A65A0E220895E0E00E94A65A7E
:10975A00E0210895E7EAE0937A00A1E0D6CFE0930A
:10976A00FD06F093FE060895A091FD06B091FE064F
:10977A000895FADFE2E3F0E00E94ED5A0E2E089512
:10978A00AFA5B8A9E2E3F0E00E94ED5A0E2E0895C3
:10979A00EEE1F0E00E94E75A0E2EA52DE1E00E94CC
:1097AA00C45A0E220895EAEFF0E00E94ED5A0E2EF6
:1097BA00A52DE1E00E94C45A0E220895E4E00E9419
:1097CA00BF5AE0210895E0E0E093FD06E093FE062B
:1097DA000895E4E00E94A65A0E2E0895ABADE5E086
:1097EA000E94A65A08950E94235BDF01E6EDF0E08D
:1097FA000E945B5B0895E091FD06F091FE060895D4
:10980A00A2EEB7E00E949C5A0E94EB580E94F15BBC
:10981A000895E885F985E0935C07F0935D0708955C
:10982A000E949C5A0E94EB580895662777270E9447
:10983A00EB580895E0E0F4E0EA1BFB0BF1DFDF01EF
:10984A00CB01EAE9F9E969E271E40E94C359DF014F
:10985A00CB01E0E0F0E068E571E46BCEEEE7F7E01B
:10986A00A0E0B0E0A083B183E0E8F7E0A083B18391
:10987A00E2E8F7E0A083B183E9A9E0300895A09176
:10988A009607B09197071196E2E0F0E00E946E5BAE
:10989A00E0936807F09369070895A0E0B4E00E9496
:1098AA00105CEA1BFB0BBCDFDF01CB01EAE9F9E93B
:1098BA0069E271E40E94C359DF01CB01E0E0F0E004
:1098CA0068E571E436CEA0919807B0919907119690
:1098DA00E2E0F0E00E946E5BE0936E07F0936F07A0
:1098EA000895A0919A07B0919B071196E2E0F0E0E3
:1098FA000E946E5BE0937407F09375070895A09138
:10990A009C07B0919D071196E2E0F0E00E946E5B21
:10991A00E0937A07F0937B0708951196E2E0F0E06E
:10992A000E946E5B0895E0917E07F0917F07EA1727
:10993A00FB070895E0937E07F0937F070895E0916F
:10994A008007F0918107EA17FB070895E0938007E3
:10995A00F09381070895E0918207F0918307EA174F
:10996A00FB070895E0938207F09383070895ADE318
:10997A00B7E0F0E00E94825AAE0FBF1F0895A0918F
:10998A00BA07B091BB078091BC079091BD070895B3
:10999A00E091BA07F091BB076091BC077091BD07CF
:1099AA000895E093BA07F093BB076093BC077093DE
:1099BA00BD070895E0910F07F09110070895E0910F
:1099CA00B207F091B3076091B4077091B507089593
:1099DA00A6DD0E94345A0895E093C207F093C307A4
:1099EA006093C4077093C5070895E0E00E94A65AE1
:1099FA006DCEA0911505A9CEE2E00E94A65A0E2EC0
:109A0A000895DE01A85BBF4FAC910895E3E00E9480
:109A1A00A65A0E2E0895F297ADE7B0E00E94235B96
:109A2A000F010895F0E0DE01AF5BBF4FAE0FBF1F1D
:109A3A00EC91F0E0D0010E945B5B0895F0E0DE015A
:109A4A00AB5BBF4FAE0FBF1FEC91F0E008958CDE09
:109A5A000E94235BDF010895E4E6F0E00E945B5B6D
:109A6A000895E12FF0E0DE01DD96AE0FBF1F0895E5
:109A7A00A091AA07B091AB078091AC079091AD076E
:109A8A000895E8EEF3E060E070E00E94985BDF0181
:109A9A00CB01B1DE662777270895EC91F0E0A0E4C8
:109AAA00BCE90E945B5BE4DF662777270895E093B1
:109ABA00AA07F093AB076093AC077093AD070895BC
:109ACA00D7DFDFCF0E943F5AE5E0F0E060E070E0C8
:109ADA000E94035B08950E943F5AE4E1F0E060E0CF
:109AEA0070E00E94FB5A08950E943F5AA431E0E0B8
:109AFA00BE07E0E08E07E0E09E07089560DFA0E57C
:109B0A00B4E180E090E00E94565BD1CFE8EEF3E04A
:109B1A0060E070E00895A02FE3E60E94BF5A08951E
:109B2A00A0E0F0FCA1E011CEE0910608F091070850
:109B3A0060910808709109080895A0910608B091EB
:109B4A000708809108089091090808950DDEE0E061
:109B5A00F0E00E94C95A0895E0E0E0930608E09315
:109B6A000708E0930808E09309080895E89423F8A1
:109B7A00E0E0E09329050895F7DDA7CC0E22DDDFAA
:109B8A00E0E0F0E068E473E40E942E5A08950E22A1
:109B9A00A0E021FCA1E0E1E00E94A65A0895E1E0DC
:109BAA000E94A65AE0210895BFDFA0E0B0E080E855
:109BBA009FE308950E942559E0930608F093070849
:109BCA0060930808709309080895B7DF01CF0E94CF
:109BDA001E59E0930608F0930708609308087093EB
:109BEA0009080895A0E023FCA1E034CCA8ADE3E085
:109BFA000E94BF5AE0210895E0933705B7CFE0915C
:109C0A003307F091340759DD6627772708950E2E1A
:109C1A0094DF08DD0E94345A08950E2EAFA5B8A924
:109C2A00E0E0F0E00E94C95A0E22089586DF0E9401
:109C3A00235C08950E2EA0E020FCA1E081CDA09126
:109C4A003005E2E00E94A65AE021E1290895E09158
:109C5A000605F0E0359788DD0E94E75A0E2EE0915E
:109C6A0036052BDDFF27662777270895A0E021FC1C
:109C7A00A1E06BCDE9A5FAA50E94FB5B66277727D1
:109C8A000E94135B0E2EEAE0F0E060E070E00E94B2
:109C9A001B5B0E2208950E94F65BA9A5BAA5882728
:109CAA0099270E943F5A0895A630E0E0BE07E0E0F7
:109CBA008E07E0E09E070895A0915007B0915107E2
:109CCA000895E0915007F09151070895E9A5FAA582
:109CDA000E94FB5B6627772708950E2EA8AD6ECDEE
:109CEA00EB8DFC8DA885B9850E94ED5A0E2E08953C
:109CFA003BDDEAE00E944B5B0895AB8DBC8DE885A5
:109D0A00F985EA1BFB0B0895A0915207B0915307FE
:109D1A000895E0915207F09153070895A885B985EF
:109D2A00EB8DFC8DEA1BFB0B0895EAE0F0E00E9444
:109D3A006E5B15CDEBA9C1DCFF276627772708954F
:109D4A00E0935A07F0935B070895EBA9F0E0B5DCBE
:109D5A000E949C5A0E943F5A08950E94515BA0910A
:109D6A005A07B0915B070895E0915A07F0915B0793
:109D7A000895ABA9BB2723DE0E94A15A0E943F5A2D
:109D8A000895A8ECB0E0A083B1830895A091590585
:109D9A00BB27E0917E07F0917F07AE1BBF0B0895AA
:109DAA00EAE0F0E00E94D55A0E2E0895A0915905D6
:109DBA00E3E80E94BF5AE0210895E4E1F0E00E943E
:109DCA00515B0895A0E0B0E0A083B1830895A0910B
:109DDA005A05BB27E0918007F0918107AE1BBF0BA4
:109DEA000895A0915A05E7E40E94BF5AE021089518
:109DFA00A0915B05BB27E0918207F0918307AE1B18
:109E0A00BF0B0895A0915B05E5E60E94BF5AE021C9
:109E1A000895AADCEA17FB070895AFA5B8A9E2E3FB
:109E2A00F0E00E94ED5A0E2EA09130050895E1E06F
:109E3A000E94A65A0E220895EAE0F0E00E945B5BB7
:109E4A0006CEE4E1F0E00E945B5BEFA3F8A7089579
:109E5A00ED8DFE8DAB8DBC8DAE0FBF1F0895EAE070
:109E6A00F0E00E945B5B0895AFA5B8A92ECBAE0FB8
:109E7A00BF1FE0E0F0E008950E22A02FE3E60E9463
:109E8A00A65AE0210895E093670532C9A1E0B0E03F
:109E9A000C9475589BD9E0E0F0E060E873E40E9406
:109EAA00C3590895E091DE07F091DF076091E0075A
:109EBA007091E1070E94B258EC930895E0E0F0E057
:109ECA0060E873E40E94C35908951BDA0CDA23C9C7
:109EDA00A0914C05E3E00E94BF5AE0210895E09169
:109EEA00EF05E09350050895E1E0E0933205A09173
:109EFA002B05A2300895E0913305F0E0E05EFA4FB9
:109F0A00E081E7BDE0E0E8BD0895A0914C05E4E0FA
:109F1A000E94A65AE0210895A0914C05E5E00E940E
:109F2A00A65AE0210895E0913305F0E0E05EFA4F89
:109F3A000895C3DBF4DA0E94035B0895E0910505F6
:109F4A00E170AFEFEA02F0010895EBA1FCA1AF893D
:109F5A00B88DEA17FB070895E0910F05F0E0E65F78
:109F6A00FA4F0895E0E0E0936405E09365050895EB
:109F7A00FE01EA5BFF4FE0810895FE01E95BFF4FB6
:109F8A00E0810895FE01E85BFF4FE0810895E0E07B
:109F9A00E093EA05E093EB05E093EC05E093ED0529
:109FAA000895A02FE3E60E94A65AE0210895E091C1
:109FBA003F05EF5FE0933F05E0913E05A0913F0525
:109FCA00EA170895E0931905F0E02ADCACE5BFE84A
:109FDA0082E290E40E947559A3ECB5EF88E490E41C
:109FEA000E947559AFE0B7E083CADE01AA5BBF4F92
:109FFA00AC910895DF01EC91EF5FEC930895DE01D7
:10A00A00A95BBF4FAC910895DF01EC91EB5FEC9334
:10A01A00089548D9E8E1F0E00E94C95A0E2EA9A590
:10A02A00BAA50895E0211E2E3DD9E4E2F0E00E948F
:10A03A00C95A0E2EA9A5BAA50895E0211E2A32D919
:10A04A00E0E3F0E00E94C95A0E2EA9A5BAA5089528
:10A05A00AC85E9E10E94A65A0E2EA0914705089503
:10A06A00AB8DBC8DA43FE1E0BE070895EB8DFC8D5E
:10A07A003A96EB8FFC8F0895E2E00E94A65AE021FF
:10A08A000895EB8DFC8DED8FFE8F0895E3E00E941D
:10A09A00A65AE0210895E4E00E94A65AE021089514
:10A0AA00B5D888DCC2DBDF01CB01ECE5FFE862E270
:10A0BA0070E40E94C359DF01CB01E3ECF5EF68E4D9
:10A0CA0070E40E94C359A9E1B5E00E94B258EC932A
:10A0DA000895A0910105B0E0EAE0F0E00E946E5B0D
:10A0EA000895A0910105BB27EAE0F0E00E94A05B79
:10A0FA000895E3E0EA93E0E0F0E0FA93EA93A0E05F
:10A10A000C94D645AC85EFE30E94A65A0E2EEBA11D
:10A11A00FCA1AF89B88D0895DE01A75BBF4FAC9152
:10A12A000895FE01E75BFF4FE0810895A091330592
:10A13A00B0E0A05EBA4FEC910895AC85E3E60E94C8
:10A14A00A65A0E2EEBA1FCA1AF89B88D0895DF01A6
:10A15A00EC91E150EC930895DF01EC91E550EC931A
:10A16A000895EB8DFC8D3A97EB8FFC8F0895B0E044
:10A17A00EAE0F0E00E946E5B0895A0910205BB2719
:10A18A00EAE0F0E00E94A05B0895E8ECF0E0EFA7B7
:10A19A00F8AB0895EDA1FEA10E94FB5B6627772725
:10A1AA0008950E94FB5B0895A885B985EAE0F0E06E
:10A1BA000E946E5B0895A0917E07B0917F07089573
:10A1CA000E94ED5A2ACDA0918007B0918107089587
:10A1DA00A0918207B09183070895DF01E4E6F0E0D9
:10A1EA000E946E5B0895A0919E07B0919F07089503
:10A1FA00E4E00E94A65AE0290895FE01E65BFF4FBB
:10A20A00E0810895DE01A65BBF4FEC930895DE015D
:10A21A00A259BF4FEC930895DE01A159BF4FEC93A9
:10A22A000895EAE0DE01A059BF4FEC930895DE01DC
:10A23A00AF58BF4FEC930895DE01AE58BF4FEC9371
:10A24A000895DE01AD58BF4FEC930895EAE0DE01B0
:10A25A00AC58BF4FEC930895EAE0DE01AB58BF4F0C
:10A26A00EC93DE01AA58BF4FEC93DE01A958BF4F09
:10A27A00EC93DE01A858BF4FEC93DE01A758BF4FFD
:10A28A00EC93DE01A658BF4FEC93DE01A558BF4FF1
:10A29A00EC93DE01A458BF4FEC93089559E0E09186
:10A2AA003905E170EE0FAE2FE0913905E695E170C0
:10A2BA00EE0FEE0FEE0FEA0F0E2E0895E09139051C
:10A2CA00E695E695E170AE2FE0E0F5FCE1E0EA2BD9
:10A2DA00EE0FEE0FE00D4E2F08955E2FE091390537
:10A2EA00E170EE0FAE2FE0913905E695E170EE0FC1
:10A2FA00EE0FEE0FEA0F0E2EE1CFE295E07FEE0FA2
:10A30A00EE0F0895E0E0F799E1E0E0930305AD85EB
:10A31A00BE850895A436E0E0BE07E0E08E07E0E0DF
:10A32A009E070895E093B207F093B3076093B407CA
:10A33A007093B5070895A73FEFEFBE07EFEF8E07BB
:10A34A00EFEF9E070895AA30E0E0BE07E0E08E072F
:10A35A00E0E09E070895B1D9EAE0F0E060E070E03D
:10A36A0008950E94985BDF01CB01EAE0F0E060E02B
:10A37A0070E00E94B25B0895FE01E359FF4F3496E4
:10A38A000895DE01A059BF4FEC9308950E94485AE0
:10A39A00DF01CB01EAE0F0E060E070E00E94B25B2E
:10A3AA000895EAE0F0E00E946E5B0895E0935E078C
:10A3BA00F0935F070895A0915E07B0915F07089533
:10A3CA00FE01E359FF4F3196BF01F5DFEACFDF0106
:10A3DA00EAE0F0E00E94A05BDB01EC930895FE0145
:10A3EA00E359FF4F32960895BF01E5DFEAE0F0E056
:10A3FA000E94A05BDB01EC9308950E94445ADF019E
:10A40A00D0CFE0912C05ACE7B7E0F0E0EE0FFF1FEC
:10A41A00AE0FBF1F0E94E75B0895FE01E359FF4F8D
:10A42A0035960895E4E6F0E00E946E5BD0CFFE0117
:10A43A00E359FF4F36960895FE01E359FF4F3796C9
:10A44A000895EAE0F0E00E94A05BDB01EC93089536
:10A45A00DE01AC58BF4FEC930895A0E0F799A1E054
:10A46A00EA2FE295E07F4E0F0895A0910707B09179
:10A47A0008070895FE01E359FF4F3D96BF01F5CF46
:10A48A00E8EEF3E00E945B5BDF01EAE0F0E00E94A5
:10A49A009D5BDB01EC93FE01E359FF4F0895DF0159
:10A4AA00EAE0F0E00E949D5BDB01EC930895FE0177
:10A4BA00E359FF4F3F96BF01D8CFFE01E359FF4F43
:10A4CA003E9608950E949D5BDB01EC930895E2E0BD
:10A4DA00DE01AB58BF4FEC930895FE01E359FF4FDD
:10A4EA003996BF010895FE01E359FF4F3A96089540
:10A4FA00FE01E359FF4F3B9608950E94735BDF010B
:10A50A00CB01EAE0F0E060E070E00E94AE5B089503
:10A51A00A031E7E2BE07E0E08E07E0E09E0708957B
:10A52A00A83EE3E0BE07E0E08E07E0E09E0708955C
:10A53A00FE01E359FF4F3C960895FE01E359FF4F90
:10A54A003D960895E4E6F0E060E070E008950E9428
:10A55A006549EAE0F0E060E070E00895FE01E35941
:10A56A00FF4F3F960895DE01AA58BF4FEC93E4E7E8
:10A57A00DE01A958BF4FEC930895A091B607B09198
:10A58A00B7078091B8079091B9070895F6DFEAE016
:10A59A00F0E060E070E00895E091B607F091B70747
:10A5AA006091B8077091B9070895E0E4DE01A558F3
:10A5BA00BF4FEC930895F0DF0E94485ADF01CB01A8
:10A5CA000895EAE0F0E060E070E00895E0E4DE017A
:10A5DA00A658BF4FEC930895E0E4DE01A758BF4F99
:10A5EA00EC930895E0E4DE01A858BF4FEC93089578
:10A5FA00E4E4DE01A858BF4FEC93E1E0DE01A7587E
:10A60A00BF4FEC930895A0915807B0915907089548
:10A61A000E946E5BDCCEE8EEF3E0FACFBF01E09178
:10A62A005807F091590708950E94445AD6CDE5E09B
:10A63A000E94A65A0E2E0895E0E5DE01A858BF4FE3
:10A64A00EC930895A0916007B09161070895DE0127
:10A65A00AA58BF4FEC930895DE01A958BF4FEC9357
:10A66A000895E8E7DE01A858BF4FEC930895EFA5D7
:10A67A00F8A9F695E7950895E8ECF0E00E945B5B8F
:10A68A000ECFE4E1F0E00E945B5B09CFEFA1F8A5F1
:10A69A00F695E7950895DE01A758BF4FEC93089504
:10A6AA00EAE0DE01A658BF4FEC930895E7E7DE0122
:10A6BA00A658BF4FEC930895A0911307B0911407C1
:10A6CA000895EAE0F0E0FECEDE01A658BF4FEC9313
:10A6DA000895DE01A558BF4FEC930895E4E5DE0125
:10A6EA00A458BF4FEC930895B7DFE8E3DE01A858FA
:10A6FA00BF4FEC930895E8EEF3E00E945B5BCFCE88
:10A70A000E94D55A0E2E6FCDE7E3A1DFE8E7A4DF5A
:10A71A0093CFE3E6DE01A458BF4FEC930895EAE035
:10A72A00F0E00E94A05BDB010895ECE790DFE7E729
:10A73A0093DF97CFE9E38BDFE8E78EDF7DCFE17028
:10A74A00EE0FEE0FEE0F0895ECE786DF75CFABAD97
:10A75A00E4E00E94A65AAE2FE0E0F799E1E0EA238E
:10A76A000895AE2FE0E0F799E1E0EA230895ECE7D7
:10A77A00ABDFE0E5AECFECE0DE01A458BF4FEC93CF
:10A78A000895DE01A458BF4FEC930895E9E3A1DFD1
:10A79A00EBE0F7CFA0E0F799A1E00C94A54BE0938A
:10A7AA002C055F77EAE053CF76DF7ACFE8E791DFCF
:10A7BA00EBE0E7DFE1E0E09343050895E32FF0E003
:10A7CA00DE01A359BF4FAE0FBF1F08950E94A65ABC
:10A7DA000E2EAC850895EB8DFC8D27D8ADECBCEC24
:10A7EA008CEC9DE30E947559DE019B960C947D4A80
:10A7FA000E941A4CADECBCEC8CEC9DE30E9475599E
:10A80A00DE019B960C947D4A0E94A65A0E2AAC85BC
:10A81A000895AC85E2E30E94A65A0E2EABA5BCA50C
:10A82A00E4EAF1E00895E0E1F7E20E945B5B37CEEB
:10A83A00BF01ABA5BCA513CBFFDCE9E702CD0CDF5A
:10A84A00E4E5DE01A858BF4FEC93089501DEEBA5BD
:10A85A00FCA530970895E0E037DFE1E73ADFE1E76A
:10A86A0090CFE0E036DF3ACFECDCE8E3F1CDE4DC90
:10A87A00E0E3E7CCE9E3E0DCE0E5E3DCEEE30895DE
:10A88A00E7E7DADCE9E3DDCC24DFE9E77ACF21DFA9
:10A89A00E8E777CFDE01A858BF4FEC930895CCDCE8
:10A8AA00E7E7CFCCE3E10E94A65AE0290895E091B8
:10A8BA00FF06F09100070895E0933107F0933207FD
:10A8CA0008950E94235BDF01C7C8E72DF0E0DE018F
:10A8DA00DD96AE0FBF1F0895A091AE07B091AF07E6
:10A8EA008091B0079091B107089510D90E94985BA2
:10A8FA00DF01CB01DCDF662777270895EC91F0E0D2
:10A90A00A0E4BCE90E945B5BE7DF6627772708952E
:10A91A00E093AE07F093AF076093B0077093B10767
:10A92A000895DADFE2CF4BD8A0E5B4E180E090E009
:10A93A000E94565BEDCFE0913107F0913207F69510
:10A94A00E795E0932F07F093300708955BDCA09119
:10A95A002F07B0913007A436E0E0BE070895BF0183
:10A96A00A0912F07B09130070895A0912F07B091B9
:10A97A0030071A970895A0914D0511C90E94235BCB
:10A98A00DF016DCAE0932F07F09330070895E72D92
:10A99A00F0E0DE01AB5BBF4FAE0FBF1F6C917727B4
:10A9AA000895BF01A0911F07B09120070895A091B3
:10A9BA000B07B0910C070895A0911707B0911807DB
:10A9CA0008953FDC39CD67DEE0E07ECEE8E534DC91
:10A9DA00E4E537CCEDE630DCE8E333CC32DCE8E71B
:10A9EA0037CD2ADCEEE52DCC27DCE8E32ACC24DCC3
:10A9FA00E5E03ACFE0E06DDEE0E0C3CEE0E04BDE3A
:10AA0A00E1E062DEF7CFE1E046DEE1E05DCEE1E0E3
:10AA1A0060DEE1E0B6CEEAE05CDEEAE0B2CEA0912A
:10AA2A000107B091020708950E94C45A0E2E74CBF2
:10AA3A000EDEECE711CE2EDF80CDDF0172DBF0E017
:10AA4A003897EE5AFA4FE0810895DF016ADBF0E0A9
:10AA5A003C97EA51FA4FE0810895E695E695E69526
:10AA6A00E1700895E9DBE3CCBF015BDBF0E07097AE
:10AA7A00A5E2B7E0EE0FFF1FAE0FBF1F0E94E75B14
:10AA8A00DF010895BF014DDBF0E00895EE0FFF1FCF
:10AA9A00AE0FBF1F0E94E75B089543DBF0E0749797
:10AAAA00DE011F96F3CF7497DE011F96EFCFFE01EA
:10AABA00E658FF4FE0810895CADDE3E7CDDDEBE01C
:10AACA00E9CECADDEBE0E6CEE3E603DEE9E359CE02
:10AADA00E170E295E07FAE2F0895FE01EE58FF4F38
:10AAEA00E0810895E295EF70E695E170E295E07FE6
:10AAFA00EE0FEA2BAE2F0895E295EF70E695E695F4
:10AB0A00E170FBDBEA2BAE2F0895E295E170E79541
:10AB1A00E0E0E795EA2BAE2F0895EA2BAE2FDDCFC2
:10AB2A00E695E695E170EE0FEE0F0895E695E69547
:10AB3A00E69505CEEA2BD001EC93FE01E45AFF4FCD
:10AB4A000895AE2FFE01ED58FF4FE0810895FE01F2
:10AB5A00ED58FF4FE0810895FE01EC58FF4FE08168
:10AB6A000895EA2BAE2FF8CFE695E170EE0FEA2BA7
:10AB7A000895FE01EA58FF4FE0810895E695E170D5
:10AB8A00E295E07FEE0FEA2BAE2F0895E695E69563
:10AB9A00E170B3DBEA2BAE2F0895E795E0E0E79585
:10ABAA00EA2BAE2FE52F0895EA2BAE2F80CFE29540
:10ABBA00EF70E695E170EE0F0895E295EF70E69575
:10ABCA00E695E170EE0FEE0F0895FE01E758FF4F8C
:10ABDA00E0810895EA2BAE2FFE01E558FF4FE08190
:10ABEA000895E295EF70E69573CFFE01E858FF4F9E
:10ABFA00E0810895EA2BAE2FF8CFFE01E558FF4F0A
:10AC0A00E0810895E295EF70E695E6950895FE01D4
:10AC1A00E958FF4FE0810895EA2BAE2FFE01E45870
:10AC2A00FF4FE0810895FE01E458FF4FE081089547
:10AC3A00E795E0E0E795EA2BAE2F0895EA2BAE2FD1
:10AC4A00FE01E259FF4FE0810895E170E295E07F4D
:10AC5A00EE0F0895E695E695E170EE0FEA2BAE2F1A
:10AC6A000895E170EE0FEE0FEA2BAE2F0895FE0164
:10AC7A00E159FF4FE0810895E295EF70E695E170A2
:10AC8A00D7CFEA2BAE2FB9CAFE01E059FF4FE081B8
:10AC9A000895FE01EF58FF4FE0810895E32FF0E099
:10ACAA00DE01A45ABF4FAE0FBF1F0895449888E231
:10ACBA008A95F1F731E00895439884E08A95F1F78F
:10ACCA00089584E08A95F1F7439A84E08A95F1F72A
:10ACDA000895429A88E28A95F1F7449A88E28A9519
:10ACEA00F1F7E4CFA09143050C942F4AA0914205B5
:10ACFA000C94A54BE0E00E94A65A0E2A0895EDE4B2
:10AD0A00E093C400A0911E0808950E94A65A0E2E30
:10AD1A00A0911F0808950E94A65A0E22A0912F08FA
:10AD2A000895E0912308FF2766277727E0933D07D8
:10AD3A00F0933E0760933F0770934007E091240821
:10AD4A00E0933A05E0E0E0932F08E09304050895C4
:10AD5A00E0E0E0931E08E0931F08E0932008E093E8
:10AD6A002108E09322080C94A548E0E0E093250826
:10AD7A00E0932608E0932708E0932808E0932F0839
:10AD8A000895E0E0E0932F08E09304050895E0E0D9
:10AD9A00E0931E08E0931F08E0932008E09321083F
:10ADAA00E0932208E0932308E0932408E09325081F
:10ADBA00E0932608E0932708E0932808EBE0E09365
:10ADCA002908E8EBE0932A08E0E0E0932F080895C9
:10ADDA00EC93A1E2B8E0EC910895E695E695EC9340
:10ADEA00A091D505B0E00895E0912108E170F0CF77
:10ADFA00EC93A091D505B0E00895E091D505F0E077
:10AE0A00DE011F96EE0FFF1F0895EA0FFB1F0F01C9
:10AE1A00DF010E94E75BDF010895F0E0EA0FFB1F04
:10AE2A00D001ED93FC93E091D5050895A5E2B7E032
:10AE3A00F0E0EE0FFF1F0895ED93FC93E091D50526
:10AE4A000895EC93E091D505A6E9B7E0F0E0EE0F9E
:10AE5A00FF1F0895AE0FBF1FE0912908F0E0E370CD
:10AE6A00F070EACFF0E0EE0FFF1FAE0FBF1FED91BB
:10AE7A00FD91FE2FE0E0FE93EE93A9E2B8E0EC919B
:10AE8A00E695E6950895AEE8B7E0F0E0EE0FFF1F0D
:10AE9A000895A6E8B7E0F0E0EE0FFF1F0895EE0F61
:10AEAA00EE0FEA0FA0913905EA2BE09339050895D0
:10AEBA00E9AFEDE4E093C4000C94254AE8E9E09395
:10AECA00C100EDE4E093C4000895E0930D07F09308
:10AEDA000E070895AE2F0E949D45A091FD060C9481
:10AEEA009D450E949D45E0910E07AE2F0E949D450B
:10AEFA00A0910D070C949D45F0E0AE0FBF1FE091A5
:10AF0A001B05F0E00895F0E0AE0FBF1FE0914C057D
:10AF1A00F0E0AE0FBF1FE0914D050895EA0FFB1F49
:10AF2A00D4CF0E949D45A09117050E949D45A091EE
:10AF3A0018050C949D450E949D45A0911B050C94F3
:10AF4A009D450E949D45A0911C050C949D45A1E03C
:10AF5A000E949D45A6E30C949D450E949D45A091A3
:10AF6A000D070C949D450E949D45A0E00E949D45B9
:10AF7A00A0E00895A091EA05E3E00E94C45AE02106
:10AF8A000895A091EB05E3E00E94C45AE0210895D8
:10AF9A00A091EC05E3E00E94C45AE0210895A09133
:10AFAA00ED05E3E00E94C45AE0210895DE01A55BA5
:10AFBA00BF4FEC93EFE0DE01A45BBF4FEC93FE01C1
:10AFCA00E55BFF4F32960895EC93FE01E55BFF4F78
:10AFDA0032960895DF01EC91EE0FEE0F0895EA0F15
:10AFEA00D001EC93FE01E55BFF4F33960895A083F1
:10AFFA00FE01E55BFF4F0895EC93FE01E55BFF4F11
:10B00A0033960F01E0810895EC93FE01E55BFF4F53
:10B01A000895FE01E55BFF4F34960895A091480517
:10B02A00E2E00E94A65A0E2AE3C8E0E0DE01AC5A2A
:10B03A00BF4FEC93DE01AB5ABF4FEC930895A0913A
:10B04A004705E2E00E94A65A0E2AD2C8EA0FD001AA
:10B05A00DBCFE0E0DE01A85ABF4FEC93DE01A75A2E
:10B06A00BF4FEC930895E0E0E0930D07E0930E07DD
:10B07A0031E00895E32FF0E0DE01A55BBF4FAE0F8C
:10B08A00BF1F0895EC91F0E0A0910D07B0910E0753
:10B09A0045CFA0E0A083E32FF0E00895FE01E55B31
:10B0AA00FF4F3396DF01EC91EE0F0895DF01EC912B
:10B0BA00EE0FAACFE0914A05F0E0DE015B96E6CCFE
:10B0CA000E941A4CADECBCEC8CEC9DE30E947559C5
:10B0DA000895BF01E0912D07AAE0EA9FF0010895C3
:10B0EA00109639F088EB9BE00197F1F7A895119734
:10B0FA00C9F7089530976040704009F07058089574
:10B10A00552342F4503811F4E0FF04C03196691F08
:10B11A00791F6BF050E8572711F45F93CFC05F3F58
:10B12A0031F0660F000C57956795752F08955F9358
:10B13A0000200AF0CFC0C8C050E8192E1522880F87
:10B14A00991F9527550F879550E8072E0522660FF8
:10B15A00771F7527550F67950895689401C0E8947D
:10B16A005F93F2DF703818F07F3F08F4A7C056E10A
:10B17A00571BAAF4519558300EF4593030F0EFEFBE
:10B18A00FFEF6FEF7FE777F91AC077275523B9F0FA
:10B19A00EE0FFF1F661F771F5A95D1F710C077274A
:10B1AA00583028F0EF2FF62F672F5850F9CF552334
:10B1BA0031F076956795F795E7955A95D1F700207E
:10B1CA000AF461D15F910895689401C0E8943097B8
:10B1DA0060407040B1F0002426F0772312F4009406
:10B1EA0052D1172E7EE1112032F07A95EE0FFF1F11
:10B1FA00661F111CF9CFEF2FF62F612D5F938ADF9F
:10B20A005F9108954F93AF01FD01DA01AB01BC01D3
:10B21A00CA01402D012C142E4F910895EA0FFB1FED
:10B22A00681F0895E095F0956095EF5FFF4F6F4FA7
:10B23A0008955F9381DF903871F150E8152604C0B4
:10B24A005F937ADF903839F1703821F1572F591B03
:10B25A002BF112F4D7DFFACF583118F0AA27BB27FF
:10B26A008827583028F0AB2FB82F88275850F9CFA5
:10B27A00552329F08695B795A7955A95D9F7502D54
:10B28A00512572F0CBDF38F46795F795E7957395FA
:10B29A0013F420C0B7DF3EDF5F910895D8F7FBCFE4
:10B2AA00EA1BFB0B680B51F010F40094BBDF66231A
:10B2BA0092F3EE0FFF1F661F7A95CBF7EE27FF2753
:10B2CA00662777275F910895EFEFFFEF6FE77FEF2C
:10B2DA005F910895EFEFFFEF6FE77FE75F910895C2
:10B2EA005F932ADF703851F3903841F301240894B0
:10B2FA00791F23F41CF300203AF3ECCF0F921F932B
:10B30A002F933F934F93112722279927689FA001D4
:10B31A008F9F302D410D591F6B9F300D411D591FB5
:10B32A008E9F27D0BF9F25D06A9F23D0BE9F1DD056
:10B33A00AF9F1BD0AE9F110D291F391F491F591FDF
:10B34A00E32FF42F652F522F4F913F912F911F9189
:10B35A000F9066232AF0550FEE1FFF1F661F02C0CB
:10B36A0073954BF2CDDE5F910895100D211D391FA3
:10B37A0002C0200D311D491F591F08955F93DCDE5D
:10B38A00703821F411200AF49FCFA4CF903809F421
:10B39A0095CF01240894970B1BF4D4F30020F3CF24
:10B3AA00792F1F932F933F934F931124112722270D
:10B3BA0033274427552790E2AE17BF078607410770
:10B3CA0030F0AE1BBF0B860B410B089401C088946A
:10B3DA00551F221F331F111CAA1FBB1F881F441F82
:10B3EA009A9551F7F901612D4F913F912F911F9134
:10B3FA00662332F0550FEE1FFF1F661F7A9543F240
:10B40A007FDE5F91089599239AF0772342F0971788
:10B41A0048F029F4AE17BF07860720F031F0989458
:10B42A00889408959894089408951894889408958F
:10B43A007723C2F7971798F3A9F7EA17FB07680764
:10B44A0088F399F3ECCFDFDFE1E011F008F0EE27A3
:10B45A000895D9DFE1E009F008F0EE270895D3DF77
:10B46A00E1E009F008F4EE270895EA0FFB1F681FD0
:10B47A00791F0895AE1BBF0B860B970B0895F195A4
:10B48A00E195F0400895F09560957095E195FF4F2C
:10B49A006F4F7F4F0895EE230E2EEA2F19F0E6958F
:10B4AA000A94E9F70895EE230E2EFD0121F0EE0F1E
:10B4BA00FF1F0A94E1F70895EE230E2EFD0121F0F5
:10B4CA00F695E7950A94E1F70895EE230E2EFD010D
:10B4DA00BC0131F0EE0FFF1F661F771F0A94D1F7E8
:10B4EA000895EE230E2EFD01BC0131F07695679585
:10B4FA00F795E7950A94D1F70895EE0FFF1FEE0F1F
:10B50A00FF1F0895F695E795F695E7950895EF2FAD
:10B51A00FF27E7FDFFEF0895E62FF72F60E070E0C1
:10B52A000895FE2FFF0FFF0B6F2F7F2F08956F2FA8
:10B53A00660F660B762F08958B2F880F880B982F2E
:10B54A000895EA17E1E009F0EE270895EA17E1E025
:10B55A0009F4EE270895AE17E1E00CF4EE270895FA
:10B56A00AE17E1E00CF0EE270895EA17E1E00CF0DF
:10B57A00EE270895AE17E1E008F0EE270895EA17DE
:10B58A00E1E008F0EE270895EA17FB07E1E009F089
:10B59A00EE270895EA17FB07E1E009F4EE2708957C
:10B5AA00AE17BF07E1E00CF0EE270895EA17FB0794
:10B5BA00E1E00CF0EE270895EA17FB07E1E008F452
:10B5CA00EE270895AE17BF07E1E008F0EE270895C9
:10B5DA00EA17FB07E1E008F0EE270895EA17FB07F0
:10B5EA0068077907E1E009F0EE270895AE17BF076B
:10B5FA0086079707E1E00CF0EE270895EA17FB07A4
:10B60A0068077907E1E00CF0EE270895EA17FB07CF
:10B61A0068077907E1E008F4EE270895AE17BF0737
:10B62A0086079707E1E008F0EE270895EA17FB0777
:10B63A0068077907E1E008F0EE270895FA9FF02DF0
:10B64A00EB9FF00DEA9FE02DF10D08957A9F702D82
:10B65A006B9F700DF89F700DE99F700D6A9F602DAA
:10B66A00710DFB9F600D711DE89F600D711D88278C
:10B67A00FA9FF02D610D781FEB9FF00D611D781F69
:10B68A00EA9FE02DF10D681F781F08956E2F6A9FBB
:10B69A00F0016B9FF00D089574D0D0DF0EF4EFDE49
:10B6AA0008957DD0D3DF0EF4EEDE08950024112430
:10B6BA0090E1AA0FBB1F001C111C0E1A1F0A18F4D6
:10B6CA000E0E1F1E01C0A1609A9599F7FD01D001C7
:10B6DA00089557D0EBDF0EF4D2DE08953F934F93CF
:10B6EA005F93002411244427552730E2AA0FBB1F79
:10B6FA00881F991F001C111C441F551F0E1A1F0A70
:10B70A00460B570B28F40E0E1F1E461F571F01C06B
:10B71A00A1603A9559F7FD01BC01D001CA015F91B8
:10B72A004F913F9108953BD0D9DF0EF4ACDE0895D6
:10B73A00BDDFFD010895E894B7FF04C0A095B09558
:10B74A0011966894F7FD9BDEB1DFFD010EF497DEDA
:10B75A000895C4DFFD01BC010895E89497FF09C06C
:10B76A00A095B09580959095AF5FBF4F8F4F9F4F33
:10B77A00689477FD88DEB2DFFD01BC010EF483DE3A
:10B78A000895E894F7FF02C07ADE6894B7FF06C00E
:10B79A00A095B095119600F8039400FA0895E894DC
:10B7AA0077FF02C070DE689497FF0BC00024A09553
:10B7BA00B095809590951196801D901D00F8039480
:10B7CA0000FA0895ED91FC9111970895ED91FD917C
:10B7DA006D917C9113970895ED93FD936D937C93EE
:10B7EA000895E881F9816A817B810895A881B981E8
:10B7FA008A819B810895E883F9836A837B8308950C
:10B80A00689401C0E89401D0E2DC182E862F612DDD
:10B81A00192E972F712D1B2EBF2FF12D1A2EAE2FF9
:10B82A00E12D089500240E160F0608953097604002
:10B83A007040089500240A160B06089500240A167B
:10B84A000B06080609060895EA17FB076807790731
:10B85A000895AE17BF07860797070895E894EE2361
:10B86A0009F0689408955A934A933A932A931A933B
:10B87A000A9308955D814C813B812A81198108814F
:10B88A000895AC0FBD1F05900D928A95E1F70895B2
:00000001FF
